:100000000C9461090C94B0090C94B0090C94B009DB
:100010000C94B0090C94B0090C94B0090C94B0097C
:100020000C94B0090C94DA1B0C94B0090C94B00930
:100030000C94D9350C94B0090C94B0090C94B00907
:100040000C94B0090C94B0090C94AE180C94B0093F
:100050000C94DC0E0C94B0090C94A60E0C94B00910
:100060000C94BD1E0C94B0090C945F310C94B00933
:100070000C94D5870C94B0090C94AB800C94B00907
:100080000C94B0090C94B0090C94B009E41EE91E5C
:10009000EE1EF71E0E1F251F351F451F801F6C21EA
:1000A000251F2E203F206E208C20A92003215E21B9
:1000B00079234624D52455258D2530263728A12897
:1000C0001B296429AE29DC29092A6C2AB62A002BAF
:1000D000F92B7E31B231F53165327D32BE32753366
:1000E0003C343C343C343C343C343C343C343C3490
:1000F0003C343C343C34F133F333F83310341234B1
:100100004574DE746375C57519768276197E20771D
:1001100066776A776A776A776A776A776A776A77DB
:100120006A7798771778AC78D17814797079FB79F9
:10013000E47A307B347B347B347B347B347B347B9C
:10014000347B347B6C7B8A7BB27B177C537CC27C98
:10015000EF7C8F7DEF7DF47DF47DF47DF47DF47D87
:10016000F47DF47DF47D0A0D426174743A0020251B
:10017000642043656C6C732000204C6F772077619E
:10018000726E696E67206C6576656C3A2025642E08
:100190002564000A0D466F756E6420424C2D437431
:1001A000726C3A20002564000A0D0A0D2121204DB1
:1001B000495353494E4720424C2D4354524C3A2008
:1001C0002564202121000A0D3D3D3D3D3D3D3D3D45
:1001D0003D3D3D3D3D3D3D3D3D3D3D3D3D3D3D3D4F
:1001E0003D3D3D3D3D3D3D3D3D3D3D000A0D4361B5
:1001F0006C6962726174696E672070726573737581
:1002000072652073656E736F722E2E004F4B0A0D50
:10021000000A0D466C696768742D74696D65202548
:1002200075206D696E2020546F74616C3A257520BD
:100230006D696E000A0D436F6E74726F6C3A200028
:1002400048656164696E67486F6C64004E6F726DDB
:10025000616C20284143432D4D6F646529000A0DD0
:100260003D3D3D3D3D3D3D3D3D3D3D3D3D3D3D3DBE
:100270003D3D3D3D3D3D3D3D3D3D3D3D3D3D3D3DAE
:100280003D3D3D0A0D00416E676C654E69636B2014
:10029000202020202020416E676C65526F6C6C20FE
:1002A0002020202020204163634E69636B202020A2
:1002B000202020202020416363526F6C6C2020207E
:1002C0002020202020205961774779726F2020203C
:1002D0002020202020204865696768742056616CC2
:1002E0007565202020204163635A20202020202093
:1002F0002020202020204761732020202020202043
:10030000202020202020436F6D7061737320566180
:100310006C7565202020566F6C74616765205B30BA
:100320002E31565D20205265636569766572204CDA
:100330006576656C20204779726F20436F6D706120
:100340007373202020204D6F746F72203120202085
:100350002020202020204D6F746F7220322020201A
:100360002020202020204D6F746F72203320202009
:100370002020202020204D6F746F722034202020F8
:100380002020202020203136202020202020202046
:100390002020202020203137202020202020202035
:1003A0002020202020203138202020202020202024
:1003B0002020202020203139202020202020202013
:1003C000202020202020536572766F2020202020BE
:1003D000202020202020486F7665726761732020DE
:1003E00020202020202043757272656E74205B30BF
:1003F0002E31415D20204361706163697479205B17
:100400006D41685D20204865696768742053657494
:10041000706F696E7420323520202020202020202B
:1004200020202020202032362020202020202020A4
:10043000202020202020436F6D706173732053654E
:1004400074706F696E744932432D4572726F7220F9
:10045000202020202020424C204C696D69742020EF
:100460002020202020204750535F4E69636B2020BE
:100470002020202020204750535F526F6C6C20209A
:1004800020202020202021212120494E434F4D5063
:10049000415449424C4520212121002A002E000AC6
:1004A0000D20444143206F7220493243204552526F
:1004B0004F522120436865636B204932432C20331F
:1004C000567265662C2044414320616E6420424C84
:1004D0002D4374726C005B25695D005B25695D00CE
:1004E0002B204D696B726F4B6F70746572202B00FF
:1004F00048573A5625642E25642053573A25642ED2
:10050000256425630053657474696E673A25642019
:100510002573004D69786572204572726F722100F3
:100520004552522532643A004861726477617265BF
:10053000204572726F7220313A2564202121004DCE
:10054000697373696E6720424C2D4374726C3A254F
:1005500064212100493243204552524F522121212A
:10056000004865696768743A20202535690053653D
:1005700074706F696E743A253569005072657373D3
:100580007572653A253569004F66667365743A2061
:10059000202535690048656967687420636F6E744B
:1005A000726F6C0044495341424C4544006163748E
:1005B0002E2062656172696E67004E69636B3A2036
:1005C000202020202025356900526F6C6C3A2020B5
:1005D0002020202025356900436F6D706173733AC8
:1005E000202020253569004B25693A2534692020D3
:1005F0004B25693A25346920004E693A2534692033
:1006000020526F3A253469200047733A2534692017
:100610002047693A253469200050313A2534692051
:100620002050323A253469200050333A253469206D
:100630002050343A25346920004779726F202D20EC
:1006400053656E736F72004E69636B2534692028A1
:100650002533692E25692900526F6C6C2534692079
:10066000282533692E256929004769657225346973
:10067000202825336929004E69636B2025346920C1
:10068000282533692E25782900526F6C6C2025347B
:100690006920282533692E25782900596177202083
:1006A000253469202825336929004E69636B20258C
:1006B0003469202825336929282533692900526F98
:1006C0006C6C202534692028253369292825336955
:1006D000290059617720202534692028253369298C
:1006E000282533692900414343202D2053656E732B
:1006F0006F72004E69636B202534692028253369A9
:100700002900526F6C6C2025346920282533692913
:10071000005A20202020253469202825336929000B
:10072000566F6C746167653A2020202533692E2549
:100730003169560043757272656E743A2020202527
:1007400033692E2531694100506F7765723A202058
:1007500020202025346957004469736368617267FB
:10076000653A202535696D41680052656365697693
:1007700065720052432D525353493A2020202025C0
:1007800034690052432D5175616C6974793A2025A2
:1007900034690052432D4368616E6E656C733A256F
:1007A000346900436F6D70617373004D61676E65EE
:1007B000743A202020253569004779726F3A20204D
:1007C00020202025356900536574706F696E743A76
:1007D0002025356900506F746925693A202025333A
:1007E0006900506F746925693A20202533690053E8
:1007F0006572766F202000536574706F696E742087
:100800002025336900506F736974696F6E3A202533
:1008100033690052616E67653A2533692D25336966
:1008200000424C2D4374726C204572726F727320BB
:100830000025336420253364202533642025336468
:100840002000424C2054656D70657261747572654C
:100850000025336420253364202533642025336448
:100860002000424C2D4374726C20666F756E6420BC
:1008700000202563202020256320202025632020C0
:1008800020256320002025632020202563202020B0
:100890002563202020256320002025632020202D93
:1008A0002020202D2020202D20003130003131004B
:1008B000313200466C696768742D54696D6520207B
:1008C00000546F74616C3A2535756D696E00416333
:1008D000743A20202535756D696E00287265736540
:1008E0007429000A0D47656E65726174696E672030
:1008F00064656661756C7420506172616D657465C4
:100900007220536574202564000A0D5573696E6763
:1009100020506172616D6574657220536574202585
:1009200064000A0D47656E65726174696E672064C4
:10093000656661756C74204D6978657220546162DA
:100940006C65000A0D4D697865722D436F6E66699E
:10095000673A202725732720282575204D6F746F4F
:10096000727329000A0D3D3D3D3D3D3D3D3D3D3D00
:100970003D3D3D3D3D3D3D3D3D3D3D3D3D3D3D3DA7
:100980003D3D3D3D000A0D414343206E6F742063A1
:10099000616C69627261746564210D0A0000008FE8
:1009A000001E01AD013B02CA025803E603740402B3
:1009B000058F051B06A7063307BE074808D2085B4C
:1009C00009E3096B0AF20A780BFD0B810C040D8612
:1009D0000D070E870E060F840F00107B10F5106EAA
:1009E00011E5115B12CF124213B31323149214FEBC
:1009F000146A15D3153B16A11605176717C81727D4
:100A0000188318DE1837198E19E319361A871AD683
:100A10001A231B6E1BB61BFD1B411C831CC31C0031
:100A20001D3C1D751DAB1DE01D121E421E6F1E9A42
:100A30001EC31EE91E0D1F2E1F4D1F691F841F9B05
:100A40001FB01FC31FD31FE11FEC1FF51FFB1FFFAC
:100A50001F002004010000E66C000201010F6E017E
:100A6000030202A36E020403034B6F03000404009D
:100A70006F2532692E2531695600253364256320A0
:100A8000253033646D2563005374617475730045BC
:100A900052524F523A2025326420002534692025D5
:100AA00032693A25303269002534696D25630025A5
:100AB00033692025336920253369202533690025D2
:100AC0003369202533692025336920253369005493
:100AD000656D7065726174757265732020202000E9
:100AE0002563432020202020002532692E253169EE
:100AF00056202533692E2531694100253469572058
:100B00002536696D4168004D61676E65743A25331D
:100B100069252520253369256300496E636C692E9C
:100B20003A25336925632028256929200025327557
:100B30006D2F73205361743A2564200020203344C4
:100B4000004E6F4678004447505300486F6D653A39
:100B50002533646D202533642563202563004E6FA3
:100B6000204E6176694374726C21004E6F2045728D
:100B7000726F722020202020202020004E6F7420D1
:100B8000636F6D70617469626C652020004D4B333A
:100B90004D6167206E6F7420636F6D7061004E6FE2
:100BA00020464320636F6D6D756E69636174004DFF
:100BB0004B334D616720636F6D6D756E69636100C6
:100BC00047505320636F6D6D756E69636174696F13
:100BD00000636F6D706173732076616C75652020A2
:100BE00020005243205369676E616C206C6F7374F0
:100BF000202000464320737069207278206572724D
:100C00006F7220004E6F204E4320636F6D6D756EC6
:100C100069636174004643204E69636B20477972B3
:100C20006F2020202000464320526F6C6C204779B3
:100C3000726F202020200046432059617720477999
:100C4000726F2020202020004643204E69636B20D5
:100C5000414343202020202000464320526F6C6CEB
:100C6000204143432020202020004643205A2D418C
:100C700043432020202020202020005072657373E1
:100C80007572652073656E736F7220004932432060
:100C900046432D3E424C2D4374726C2000426C2022
:100CA0004D697373696E67202020202020004D69F4
:100CB000786572204572726F7220202020200043D8
:100CC00061726566726565204572726F72202000E0
:100CD00047505320466978206C6F73742020202081
:100CE000004D61676E6574204572726F722020201E
:100CF00020004D6F746F722072657374617274207E
:100D0000202000424C204C696D69746174696F6EDB
:100D100020202000202020202020202020202020F3
:100D20002020202020202020200020202532692E75
:100D30002531695620200020202532692E25316971
:100D400056202000414C543A2534696D202563001B
:100D5000414C543A2534696D202000414C543A2DC1
:100D60002D2D2D200020202532693A253032692092
:100D7000200020202532693A2530326920200044A5
:100D800049523A2025336425630043002000202087
:100D90002535692020002020253569202000493A8A
:100DA0002532692E2531694120004900490049005A
:100DB0002D2D2D2D2D2D2D2D2D2B2D2D2D2D2D2D65
:100DC0002D2D2D2D2D002D2D2D2D2D2D2D2D2D2D80
:100DD0002D2D2D2D2D2D2D2D2D2D2D004900534147
:100DE000543A2532642000444953543A2533646D03
:100DF000004420003344002121004D41473A25336F
:100E00007525252000484D3A253364256320256348
:100E100000696E636C3A253264256328253269299E
:100E2000004900202020202532756D2F73002048B6
:100E30004D3A2533642563202563004552523A20FC
:100E40002532642021004552523A200020777777DE
:100E50002E4D696B726F4B6F707465722E646520D6
:100E60002000202532693A25303269202025326958
:100E70002E25316956202534696D416800202532C0
:100E8000693A2530326920202532692E253169568C
:100E9000202534696D4168004449523A2533642560
:100EA0006300414C543A2534696D00414C543A2555
:100EB00034696D00414C543A2D2D2D2D20002563B1
:100EC00000484D3A25336425632020444953543A61
:100ED0002533646D202563005057523A2532692E20
:100EE00025316941202825695729200043460020E3
:100EF00020004750533A2532756D2F7320534154CB
:100F00003A256420002020334420004E4F464958A3
:100F1000004447505320002020204E6F204E617621
:100F2000694374726C202020202020200025326923
:100F30002E2569202532692E2569202532692E2526
:100F400069202532692E2569410025336920253322
:100F500069202533692025336925634300253269DB
:100F60002E2569202532692E256941002532692EFA
:100F70002569202532692E2569202532692E2569AB
:100F8000202532692E2569410025336920253369E2
:100F900025634320202020202020200025336920A5
:100FA00025336920253369202533692563430045AE
:100FB00052523A202532642021004552523A2000F4
:100FC000207777772E4D696B726F4B6F70746572F7
:100FD0002E646520200053657474696E673A257528
:100FE00020257320004D696E3A2532692E2531691E
:100FF000562025732000414C543A00504F54493A32
:101000002533752000284F4E29202000284F4646C2
:101010002920004C494D495400564152494F004443
:10102000495341424C45440043463A0044495341E8
:10103000424C45440020284F4E29200020284F468E
:10104000462900205445414348004750533A004444
:10105000495341424C454400284652454529002801
:10106000484F4D4529002841494429200028484F30
:101070004C4429002046533A257573656B2000487F
:101080004F4D4520414C543A0025756D00484F4C5A
:101090004420004E693A25346920526F3A2534695C
:1010A00020433A2533690047733A25346920596152
:1010B0003A253469200050313A2534692050323ABB
:1010C00025346920333A2533690050343A25346990
:1010D0002050353A25346920363A25336900434F8C
:1010E00055504C494E47204F46462120004C4F4F0B
:1010F00050494E472120004848212000434F4D5081
:10110000415353204F46462120000A0D7777772E12
:101110004D696B726F4B6F707465722E6465202819
:10112000632920486953797374656D7320476D6234
:1011300048000A0D74686520757365206F66207419
:1011400068697320736F66747761726520697320B4
:101150006F6E6C79207065726D6974746564200AB5
:101160000D6F6E206F726967696E616C204D696BDF
:10117000726F4B6F707465722D4861726477617223
:10118000650047726175706E657220486F54540037
:101190004143542044534C004A6574692073617480
:1011A000656C6C6974005370656B7472756D207337
:1011B0006174656C6C697420284C6F77207265735C
:1011C0006F6C7574696F6E29005370656B747275FE
:1011D0006D20736174656C6C69742028323034380A
:1011E00029005370656B7472756D20736174656C42
:1011F0006C6974004D756C74697369676E616C20FD
:1012000050504D000A0D52656365697665723A204B
:1012100000756E6B6E6F776E2E205573696E67204A
:1012200050504D2E2E2E006E6F7420737570706F9F
:101230007274656420627920686172647761726596
:1012400021000A0D3D3D3D3D3D3D3D3D3D3D3D3D8A
:101250003D3D3D3D3D3D3D3D3D3D3D3D3D3D3D3DBE
:101260003D3D3D3D3D3D3D000A0D466C696768745E
:10127000436F6E74726F6C0A0D48617264776172AD
:10128000653A25642E25640A0D536F667477617282
:10129000653A5625642E2564256320000A0D3D3DE0
:1012A0003D3D3D3D3D3D3D3D3D3D3D3D3D3D3D3D6E
:1012B0003D3D3D3D3D3D3D3D3D3D3D3D3D3D3D3D5E
:1012C0003D0011241FBECFEFD0E4DEBFCDBF11E043
:1012D000A0E0B1E0E0E5F6E101E00BBF02C007905D
:1012E0000D92A83AB107D9F719E0A8EAB1E001C018
:1012F0001D92A43AB107E1F77AEAE2E0F0E081E278
:1013000080935700D4907E010894E11CF11C20EFDB
:1013100037EF41E050E087016FE0DA01C9012F5F4C
:101320003F4F4F4F5F4FABBFFC018791F801819357
:101330008F01615067FFF1CFF7016EE0819178274F
:101340007095615067FFFACF8889781729F0F7E91F
:10135000DF1611F40000FECF0E94710A0C94278B57
:101360000C9400008091CF05E82FFF27EE0FFF1FA0
:10137000E350F94F808191818D5E9F4F14F0109260
:101380000301808191818A5B9F4FCCF4809103019E
:101390008823A9F481E0809303018091C2038F5FC9
:1013A0008093C203853038F088EE93E09093DD019E
:1013B0008093DC0104C066E970E00E94C737809129
:1013C000C20399279093500580934F0508951F936A
:1013D000CF93DF93182F882389F086E691E09F93BF
:1013E0008F9382E995E19F938F93E0918E03F09123
:1013F0008F0309950F900F900F900F908091F20539
:10140000823308F044C084EF91E00E94A119EC01FE
:10141000112329F0CE010E94AA198823D9F3C2E032
:10142000D0E026E530E080911E0190911F018217E7
:10143000930730F02196255D3F4FC730D10598F3D3
:101440008091F2059927C89F9001C99F300DD89FC0
:10145000300D1124209300011123D9F068EC70E0C5
:101460008C2F0E94C737DF93CF938EE691E09F9336
:101470008F9382E995E19F938F93E0918E03F09192
:101480008F0309958DB79EB706968DBF02C08093D6
:101490000001112311F1809100016AE00E947A8A13
:1014A000892F99279F938F93809100010E947A8AB8
:1014B00099279F938F9389E791E09F938F9382E978
:1014C00095E19F938F93E0918E03F0918F0309959F
:1014D0002DB73EB7285F3F4F2DBFDF91CF911F91B2
:1014E0000895CFEFD0E4DEBFCDBF8824992414B88F
:1014F00015B8B7EEEB2EB3E0FB2E8EEC9FEFE80EA7
:10150000F91EF7FEFACF85E18093020181E887B9E1
:101510003E9A8FEF88B98BE184B911E015B98EE35B
:101520008AB987E48BB9469A84B7877F84BF809154
:1015300060008861809360001092600084EC99E004
:101540009093DD018093DC01109279021092780271
:10155000109202071092010710927B0210927A02F9
:1015600010927D0210927C0284EC94E0A0E0B0E046
:101570008093430190934401A0934501B0934601A9
:1015800028980E940A1A0E94DB190E949A150E944C
:10159000B0350E944E1D812F0E9413310E94E564D8
:1015A0000E943A700E948A86809102018C3010F469
:1015B000299A01C0299878940E94253080912402AC
:1015C000826080932402109227020E94FC4284EFE2
:1015D00091E00E94A1197C018091240280FD05C048
:1015E000C7010E94AA198823B9F383E991E09F9368
:1015F0008F93A2E9AA2EA5E1BA2EBF92AF92E091F5
:101600008E03F0918F03099580EA9FE00E94A11953
:101610007C0100E010E00F900F900F900F90CFE949
:10162000D6E0F3E5CF2EF6E0DF2E0E94FC4280915B
:10163000240280FD05C0C7010E94AA198823B9F3BE
:10164000F60180811816A4F40BC00E94FC42809120
:10165000240280FD05C0C7010E94AA198823B9F39E
:10166000C7010E94AA19882319F4888188236CF77E
:10167000888187FF1AC00F5F1F4F1F930F93015080
:10168000104085EA91E09F938F93BF92AF92E091D3
:101690008E03F0918F0309958091A9018F5F80934C
:1016A000A9018DB79EB706968DBF0F5F1F4FE4E06F
:1016B000F0E0CE0EDF1E28960C30110508F4B5CFF1
:1016C00000E010E0CCE9D6E0E3E5EE2EE6E0FE2E09
:1016D0008B8187FD1EC0F70180811816D4F40F5F3F
:1016E0001F4F1F930F930150104088EA91E09F9382
:1016F0008F9382E995E19F938F93E0918E03F09110
:101700008F03099582E08093DA018DB79EB7069624
:101710008DBF8B8180788B830F5F1F4FE4E0F0E0FB
:10172000EE0EFF1E28960C30110590F286EC91E02B
:101730009F938F93C2E9D5E1DF93CF93E0918E031E
:10174000F0918F0309959091CD058091A9010F909B
:101750000F900F900F90981728F48091A803806144
:101760008093A8038CEE91E09F938F93DF93CF93A8
:10177000E0918E03F0918F03099588EE93E00E942B
:10178000A1197C010E94541D0F900F900F900F9093
:10179000C7010E94AA198823D9F38CE092E09F9395
:1017A0008F93DF93CF93E0918E03F0918F03099590
:1017B00080E00E949638809102010F900F900F9068
:1017C0000F908A3011F0843110F0289801C0289AC7
:1017D00080ED97E09093DD018093DC0185E58093B7
:1017E000C4038EE090E00E94542E9927182F002702
:1017F0008FE090E00E94542E080F111D1093AF014E
:101800000093AE018AE090E00E94542E9927182F91
:1018100000278BE090E00E94542E080F111D1093BA
:10182000AD010093AC010F5F1F4F39F08091AE0105
:101830009091AF018F5F9F4F41F41092AF011092D2
:10184000AE011092AD011092AC018091AC0190916B
:10185000AD019F938F938091AE019091AF019F93C3
:101860008F9381E192E09F938F93DF93CF93E091E9
:101870008E03F0918F0309958DB79EB708968DBFA3
:1018800084E392E09F938F93DF93CF93E0918E0355
:10189000F0918F0309958091DB050F900F900F90C9
:1018A0000F90E0918E03F0918F0382FF07C080E4D8
:1018B00092E09F938F93DF93CF9308C08CE492E0E4
:1018C0009F938F9382E995E19F938F9309950F9052
:1018D0000F900F900F900E94EB2288E893E1909375
:1018E0003E0180933D0111E01093C303812F0E94BC
:1018F000E7098091F5050E94CF858EE592E09F93E0
:101900008F93DF93CF93E0918E03F0918F0309952E
:1019100080ED97E00E94A1197C018AEF90E00E947F
:10192000A11983E0809327051092A80180913806C1
:101930000F900F900F900F9084FF02C01093B00192
:101940008091B201882311F04798FECF8091E00189
:10195000882309F4F3C180911001882309F4EEC1B2
:101960001092E0018091C203882319F00E94B2090D
:1019700002C00E9401460E94FC42209102012A30CE
:1019800011F0243110F0289801C0289A80916C023F
:10199000882331F080916C02815080936C020EC0DC
:1019A00080916F00806280936F001092FE0610920B
:1019B000FD068091A80388608093A80380913D0173
:1019C00090913E01019790933E0180933D0180915B
:1019D0003D0190913E01892B21F0809125028823C1
:1019E000C9F180913D0190913E01892BD9F40E946B
:1019F0003D3185E090E090933E0180933D018091E0
:101A0000610590916205019690936205809361054E
:101A10008091A80381608093A8038091280582604B
:101A20008093280580910801909109018F5F9F4F55
:101A3000C1F480916B028823A1F088EA91E690932B
:101A4000DD018093DC0180E890E0909309018093B0
:101A5000080107C02A3011F0243110F0289801C085
:101A6000289A0E945C878091E001882309F066C172
:101A700080910E01882311F00E94211A0E94DE1528
:101A80000E942C11C7010E94AA19882309F452C18F
:101A900084E190E0E80EF91E8091F505863011F49E
:101AA0000E94097480912502882349F08091A8033F
:101AB00082608093A8038091280582600FC0809186
:101AC000DC019091DD01892B59F480913D019091C9
:101AD0003E01079728F0809128058D7F8093280587
:101AE00080916C02882361F08091B001882341F0DD
:101AF0001092B00188E893E19093DD018093DC01BE
:101B000080910501882321F08150809305012EC02A
:101B10008093CE0310924202109241021092400232
:101B200010923F0210923E0210923D0280916C0290
:101B30008823E1F480910801909109018F5F9F4F04
:101B4000A9F42091B001223089F088E99AE39093BA
:101B5000DD018093DC0180E09CE09093090180939B
:101B60000801222319F082E08093B00180919C014A
:101B7000893C48F0815080939C018091A8038B7F21
:101B80008093A8033FC08091DE078823F9F08091FD
:101B9000A80384608093A80389E080934603809122
:101BA0000801909109018F5F9F4F81F480916B0232
:101BB000882361F088E99AE39093DD018093DC014A
:101BC00080E098EA909309018093080110923A030B
:101BD0001092390310923803109237031092360393
:101BE0001092D1071092100810920F08109212084C
:101BF000109211088FEF9FEF90930E0880930D08BD
:101C000010929C0180910001282F332780911E01A2
:101C100090911F0182179307CCF480913602806265
:101C20008093360280910801909109018F5F9F4F48
:101C3000C1F480E797E19093DD018093DC0180E0BF
:101C400093E090930901809308010BC08091DC011F
:101C50009091DD01892B29F4809136028F7D80934C
:101C600036020E949B6984E08093DB0180913602FA
:101C700081FD05C05AEA852E55E0952E12C080914F
:101C8000B1018F5F8093B101813359F41092B1019A
:101C90008091AA019091AB0101969093AB01809342
:101CA000AA010894811C911C82E788168BE0980693
:101CB00009F040C0882499242091AE013091AF01F1
:101CC0002F5F3F4F3093AF012093AE018091AC0165
:101CD0009091AD0101969093AD018093AC01832F5B
:101CE0009927682F8EE090E00E945C2E8091AE01D3
:101CF0009091AF019070682F8FE090E00E945C2E71
:101D00008091AC019091AD01892F9927682F8AE0CD
:101D100090E00E945C2E8091AC019091AD0190709A
:101D2000682F8BE090E00E945C2E84E190E00E949E
:101D3000A1197C010E94EB690E9451708091DB0126
:101D4000882309F0FDCD0E940665FACD1F920F92FF
:101D50000FB60F9211248F939F93EF93FF9380916F
:101D600007018823E1F48091CC019091CD01019687
:101D70009093CD018093CC01FC01E358FB4FE081AF
:101D8000ED3019F08A3A910539F41092CD01109294
:101D9000CC0181E080930701E093C60004C010925B
:101DA000CD011092CC01FF91EF919F918F910F90F7
:101DB0000FBE0F901F9018951F920F920FB60F92A3
:101DC00011242F933F934F935F936F937F938F9340
:101DD0009F93AF93BF93CF93EF93FF9390E0809146
:101DE000B201813029F48091C6008093CE00CCC02E
:101DF0008091B201823029F48091C6008093D10392
:101E0000C3C08091C6008093C4015091D2015A3A58
:101E100010F09093D3018091C4018D3009F065C01A
:101E20008091D301823009F060C09093D301852F57
:101E300099278F529C4FFC01329740812091CE010F
:101E40003091CF01241B3109DC0111978C91281BA3
:101E50003109C9019F709093CF018093CE0146E074
:101E6000969587954A95E1F7982F935C9093D001CA
:101E70002F733070235C2093D1018081981729F44F
:101E80008C91281711F491E006C090E08091C10177
:101E90008F5F8093C101C091C301CC2309F074C04E
:101EA000992309F471C081E08093C301580F5093C6
:101EB000C0015150E52FFF27EF52FC4F8DE080838A
:101EC0008091D303823509F05FC00E94EB2288E144
:101ED00090E02CE00FB6F894A895809360000FBEB8
:101EE00020936000C093DA014FC02091D301822F6C
:101EF000992781309105F9F0823091051CF4892BE6
:101F000021F040C0029711F13DC08091C40183329D
:101F100039F48091C301882319F481E08093D301BF
:101F20008091C4018093D10381E08093D20180919C
:101F3000C401992722C02F5F2093D301E52FFF27EB
:101F4000EF52FC4F8091C401808309C0E52FFF2729
:101F5000EF52FC4F8091C40180835A3A20F45F5FB6
:101F60005093D20102C01092D3012091C4018091FC
:101F7000CE019091CF01820F911D9093CF0180935C
:101F8000CE0102C01092D301FF91EF91CF91BF918A
:101F9000AF919F918F917F916F915F914F913F9101
:101FA0002F910F900FBE0F901F901895AC01A0E0DD
:101FB000B0E09D01A817B90748F4EDE7F4E081917E
:101FC000280F311D1196A417B507C8F33F70FD0106
:101FD000E358FB4FC90156E0969587955A95E1F76E
:101FE000835C80831196FD01E358FB4F2F733070A3
:101FF000822F835C8083A258BB4F8DE08C9310921C
:10200000070180917D048093C6000895A0E0B0E0B0
:10201000ECE0F0E10C94F38A2C859D850E85BB24C1
:1020200083E280937D049F5990937E0420937F04E4
:1020300033E0E32EF12C002309F49EC0CF84D8882E
:10204000BE016D5E7F4FA989BA890150109709F4CE
:1020500093C01097B9F0F601EB0DF11DB394908188
:10206000119791F4002349F1FB016E5F7F4FDB0173
:10207000C080D1806E5F7F4F0D90BC91A02DBB249E
:10208000015002C090E019C01097B9F0F601EB0DB5
:10209000F11DB3944081119791F4002341F1FB01AC
:1020A0006E5F7F4FDB01C080D1806E5F7F4F0D90F0
:1020B000BC91A02DBB24015002C040E018C0109775
:1020C000B1F0F601EB0DF11DB3941081119781F47D
:1020D000002371F0FB013296DB01CD90DC90BF0153
:1020E0006E5F7F4FA081B181BB24015001C010E021
:1020F000F701E358FB4F892F86958695835C808393
:102100000894E11CF11CF701E358FB4F892F992734
:102110008370907024E0880F991F2A95E1F7552766
:102120009A0194E0369527959A95E1F7822B835C86
:1021300080830894E11CF11CF701E358FB4F4F70BA
:102140005070440F551F440F551F812F992726E0CB
:10215000969587952A95E1F7842B835C8083089474
:10216000E11CF11CF701E358FB4F1F73135C108354
:102170000894E11CF11C6ACFC7010E94D60FE9E068
:102180000C940F8BA3E07A2F4091C001465044235A
:1021900009F458C0E72FFF27EF52FC4F80818D5381
:1021A0007F5FE72FFF27EF52FC4F20812D537F5F8A
:1021B000E72FFF27EF52FC4F30813D537F5FE72F22
:1021C000FF27EF52FC4F60816D537F5F9927880F87
:1021D000991F880F991F522F52955F70582B822F8D
:1021E00099278F709070F4E0880F991FFA95E1F7A6
:1021F000232F26952695282B832F9927837090705F
:10220000E6E0880F991FEA95E1F7682B41504F3FB0
:10221000C9F0EA2FFF27EF52FC4F5083AF5F4150C8
:102220004F3F81F0EA2FFF27EF52FC4F2083AF5F33
:1022300041504F3F39F0EA2FFF27EF52FC4F6083A8
:10224000AF5FA5CF84ED93E09093BF018093BE0173
:10225000A350A093BD010895A2E0B0E0E2E3F1E154
:102260000C94F98A8091C301882309F457C40E9411
:10227000C2108091D203823609F023C38091D30328
:1022800099278037910509F4AFC081379105C4F4CF
:102290008A36910509F480C28B36910544F48B345B
:1022A000910571F18636910509F45FC10AC38D3637
:1022B000910509F469C08E36910509F44DC001C33A
:1022C0008437910541F1853791054CF481379105AB
:1022D00009F491C08337910509F4DFC0F2C2873752
:1022E000910509F41BC2883791052CF485379105B7
:1022F00009F4D7C1E6C28937910509F46DC1E1C27D
:10230000E091BE01F091BF01808191819093900195
:1023100080938F01D6C28091C001A091BE01B0917F
:10232000BF01853140F080E1ECEAF3E00D900192CD
:102330008A95E1F70DC08D919D910D90BC91A02DD6
:102340008093AC039093AD03A093AE03B093AF031F
:1023500080EF8093BB014BC0809107018823E1F39C
:102360008DE490E09F938F9386E496E09F938F9304
:1023700081E08F938F938EE48F930E9406108DB728
:102380009EB707968DBF9DC2A091BE01B091BF01BF
:102390001C91113081F48DE4E6E4F6E00D90019299
:1023A0008A95E1F70E94622F19838091A8038F7E9E
:1023B0008093A80301C01982809107018823E1F36B
:1023C00081E090E09F938F93CE0101969F938F932E
:1023D00081E08F938F938DE48F930E940610ADB7A9
:1023E000BEB71796ADBF6DC281E08093C6018FEF77
:1023F0008093050166C2E091BE01F091BF01E081CA
:102400008E2F8A508A3058F48983882311F481E012
:1024100003C0863010F085E0898361E00EC08E2F06
:1024200084518A3070F48983882311F481E003C0D9
:10243000863010F085E0898360E089810E94E22F78
:1024400012C0E983EF3F19F40E94C52F8983898167
:10245000882311F481E003C0863010F085E0898381
:1024600089810E94722E809107018823E1F387E71A
:1024700090E09F938F938EEC95E09F938F9381E0F4
:1024800090E09F938F93CE0101969F938F9382E06C
:102490008F9381E08F9381E577C12091BE013091C8
:1024A000BF01D9018C918150853008F045C0F901F8
:1024B0008181883509F040C080916B028823E1F565
:1024C0002F5F3F4F87E7EEECF5E0D9010D900192C9
:1024D0008A95E1F7F90182910E94DD2E80910F0625
:1024E0009927AA27BB27BC01CD0124EC39E040E0A5
:1024F00050E00E945B8ADC01CB01809387019093BE
:102500008801A0938901B0938A01809110069927D0
:10251000AA27BB27BC01CD010E945B8ADC01CB014D
:102520008093830190938401A0938501B0938601E9
:102530000E94C52F898301C01982809107018823D9
:10254000E1F381E090E09F938F93CE0101969F93FA
:102550008F9381E08F938F9383E58F930E94061072
:102560008DB79EB707968DBF26C0E091BE01F09152
:10257000BF01E0818E2F8150853018F48E2F0E948C
:10258000722E0E94C52F8983809107018823E1F371
:1025900081E090E09F938F93CE0101969F938F935C
:1025A00081E08F938F9386E48F930E940610ADB7DE
:1025B000BEB71796ADBF80916B02882329F46EE6F3
:1025C00070E089810E94C73780E00E94E70980910E
:1025D000F5050E94CF8575C1E091BE01F091BF0164
:1025E0008081992787FD909590931807809317070E
:1025F0008181992787FD909590931A0780931907F9
:102600008281992787FD909590931C0780931B07E3
:102610008381992787FD909590931E0780931D07CE
:102620008481992787FD90959093200780931F07B9
:102630008581992787FD90959093220780932107A4
:102640008681992787FD909590932407809323078F
:102650008781992787FD909590932607809325077A
:102660008085992787FD9095909328078093270769
:102670008185992787FD909590932A078093290754
:102680008285992787FD909590932C0780932B073F
:102690008385992787FD909590932E0780932D072A
:1026A00010C1E091BE01F091BF0180810E94093507
:1026B0008A83882319F481E0898301C0198280917B
:1026C00007018823E1F388E090E09F938F9384E9EA
:1026D00096E09F938F9321E030E03F932F9380917A
:1026E000BE019091BF019F938F933F932F93CE0193
:1026F00002969F938F933F932F93CE01820F931F48
:102700009F938F9384E08F9381E08F9385E58F93E0
:102710000E940610EDB7FEB773963CC08091BD01D4
:10272000893008F4CEC02091BE013091BF012F5FE7
:102730003F4F88E0A4E9B6E0F90101900D928A9537
:10274000E1F7D9018E910E945F348A83882319F4BE
:1027500081E0898301C01982809107018823E1F318
:1027600021E030E03F932F93CE0102969F938F9309
:102770003F932F93CE01820F931F9F938F9382E0FD
:102780008F9381E08F9387E58F930E940610EDB7BA
:10279000FEB73B96EDBF95C080916B02882309F090
:1027A00090C00E9482858983823019F0843009F0BC
:1027B00088C020E430E0F8948091C1008F7380934A
:1027C000C1008091C9008F738093C9008091C100BE
:1027D000877E8093C1008091C900877E8093C90065
:1027E0008091C80087FF03C08091CE00F9CF80910F
:1027F000C00087FF03C08091C600F9CFE091BE0101
:10280000F091BF01E081E13021F482E08093B201D8
:102810002EC0E43611F421E830E081E08093B2016B
:10282000832F99278093CD002093CC008091CD00F9
:102830008093C5008091CC008093C4008091CA0031
:102840008F7D8093CA008091CA008F7E8093CA00DA
:102850008091C9008B7F8093C9008091CA008460F9
:102860008093CA008091CA0082608093CA008091E0
:10287000CA00877F8093CA008091C200877F8093BF
:10288000C2008091C9008E7F8093C9008091C100F1
:1028900088618093C1008091C90088618093C900DC
:1028A0008091C10080688093C1008091C9008068D8
:1028B0008093C90010926E0010926F001092700009
:1028C00078948091D30399278436910509F4BBC08D
:1028D00085369105ACF48136910509F46FC08236D6
:1028E00091052CF48B34910509F45DC00FC182363B
:1028F000910509F470C08336910509F47FC006C1C3
:102900008C36910509F4EDC08D3691054CF487366F
:10291000910509F4F8C08836910509F4B2C0F6C0F3
:102920008437910529F08637910509F4E8C0EEC097
:102930008091C001A091BE01B091BF01803140F0F3
:1029400080E1ECEAF3E00D9001928A95E1F70DC089
:102950008D919D910D90BC91A02D8093AC0390938F
:10296000AD03A093AE03B093AF038091070188231A
:10297000E1F31F92809104018F9384E58F930E946D
:1029800006108AEF8093BB018FEF8093050180EAE8
:102990009FE00E94A1199093B4018093B3010F901E
:1029A0000F900F90B3C0E091BE01F091BF01808104
:1029B00091819093900180938F01A8C0E091BE0116
:1029C000F091BF01808180930601803298F08FE101
:1029D000809306010FC0A091BE01B091BF018BE0B2
:1029E000E4ECF3E00D9001928A95E1F78091CD033C
:1029F000809369058FEF8093050188C08091B701AE
:102A00009091B801892B89F4E091BE01F091BF014A
:102A1000E081EE2351F08AE0E89FC00111240E947A
:102A2000A11990939F0380939E03E091BE01F091C2
:102A3000BF0190818AE0989FC00111249093B80152
:102A40008093B70115C08FEF80930501E091BE011F
:102A5000F091BF0190818AE0989FC001112490936A
:102A6000BA018093B901892B19F081E08093C801E4
:102A700080EA9FE00E94A1199093B4018093B30172
:102A800045C08FEF80930501E091BE01F091BF0139
:102A9000908197FD08C082E08093C5011092B60135
:102AA0001092B5011AC0909580911D02892B8093D8
:102AB0001D0291818AE0989FC00111249093B60174
:102AC0008093B50184E08093C50180EA9FE00E9475
:102AD000A1199093B4018093B30181E08093C9015F
:102AE00015C08FEF80930501E091BE01F091BF0109
:102AF000808180931E0281E08093CA0107C081E03B
:102B00008093C70103C081E08093CB011092C30181
:102B10001092BF011092BE011092BD01E3E0CE5FA2
:102B20000C94158B982F8091C00085FFFCCF90935B
:102B3000C60008950F931F9388E18093C100809190
:102B4000C00082608093C0008091C1008068809343
:102B5000C1008091C10080648093C10000E010E05A
:102B60000093C5008AE290E08093C4008091B9018F
:102B70009091BA010E94A1199093A1038093A003A0
:102B80008CED90E00E94A1199093D0038093CF0325
:102B90001092A20386E58093A30383E08093A603AB
:102BA0008BE08093A4031092A5031093BF010093C0
:102BB000BE011092BD011F910F910895A0E1B0E0F8
:102BC000E4EEF5E10C94F68A80910701882309F47C
:102BD000C1C28091B3019091B4010E94AA198823C7
:102BE00061F01092B6011092B5011092BA011092E4
:102BF000B9011092B8011092B7018091B50190917E
:102C0000B601892B41F080917B0490917C040E9455
:102C1000AA19882329F48091C901882309F460C086
:102C200080910701882309F45BC08091C5010DE7FD
:102C300015E08430A8F00E94012380E590E09F9386
:102C40008F931F930F9381E08F938F9388E48F93DB
:102C50000E9406102DB73EB7295F3F4F2DBF34C0ED
:102C600010921F0286E894E09F938F9384EF92E284
:102C70009F938F93E0918E03F0918F03099584E1E8
:102C800090E09F938F931F930F9381E090E09F9329
:102C90008F9385EC91E09F938F9382E08F9381E0F7
:102CA0008F9388E48F930E9406108091C501982F1E
:102CB0008F5F8093C5012DB73EB7215F3F4F2DBF7A
:102CC000943010F01092C5018091B5019091B60139
:102CD0000E94A11990937C0480937B041092C901F7
:102CE0008091CA01882351F180910701882331F135
:102CF0000E94012380E590E09F938F938DE795E0FC
:102D00009F938F9321E030E03F932F9380E291E0F7
:102D10009F938F933F932F938EE192E09F938F9396
:102D200083E08F9381E08F938CE48F930E94061051
:102D30001092CA018DB79EB70F968DBF8091C701C3
:102D40008823D1F0809107018823B1F08AE090E0D8
:102D50009F938F9382EA93E09F938F9381E08F9369
:102D60008F9386E58F930E9406101092C7012DB7AE
:102D70003EB7295F3F4F2DBF8091CB018823D9F00B
:102D8000809107018823B9F08BE090E09F938F93A7
:102D900084EC93E09F938F9381E08F938091040163
:102DA0008F9387E48F930E9406101092CB018DB70A
:102DB0009EB707968DBF8091CF039091D0030E945C
:102DC000AA19882309F461C080910701882309F4B6
:102DD0005CC08091EA059927880F991F880F991F79
:102DE0007C010027F7FC0095102F8091C60290917E
:102DF000C702A091C802B091C902BC01CD01A801CF
:102E000097010E94CF8A3093BD032093BC03809129
:102E1000BE029091BF02A091C002B091C102BC015C
:102E2000CD01A80197010E94CF8A3093BF03209360
:102E3000BE0380914B028093C00380914A0280932D
:102E4000C10388E090E09F938F938CEB93E09F9376
:102E50008F9381E08F9383E08F938BE68F930E9413
:102E600006108091C2032DB73EB7295F3F4F2DBF9B
:102E7000853018F086E08093C20383E690E00E94DC
:102E8000A1199093D0038093CF038091B9019091C1
:102E9000BA01892B41F08091A0039091A1030E9477
:102EA000AA19882321F48091C801882339F18091DF
:102EB0000701882319F10E94B13682E490E09F93C4
:102EC0008F9387E295E09F938F9381E08F938F9309
:102ED00084E48F930E9406101092C8018DB79EB7AC
:102EE00007968DBF8091B9019091BA01009731F09A
:102EF0000E94A1199093A1038093A0038091B70130
:102F00009091B801892B09F4B8C080919E039091EB
:102F10009F030E94AA19882309F4AFC0809107017A
:102F2000882309F4AAC08091EA059927880F991F80
:102F3000880F991F7C010027F7FC0095102F8091C6
:102F4000C6029091C702A091C802B091C902BC010B
:102F5000CD01A80197010E94CF8A3093910320935D
:102F600090038091BE029091BF02A091C002B091E7
:102F7000C102BC01CD01A80197010E94CF8A309304
:102F80009303209392032091C6073091C707409185
:102F9000C8075091C907DA01C90163E0880F991F7A
:102FA000AA1FBB1F6A95D1F7820F931FA41FB51FDD
:102FB000820F931FA41FB51F20914301309144013C
:102FC0004091450150914601BC01CD010E94CF8A3C
:102FD000309395032093940380918E0290918F02F9
:102FE000A0919002B091910249E0B595A79597956F
:102FF00087954A95D1F78093960380918A029091A4
:103000008B02A0918C02B0918D0239E0B595A79505
:10301000979587953A95D1F780939703809196027B
:1030200090919702A0919802B091990229E0B595EC
:10303000A795979587952A95D1F7809398038EE069
:1030400090E09F938F9380E993E09F938F9381E02B
:103050008F938F9383E48F930E9406108091B70122
:103060009091B8010E94A11990939F0380939E03B1
:103070002DB73EB7295F3F4F2DBF809106018F3F8F
:1030800071F1992704E0880F991F0A95E1F78A5793
:103090009D4F40E150E0BC01CE0101960E94AE88F8
:1030A00080E190E09F938F93CE0101969F938F9341
:1030B00081E090E09F938F9386E091E09F938F93C0
:1030C00082E08F9381E08F9381E48F930E940610BA
:1030D0008FEF809306018DB79EB70B968DBF8091C1
:1030E00069058823D1F0809107018823B1F081E040
:1030F00090E09F938F9389E695E09F938F9381E073
:103100008F938F9382E48F930E940610109269052B
:103110002DB73EB7295F3F4F2DBF8091C601882351
:10312000C9F0809107018823A9F084E390E09F9380
:103130008F938DEF96E09F938F9381E08F938F9382
:1031400080E58F930E9406101092C6018DB79EB73E
:1031500007968DBFE6E0C05F0C94128B1F920F9212
:103160000FB60F9211242F933F935F936F937F932A
:103170008F939F93AF93BF93EF93FF9320E0809142
:10318000DB01882329F08091DB0181508093DB01F2
:1031900080915703882319F08150809357038091C1
:1031A000E30181508093E3018F3F09F05BC089E028
:1031B0008093E3018091E1019091E2010196909367
:1031C000E2018093E10180910F018F5F8170809314
:1031D0000F01882319F481E08093E001349903C042
:1031E00081E08093E4018091DC019091DD01892BE5
:1031F00021F18091DC019091DD010B9750F08091DD
:10320000DC019091DD010A979093DD018093DC0150
:1032100004C01092DD011092DC018091DC019091DC
:10322000DD01209108013091090182239323892B2C
:1032300011F021E008C020E006C08FEF9FEF9093CF
:1032400009018093080180910201222331F08A3024
:1032500011F45A9A07C0479A05C08A3011F45A9857
:1032600001C047988091E401882309F45AC0209155
:103270009C01222309F055C08091B60783FF51C0FD
:1032800086B19927FC01E071F07084FF13C0809132
:10329000DE019091DF0101969093DF018093DE01C2
:1032A0008091DE019091DF01895E9340D0F12093FF
:1032B000E40137C08091DE019091DF01892B69F133
:1032C0008091DE019091DF018A56914030F5809126
:1032D000DE019091DF0169E270E00E94868A8091B0
:1032E000DE019091DF01860F971F9093DF0180939D
:1032F000DE018091DE019091DF010B9750F080910B
:10330000DE019091DF010A979093900180938F01E5
:1033100004C0F0939001E0938F011092DF011092AE
:10332000DE01FF91EF91BF91AF919F918F917F91BE
:103330006F915F913F912F910F900FBE0F901F9053
:1033400018952091E1013091E201280F391FC90140
:10335000019608952091E1013091E201821B930BC7
:10336000892F99278695807490700895CF93DF9365
:103370000E94A119EC01CE010E94AA198823D9F359
:10338000DF91CF910895CF93DF930E94A119EC01B3
:1033900009C080911001882329F0909310018FECCF
:1033A00080937A00CE010E94AA19982F882389F36E
:1033B000DF91CF9108959FB7F8945F983E9A469A0F
:1033C0008091B0008F708093B0008091B0008360D6
:1033D0008093B0008091B1008B738093B100809195
:1033E000B1008B608093B1001092B2008FEF809398
:1033F000B3008091B00080688093B000809170002D
:103400008A7F80937000809170008260809370004A
:103410009FBF08958AE090E00E94A1199093EA016D
:103420008093E90182E085BD83EA84BD17BC84EB0B
:1034300088BD86E086BD80916E00816080936E00BD
:103440000895A0E0B0E0E7E2FAE10C94F58A8091FB
:103450000506E82FFF27E75BFE4F9681D08080911D
:103460000E01A92FBB27A7FDB095CB2FDB2F8130F5
:1034700009F0DDC02091C6023091C7024091C80218
:103480005091C902BD01CE010E945B8A97FF04C022
:1034900061587F4F8F4F9F4F7B018C01F7E015954F
:1034A0000795F794E794FA95D1F78D2D992787FD25
:1034B0009095A92FB92F2091BE023091BF02409163
:1034C000C0025091C102BC01CD010E945B8A97FFEE
:1034D00004C061587F4F8F4F9F4FE7E095958795C8
:1034E00077956795EA95D1F7F801E701C61BD70BE9
:1034F000E80BF90B2091410330914203C90153E0DD
:10350000880F991F5A95E1F7821B930BAA2797FD05
:10351000A095BA2FC81BD90BEA0BFB0B8091FC05B9
:103520009927AA27BB27BC01CD019E01AF010E94AC
:103530005B8A97FF04C061507E4F8F4F9F4FFC0105
:10354000EB0149E0F595E795D795C7954A95D1F7F1
:1035500080916E01992736E0880F991F3A95E1F71F
:1035600040910C0150910D01209104063327841BDA
:10357000950BB9010E949A8A80910C0190910D01DE
:10358000860F971F90930D0180930C0180910C0181
:1035900090910D0197FD0F9624E0959587952A95BA
:1035A000E1F79093D7018093D6018091370680FF91
:1035B00007C08091D6019091D7018C0F9D1F06C046
:1035C0008091D6019091D7018C1B9D0B9093D701D0
:1035D0008093D6018091FD05282F3327220F331FBA
:1035E000220F331F8091D6019091D7018217930744
:1035F0007CF08091FE05282F3327220F331F220FE6
:10360000331F8091D6019091D7012817390724F4F0
:103610003093D7012093D60180910201843108F4C0
:10362000C2C080910E018F5F80930E01BEC02091B9
:10363000BE023091BF024091C0025091C102BD0153
:10364000CE010E945B8A97FF04C061587F4F8F4F65
:103650009F4F7B018C01C7E015950795F794E79480
:10366000CA95D1F78D2D992787FD9095A92FB92F50
:103670002091C6023091C7024091C8025091C90200
:10368000BC01CD010E945B8A9B01AC0197FF04C085
:1036900021583F4F4F4F5F4FB7E0559547953795AE
:1036A0002795BA95D1F72E0D3F1D401F511F8091D0
:1036B00000069927AA27BB27BC01CD010E945B8A7F
:1036C00097FF04C061507E4F8F4F9F4FFC01EB016D
:1036D000A9E0F595E795D795C795AA95D1F780917B
:1036E0006D01992776E0880F991F7A95E1F740914F
:1036F0000A0150910B01209104063327841B950B7E
:10370000B9010E949A8A80910A0190910B01860F5B
:10371000971F90930B0180930A0180910A01909169
:103720000B0197FD0F9664E0959587956A95E1F7F3
:103730009093D5018093D4018091370681FF07C013
:103740008091D4019091D5018C0F9D1F06C080916E
:10375000D4019091D5018C1B9D0B9093D501809342
:10376000D40180910106282F3327220F331F220F07
:10377000331F8091D4019091D501821793077CF07B
:1037800080910206282F3327220F331F220F331F69
:103790008091D4019091D5012817390724F43093F2
:1037A000D5012093D40110920E01E7E0CDB7DEB72A
:1037B0000C94118B1F920F920FB60F9211242F931E
:1037C0003F934F935F938F939F93EF93FF938091DA
:1037D00002019091E501843108F04CC0992309F071
:1037E0001CC18091B00086FF24C08091B0008F7B07
:1037F0008093B0008091D6019091D70187559E4F5C
:103800009093D9018093D80125E08D3D920718F05F
:103810008CED95E005C08757914030F487E791E043
:103820009093D9018093D8018091D8019091D901CA
:10383000BAC08091B00080648093B000809103068C
:10384000282F33278DED96E0289FA001299F500D4A
:10385000389F500D1124CA012091E6013091E701F3
:10386000821B930B9093D9018093D80181E08093C0
:103870000E01D0C0992309F0D0C08091B00086FF1E
:1038800097C08091B0008F7B8093B000E091E801F9
:10389000EE23F1F480910306282F33278DED96E077
:1038A000289FA001299F500D389F500D1124CA0157
:1038B0002091E6013091E701821B930B9093D9018F
:1038C0008093D8011092E7011092E601469AA2C0B7
:1038D00089EA93E09093D9018093D8018E2F99279C
:1038E00083309105D9F08430910534F4813091050D
:1038F00049F0029761F020C08430910591F005975E
:1039000099F01AC08091D6019091D70104C080919E
:10391000D4019091D50187559E4F1DC0809192078B
:1039200005C080916B0702C080919B079927880F83
:10393000991F880F991FEFCFFF27EE0FFF1FE3504E
:10394000F94F20813181220F331F8091D80190914E
:10395000D901820F931F9093D9018093D801809150
:10396000D8019091D90155E08D3D950718F08CED67
:1039700095E005C08757914030F487E791E0909338
:10398000D9018093D8012091D8013091D9012C5BC5
:1039900030403093D9012093D8018091E601909175
:1039A000E701820F931F9093E7018093E60132C0F5
:1039B0008091B00080648093B0008CEB90E0909395
:1039C000D9018093D8018091E6019091E701845458
:1039D0009F4F9093E7018093E6018091DA0188235D
:1039E00021F080916C02882321F48091DA018230E9
:1039F00011F4469801C0469A8091E8018F5F809348
:103A0000E80190910306981728F481E080930E0155
:103A10001092E80181E08093E5012091D801309176
:103A2000D90141E02F37340730F08FEF8093B30096
:103A30002F5F30400FC02F3F3105C9F0C0F0A90102
:103A40004F5F50404F37510550F480E88093B300EA
:103A5000205830403093D9012093D80112C08FEF05
:103A60008093B3005093D9014093D8010AC080914C
:103A7000D8018093B3001092D9011092D80110920E
:103A8000E501FF91EF919F918F915F914F913F9150
:103A90002F910F900FBE0F901F90189510927C00E1
:103AA0008FEC80937A000895CF93DF931092EF010B
:103AB00086E987BD83E090E00E94542EC82F863EA1
:103AC00008F4C65FC8BD84E690E00E94C3198091E7
:103AD0001401909115018152934010F0C0EF02C083
:103AE000C530F8F0C8BD82E390E00E94C3198BE9AD
:103AF00094E09F938F9382E995E19F938F93E09158
:103B00008E03F0918F030995809114019091150116
:103B10000F900F900F900F908152934010F4C5506A
:103B2000DFCF6C2F83E090E00E945C2ECF3018F046
:103B3000CCE8D0E002C0C0E0D0E0CA3FD105F8F444
:103B4000C7BD82E390E00E94C3198DE994E09F9382
:103B50008F9382E995E19F938F93E0918E03F0918B
:103B60008F03099580911401909115010F900F908A
:103B70000F900F908052934010F02196DECFC093AB
:103B80007A058091DB0580FF09C08C2F8A508B3E1F
:103B900028F08091A70380648093A703C7BD8CE2BF
:103BA00091E00E94C319DF91CF910895EF92FF92A7
:103BB0001F93CF9310E080ED97E00E94A1197C0144
:103BC000CCE8133019F4CB3008F0C9E010E0809154
:103BD000FF01909100028C5F934024F480911301C7
:103BE00081500AC08091FF0190910002875094405B
:103BF00034F0809113018F5F8093130101C011E0B5
:103C00008091FD019091FE018C5F934024F480919E
:103C1000120181500AC08091FD019091FE018750F0
:103C2000944034F0809112018F5F8093120101C0A3
:103C30001F5F8091FB019091FC018C5F934024F405
:103C40008091110181500AC08091FB019091FC018B
:103C500087509440C4F0809111018F5F80931101CF
:103C600013C08FE994E09F938F9382E995E19F932E
:103C70008F93E0918E03F0918F0309950F900F9031
:103C80000F900F905FC01F5F82E180932A028091A6
:103C900024028E7F8093240285EA8093BC00809169
:103CA00013018A3040F48091A70381608093A703B9
:103CB0008AE08093130180911301863F40F0809148
:103CC000A70381608093A70385EF80931301809100
:103CD00012018A3040F48091A70382608093A70389
:103CE0008AE08093120180911201863F40F080911A
:103CF000A70382608093A70385EF809312018091D0
:103D000011018A3040F48091A70384608093A70357
:103D10008AE08093110180911101863F40F08091EB
:103D2000A70384608093A70385EF8093110180919E
:103D30002A02882339F0C7010E94AA19882309F0B2
:103D400090CFF5CF109210018FEC80937A00809184
:103D500010018823E1F3CA3020F48AE090E00E9449
:103D6000C319C15009F02DCF86E490E00E94C31919
:103D7000CF911F91FF90EF9008951F920F920FB671
:103D80000F921124EF92FF920F931F932F933F9363
:103D90004F935F936F937F938F939F93AF93BF9353
:103DA000EF93FF9380910802282F3327442755274C
:103DB0008F5F80930802F9012231310508F0E6C3D4
:103DC000EA5BFF4F0C94218B8091780090917900F1
:103DD00046C080917800909179004AC18091780026
:103DE0009091790090930B0280930A0275C18091A3
:103DF000CF029091D0022091780030917900821BFF
:103E0000930B90936B0580936A0580916A0590915E
:103E10006B0590931502809314027CC18091780009
:103E2000909179002091D1023091D202821B930BA4
:103E30009093790580937805809178059091790524
:103E40009093170280931602A3C380910E02909163
:103E50000F022091780030917900820F931F909388
:103E60000F0280930E0281E094C380910C02909126
:103E70000D022091780030917900820F931F90936A
:103E80000D0280930C0284E084C38091380683FF86
:103E90001AC080911E0190911F019C01220F331FB7
:103EA000280F391F40917800509179008BE090E005
:103EB000489FB001499F700D589F700D1124CB0190
:103EC0006EE170E00FC080911E0190911F019C0176
:103ED000220F331F280F391F8091780090917900AD
:103EE00063E070E00E94868A260F371F369527957B
:103EF0003695279530931F0120931E0185E049C315
:103F000080917800909179004091CB025091CC0241
:103F1000841B950B9093F6018093F5018091F50138
:103F20009091F601029704F172E04E3E570784F437
:103F3000209109022B5F20930902255080913702BE
:103F400090913802845F914018F4215F2093090218
:103F500080910902853684F14F5F5F4F5093CC0208
:103F60004093CB02845626C08091F5019091F601D2
:103F70008F5F9F4F0CF572E047325707ECF02091AE
:103F800009022550209309022B5F809137029091FE
:103F90003802845F914018F42F50209309028091D9
:103FA00009028C394CF4415050405093CC0240935C
:103FB000CB028C598093090281E08093F4018091B7
:103FC00078009091790090937105809370058091AD
:103FD000F5019091F6019C01442737FD4095542F3F
:103FE0008091860290918702A0918802B091890207
:103FF000820F931FA41FB51F8093860290938702A0
:10400000A0938802B09389022091860230918702A2
:10401000409188025091890257FF04C021503C4FC3
:104020004F4F5F4F6AE055954795379527956A95AD
:10403000D1F78091860290918702A0918802B09179
:104040008902821B930BA40BB50B8093860290937D
:104050008702A0938802B09389022EC180910C023E
:1040600090910D022091780030917900820F931F7A
:1040700090930D0280930C02109207028CC28091E3
:1040800002018A3071F4809178009091790020913A
:104090000A0230910B02820F931F01969695879525
:1040A00017C040910A0250910B02843158F02091C0
:1040B000780030917900240F351F8FEF97E0821B35
:1040C000930B06C08091780090917900840F951F22
:1040D0009093FC018093FB0186E05BC28091CF024C
:1040E0009091D0022091780030917900821B930B3F
:1040F00090936B0580936A0580916A0590916B059A
:104100002091140230911502820F931F9093FA01AF
:104110008093F90187E03DC2809178009091790009
:104120002091D1023091D202821B930B909379059A
:1041300080937805809178059091790520911602F9
:1041400030911702820F931F9093F8018093F7012B
:104150001FC220910E0230910F0280917800909141
:104160007900280F391F30930F0220930E0280919F
:1041700002018A3019F4220F331F04C0220F331FAB
:10418000220F331F30930F0220930E0220910E0254
:1041900030910F02C90137FD079603E09595879589
:1041A0000A95E1F7909300028093FF01809110023D
:1041B00090911102820F931F97FD01969595879517
:1041C00090931102809310022091DB023091DC0267
:1041D000821B930B90931D0180931C01209105027B
:1041E0003091060280911C0190911D01280F391F0A
:1041F00037FF02C02F5F3F4F35952795309306025A
:104200002093050230CE20910C0230910D02809156
:10421000780090917900280F391F30930D02209378
:104220000C02809102018A3019F4220F331F04C05E
:10423000220F331F220F331F30930D0220930C02E5
:1042400020910C0230910D02C90137FD0796F3E071
:1042500095958795FA95E1F79093FE018093FD017E
:104260008091120290911302820F931F97FD019685
:104270009595879590931302809312022091D9020D
:104280003091DA02821B930B90931B0180931A01E9
:10429000209103023091040280911A0190911B0138
:1042A000280F391F37FF02C02F5F3F4F35952795E5
:1042B000309304022093030283E06BC11092080242
:1042C00081E0809310018091EB019091EC010196C7
:1042D0009093EC018093EB018091780090917900AC
:1042E0009093150180931401809114019091150110
:1042F000AA27BB27209118023091190240911A0277
:1043000050911B02280F391F4A1F5B1F2093180270
:104310003093190240931A0250931B0280911C02A1
:104320008F5F80931C02823108F432C180911601A4
:1043300090911701A0911801B09119017C018D0194
:1043400063E0EE0CFF1C001F111F6A95D1F7E81AFD
:10435000F90A0A0B1B0BE20EF31E041F151F8091B6
:10436000EF01992787FD9095A92FB92FBC01CD01A9
:1043700026EC34E240E050E00E945B8ADC01CB0195
:10438000E81AF90A0A0B1B0BD801C7010496A11DF4
:10439000B11DB7FF05C0D801C7010B96A11DB11D06
:1043A00023E0B595A795979587952A95D1F78093A2
:1043B000160190931701A0931801B09319018091F1
:1043C0007205909173057C010027F7FC0095102F72
:1043D0008091160190911701A0911801B0911901D7
:1043E000E81AF90A0A0B1B0BE0926602F0926702C8
:1043F00000936802109369022091F0013091F1015D
:104400004091F2015091F30157FF04C0215F3F4FEB
:104410004F4F5F4F84E055954795379527958A957F
:10442000D1F78091F0019091F101A091F201B0914A
:10443000F301821B930BA40BB50B8093F0019093B7
:10444000F101A093F201B093F3018091F0019091FA
:10445000F101A091F201B091F3018E0D9F1DA01FFB
:10446000B11F8093F0019093F101A093F201B093FA
:10447000F3018091F0019091F101A091F201B091CE
:10448000F301B7FF03C00F96A11DB11D14E0B59550
:10449000A795979587951A95D1F720916602309147
:1044A0006702281B390B64E0213036071CF020E03E
:1044B00034E006C07CEF2030370714F420E03CEFF6
:1044C0008091ED019091EE018091ED019091EE01CE
:1044D00097FF03C0909581959F4FA901F3E0440F8A
:1044E000551FFA95E1F78D5B9240C4F08091ED0184
:1044F0009091EE019C01E4E0220F331FEA95E1F771
:10450000281B390B240F351F37FF02C0215F3F4F97
:1045100074E0359527957A95E1F717C08091ED0104
:104520009091EE019C0165E0220F331F6A95E1F73F
:10453000281B390B240F351F37FF02C0215E3F4F68
:1045400045E0359527954A95E1F73093EE012093A4
:10455000ED018091180290911902A0911A02B09178
:104560001B02B7FF03C00196A11DB11DB595A7950C
:10457000979587958093180290931902A0931A0239
:10458000B0931B0289E080931C0202C010920802C3
:1045900082E0809307028091070280937C008091E3
:1045A0000802882319F08FEC80937A00FF91EF9135
:1045B000BF91AF919F918F917F916F915F914F913B
:1045C0003F912F911F910F91FF90EF900F900FBE91
:1045D0000F901F90189590E2EDE7F5E08FE491932E
:1045E000815087FFFCCF089590911F02903540F4D1
:1045F000E92FFF27E358FA4F80839F5F90931F02B4
:104600000895AF92BF92CF92DF92FF920F931F93C4
:10461000CF93DF9320911D0220FF0AC080911E02DC
:10462000882311F0815002C08091200180931E02E6
:1046300021FF0CC090911E0280912001981719F45F
:1046400010921E0203C09F5F90931E02822F992733
:1046500080FF04C081FF02C010921E020E94EB2264
:1046600080911E02282F332794EFC92E92E2D92E73
:10467000C0918E03D0918F038A3098F481E18093AA
:104680001F023F932F9386ED94E09F938F93DF92C9
:10469000CF92FE0109952DB73EB72A5F3F4F2DBF40
:1046A00011C080E180931F023F932F938BED94E024
:1046B0009F938F93DF92CF92FE0109958DB79EB79E
:1046C00006968DBF20911E02822F9927AA27BB270D
:1046D000FC01419710F00C94592CE85AFF4F04EF5D
:1046E000C02E02E2D02EC0918E03D0918F030C9485
:1046F000218B10921F0280EE94E09F938F9304EF22
:1047000012E2DF92CF92FE01099584E180931F02AD
:104710000F900F900F900F9084E690E09F938F93EF
:1047200086E590E09F938F931F921F9280910201E4
:104730006AE00E947A8A892F99279F938F938091AC
:1047400002010E947A8A99279F938F9380EF94E0C9
:104750009F938F93DF92CF92E0918E03F0918F031E
:10476000099588E280931F02EDB7FEB73E96EDBF34
:1047700087E496E09F938F930E94C52F99279F937C
:104780008F9385E095E09F938F93DF92CF92E09196
:104790008E03F0918F0309958091A80399272DB777
:1047A0003EB7285F3F4F2DBFEC01C071D07084FF32
:1047B00006C08CE380931F0283E195E0F1C09091E5
:1047C0004603992349F18CE380931F02892F99278F
:1047D0009F938F9380E295E09F938F931F930F9306
:1047E000E0918E03F0918F030995DF93CF93909121
:1047F000460381E1989FC00111248559944F9F93EE
:104800008F931F930F93E0918E03F0918F0309957F
:104810008DB79EB70C9647C19091A7039923B1F02D
:104820008CE380931F02892F99279F938F9388E2AF
:1048300095E09F938F931F930F93E0918E03F091D8
:104840008F030995EDB7FEB7369679C4909125028E
:10485000992371F08CE380931F02892F99279F93EE
:104860008F938FE395E09F938F931F930F93D9C4FA
:1048700080913D0190913E01069710F00C94622CBE
:104880008CE380931F0284E595E0A5C78091B6076D
:1048900014EFC12E12E2D12EC0918E03D0918F035E
:1048A00080FF6BC010921F02809166029091670298
:1048B000A0916802B0916902BC01CD0125E030E011
:1048C00040E050E00E94CF8A3F932F9381E695E02D
:1048D0009F938F93DF92CF92FE01099584E180939D
:1048E0001F028DB79EB706968DBF80916202909190
:1048F0006302A0916402B0916502BC01CD0125E084
:1049000030E040E050E00E94CF8A3F932F938EE644
:1049100095E09F938F93DF92CF92E0918E03F09179
:104920008F03099588E280931F02EDB7FEB7369694
:10493000EDBF80911401909115019F938F938BE7A8
:1049400095E09F938F93DF92CF92E0918E03F09149
:104950008F0309958CE380931F022DB73EB72A5F22
:104960003F4F2DBF87B599279F938F9388E895E098
:104970009F938F93DF92CF928EC010921F0285E992
:1049800095E09F938F93DF92CF92FE01099584E18A
:1049900080931F020F900F900F900F9084EA95E084
:1049A0009F938F93DF92CF921AC710921F028DEAC6
:1049B00095E09F938F9304EF12E2DF92CF92FE0176
:1049C000099584E180931F020F900F900F900F9034
:1049D0008091C6029091C702A091C802B091C9020D
:1049E000B7FF04C081509C4FAF4FBF4FCAE0B59591
:1049F000A79597958795CA95D1F7BF93AF939F9346
:104A00008F938AEB95E09F938F931F930F93E09181
:104A10008E03F0918F03099588E280931F02EDB712
:104A2000FEB73896EDBF8091BE029091BF02A09173
:104A3000C002B091C102B7FF04C081509C4FAF4F7C
:104A4000BF4FFAE0B595A79597958795FA95D1F759
:104A5000BF93AF939F938F9389EC95E09F938F9330
:104A60001F930F93E0918E03F0918F0309958CE3D0
:104A700080931F022DB73EB7285F3F4F2DBF809117
:104A80007307909174079F938F9388ED95E09F93A0
:104A90008F931F930F93E0918E03F0918F030995ED
:104AA0008DB79EB706968DBF0DC7E1E0FE2EC1E023
:104AB000D0E00FEF16E09F2D969584E1989FC001FE
:104AC000112480931F02F801828193819F938F9319
:104AD0002196DF93CF932197808191819F938F932C
:104AE000DF93CF9387EE95E09F938F9384EF92E2CD
:104AF0009F938F93E0918E03F0918F0309952DB7CB
:104B00003EB7245F3F4F2DBF32E0F30E22960C5F7D
:104B10001F4F88E08F1578F6D5C610921F0280913E
:104B2000D005E82FFF27EE0FFF1FE350F94F8081DC
:104B300091819F938F938091CF05E82FFF27EE0FF0
:104B4000FF1FE350F94F808191819F938F9389EFED
:104B500095E09F938F93DF92CF92FE01099584E1B8
:104B600080931F02EDB7FEB73896EDBF8091D20556
:104B7000E82FFF27EE0FFF1FE350F94F808191814F
:104B80009F938F938091D105E82FFF27EE0FFF1F92
:104B9000E350F94F8081918181589F4F9F938F936C
:104BA00089E096E09F938F93DF92CF92E0918E03FE
:104BB000F0918F03099588E280931F022DB73EB7CD
:104BC000285F3F4F2DBF8091D405E82FFF27EE0FC0
:104BD000FF1FE350F94F8081918181589F4F9F9330
:104BE0008F938091D305E82FFF27EE0FFF1FE3502F
:104BF000F94F8081918181589F4F9F938F9389E1D5
:104C000096E09F938F93DF92CF92E0918E03F09185
:104C10008F0309958CE380931F028DB79EB708968A
:104C20008DBF8091D605E82FFF27EE0FFF1FE350C1
:104C3000F94F8081918181589F4F9F938F938091ED
:104C4000D505E82FFF27EE0FFF1FE350F94F8081B6
:104C5000918181589F4F9F938F9389E296E063C221
:104C600010921F0289E396E09F938F9304EF12E264
:104C7000DF92CF92FE010995809102010F900F9073
:104C80000F900F908A3009F09DC084E180931F023D
:104C90008091DB029091DC029C0197FF02C0295FAA
:104CA0003F4F287F821B930B9F938F938091DB0252
:104CB0009091DC0297FD079673E0959587957A951C
:104CC000E1F79F938F932091DB023091DC0237FF55
:104CD00002C0295F3F4F63E0359527956A95E1F75C
:104CE0008091FF0190910002821B930B9F938F9301
:104CF00087E496E09F938F931F930F93E0918E0329
:104D0000F0918F03099588E280931F022DB73EB77B
:104D1000265F3F4F2DBF8091D9029091DA029C010E
:104D200097FF02C0295F3F4F287F821B930B9F9301
:104D30008F938091D9029091DA0297FD079653E004
:104D4000959587955A95E1F79F938F932091D90276
:104D50003091DA0237FF02C0295F3F4F43E03595BB
:104D600027954A95E1F78091FD019091FE01821B04
:104D7000930B9F938F9388E596E09F938F931F9358
:104D80000F93E0918E03F0918F0309958CE380934C
:104D90001F028DB79EB70A968DBF8091D702909162
:104DA000D8029F938F938091D7029091D80220913F
:104DB000FB013091FC01821B930B9F938F9389E63B
:104DC00096E0ADC08B3019F0843108F4ADC084E1B9
:104DD00080931F028091DB029091DC029C0197FF7F
:104DE00002C0215F3F4F207F821B930B97FD0196EE
:104DF000959587959F938F938091DB029091DC022C
:104E000097FD0F9624E0959587952A95E1F79F9356
:104E10008F932091DB023091DC0237FF02C0295FC3
:104E20003F4FC3E035952795CA95E1F78091FF0183
:104E300090910002821B930B9F938F9387E796E0DC
:104E40009F938F931F930F93E0918E03F0918F03A5
:104E5000099588E280931F022DB73EB7265F3F4F2A
:104E60002DBF8091D9029091DA029C0197FF02C078
:104E7000215F3F4F207F821B930B97FD01969595F5
:104E800087959F938F938091D9029091DA0297FD35
:104E90000F96A4E095958795AA95E1F79F938F9338
:104EA0002091D9023091DA0237FF02C0295F3F4FCB
:104EB000F3E035952795FA95E1F78091FD01909102
:104EC000FE01821B930B9F938F9389E896E09F933B
:104ED0008F931F930F93E0918E03F0918F030995A9
:104EE0008CE380931F028DB79EB70A968DBF809189
:104EF000D7029091D80297FD0196959587959F933B
:104F00008F938091D7029091D8022091FB0130912C
:104F1000FC01821B930B9F938F938BE996E09F93E9
:104F20008F931F930F9303C18D3009F0CBC484E19D
:104F300080931F028091130199279F938F938091F3
:104F4000DB029091DC0297FD0F9674E095958795B2
:104F50007A95E1F79F938F932091DB023091DC02E9
:104F600037FF02C0295F3F4F63E0359527956A956B
:104F7000E1F78091FF0190910002821B930B9F93B8
:104F80008F938AEA96E09F938F931F930F93E091FC
:104F90008E03F0918F03099588E280931F022DB74D
:104FA0003EB7265F3F4F2DBF8091120199279F93F7
:104FB0008F938091D9029091DA0297FD0F9654E079
:104FC000959587955A95E1F79F938F932091D902F4
:104FD0003091DA0237FF02C0295F3F4F43E0359539
:104FE00027954A95E1F78091FD019091FE01821B82
:104FF000930B9F938F938EEB96E09F938F931F93CA
:105000000F93E0918E03F0918F0309958CE38093C9
:105010001F028DB79EB70A968DBF80911101992707
:105020009F938F938091D7029091D80297FD01961C
:10503000959587959F938F938091D7029091D802F1
:105040002091FB013091FC01821B930B9F938F9366
:1050500082ED96E09F938F931F930F93E0918E03C1
:10506000F0918F030995EDB7FEB73A9668C010929C
:105070001F0286EE96E09F938F93DF92CF92FE0100
:10508000099584E180931F020F900F900F900F906D
:105090008091D1029091D2029F938F938091F701DA
:1050A0009091F8019F938F9383EF96E09F938F9356
:1050B000DF92CF92E0918E03F0918F03099588E201
:1050C00080931F022DB73EB7285F3F4F2DBF8091C1
:1050D000CF029091D0029F938F938091F90190918C
:1050E000FA019F938F9382E097E09F938F93DF92D3
:1050F000CF92E0918E03F0918F0309958CE380931A
:105100001F028DB79EB708968DBF8091CB029091FC
:10511000CC029F938F938091F5019091F6019F931C
:105120008F9381E197E09F938F93DF92CF92E091ED
:105130008E03F0918F030995EDB7FEB73896EDBF5A
:10514000C1C310921F0280911E0190911F016AE05D
:1051500070E00E949A8A9F938F9380911E01909194
:105160001F016AE070E00E949A8A7F936F9380E249
:1051700097E09F938F93DF92CF92FE01099584E190
:1051800080931F022DB73EB7285F3F4F2DBF809100
:105190004B0890914C086AE070E00E94868A9F93C9
:1051A0008F9380914B0890914C086AE070E00E94C8
:1051B000868A7F936F9384E397E09F938F93DF9228
:1051C000CF92E0918E03F0918F03099588E280934E
:1051D0001F028DB79EB708968DBF80914D089091A4
:1051E0004E089F938F9388E497E09F938F93DF926D
:1051F000CF92E0918E03F0918F0309958CE3809319
:105200001F02EDB7FEB73696EDBF80914F08909123
:1052100050089F938F9388E597E09F938F93DF9239
:10522000CF92E0918E03F0918F0309952DB73EB791
:105230002A5F3F4F4FC110921F028AE697E09F936B
:105240008F93DF92CF92FE01099584E180931F0234
:105250000F900F900F900F908091FD069091FE0699
:105260009F938F9383E797E09F938F93DF92CF92E3
:10527000E0918E03F0918F03099588E280931F02DD
:105280008DB79EB706968DBF80916C0299279F932C
:105290008F9383E897E09F938F93DF92CF92E09173
:1052A0008E03F0918F0309958CE380931F02EDB775
:1052B000FEB73696EDBF8091FC06992701979F9324
:1052C0008F9383E997E0A9CF10921F0283EA97E0BA
:1052D0009F938F93DF92CF92FE01099584E1809393
:1052E0001F020F900F900F900F9080918F0190915F
:1052F00090019F938F938BEA97E09F938F93DF9218
:10530000CF92E0918E03F0918F03099588E280930C
:105310001F028DB79EB706968DBF8091730790913F
:1053200074079F938F9389EB97E09F938F93DF92FE
:10533000CF92E0918E03F0918F0309958CE38093D7
:105340001F02EDB7FEB73696EDBF809184029091B3
:1053500085029F938F9387EC97E05FCFCDE6CC2EAD
:10536000C2E0DC2E20E030E0E901B3E0FB2EC09388
:105370001F02F60181916F0199279F938F938901F5
:105380000F5F1F4F1F930F9385ED97E09F938F93B0
:1053900084EF92E29F938F93E0918E03F0918F03BD
:1053A00009952DB73EB7285F3F4F2DBFFA946496FD
:1053B0009801F7FEDCCF86C2A1E7CA2EA2E0DA2E62
:1053C000C0E0D0E08E01F3E0FF2E00931F02F60153
:1053D00081916F0199279F938F932596DF93CF93A8
:1053E00082EE97E09F938F9384EF92E29F938F9347
:1053F000E0918E03F0918F0309952DB73EB7285F9A
:105400003F4F2DBFFA940C5E1F4F2497F7FEDDCF60
:1054100059C210921F028FEE97E09F938F9304EF73
:1054200012E2DF92CF92FE01099584E180931F0280
:105430000F900F900F900F9080916E0199279F937E
:105440008F9387EF97E09F938F93DF92CF92E091B6
:105450008E03F0918F03099588E280931F028DB728
:105460009EB706968DBF8091D6019091D70197FD8A
:10547000039695958795959587959F938F9385E04E
:1054800098E09F938F931F930F93E0918E03F09179
:105490008F0309958CE380931F02EDB7FEB7369614
:1054A000EDBF8091FE0599279F938F938091FD0515
:1054B00099279F938F9383E198E09F938F931F93F6
:1054C0000F93E0918E03F0918F0309952DB73EB7AE
:1054D000285F3F4F2DBFF6C110921F0281E298E076
:1054E0009F938F9374EFA72E72E2B72EDF92CF9225
:1054F000FE0109950F900F900F900F90CCE9D6E028
:1055000000E010E062E0F62E802F8C5E80931F0298
:105510008B8D99278F7790709F938F938B89992785
:105520008F7790709F938F938B8599278F7790704B
:105530009F938F938B8199278F7790709F938F93F1
:1055400081E398E09F938F93BF92AF92E0918E0397
:10555000F0918F0309958DB79EB70C968DBFFA9485
:105560000C5E1F4FA096F7FECFCFACC110921F026A
:1055700082E498E09F938F9354EFA52E52E2B52ECC
:10558000DF92CF92FE0109950F900F900F900F9030
:10559000CCE9D6E000E010E042E0F42E802F8C5EF3
:1055A00080931F028F8D992787FD90959F938F93EE
:1055B0008F89992787FD90959F938F938F85992742
:1055C00087FD90959F938F938F81992787FD909565
:1055D0009F938F9381E598E09F938F93BF92AF92B3
:1055E000E0918E03F0918F030995EDB7FEB73C96DD
:1055F000EDBFFA940C5E1F4FA096F7FECFCF62C1AD
:1056000010921F0282E698E09F938F9304EF12E2BC
:10561000DF92CF92FE01099584E180931F020F90E3
:105620000F900F900F908091B706881F8827881FD2
:1056300097E0899FC00111248D969F938F9380914D
:10564000AF06881F8827881F96E0899FC001112414
:105650008D969F938F938091A706881F8827881F18
:1056600095E0899FC00111248D969F938F9380911F
:105670009F06881F8827881F9927880F991F880FE2
:10568000991F8D969F938F9381E798E09F938F93B7
:10569000DF92CF92E0918E03F0918F03099588E21B
:1056A00080931F022DB73EB7245F3F4F2DBF8091DF
:1056B000D706881F8827881F9BE0899FC001112477
:1056C0008D969F938F938091CF06881F8827881F80
:1056D0009AE0899FC00111248D969F938F938091AA
:1056E000C706881F8827881F99E0899FC001112459
:1056F0008D969F938F938091BF06881F8827881F60
:10570000992723E0880F991F2A95E1F78D969F939B
:105710008F9385E898E09F938F93DF92CF92E091EB
:105720008E03F0918F0309958CE380931F028DB750
:105730009EB70C968DBF8091DF06881F8827881F33
:105740009CE0899FC00111248D969F938F9389E9D6
:1057500098E09F938F93DF92CF92E0918E03F09128
:105760008F0309958091E706EDB7FEB73696EDBF3A
:1057700087FF12C080E480931F028AEA98E09F931B
:105780008F93DF92CF92E0918E03F0918F03099572
:105790000F900F900F900F908091EF0687FF12C02F
:1057A00084E480931F028DEA98E09F938F931F9368
:1057B0000F93E0918E03F0918F0309950F900F9056
:1057C0000F900F908091F70687FF7CC088E480934C
:1057D0001F0280EB98E09F938F931F930F93E091AC
:1057E0008E03F0918F0309950F900F900F900F90FB
:1057F00069C010921F0283EB98E09F938F93DF9212
:10580000CF92FE01099584E180931F020F900F90C3
:105810000F900F908091AC019091AD019F938F9369
:1058200081EC98E09F938F93DF92CF92E0918E036B
:10583000F0918F03099588E280931F022DB73EB740
:105840002A5F3F4F2DBF8091AE019091AF019F9392
:105850008F938EEC98E09F938F93DF92CF92E0919D
:105860008E03F0918F03099589E480931F028DB711
:105870009EB706968DBF8BED98E09F938F93DF9236
:10588000CF92E0918E03F0918F03099580911D02D4
:105890000F900F900F900F9083FF14C01092AF01E4
:1058A0001092AE0160E070E08EE090E00E946D2EFC
:1058B00009C080912001281719F42150209320015C
:1058C00010921E0210921D02DF91CF911F910F9135
:1058D000FF90DF90CF90BF90AF900895F999FECFE1
:1058E00092BD81BDF89A80B599270895F999FECFA8
:1058F0001FBA92BD81BD60BD0FB6F894FA9AF99AAD
:105900000FBE08954AEA20E030E02617370740F43A
:10591000FC018191480F2F5F3F4F26173707C8F3CF
:10592000842F99270895EAEA40E050E04617570788
:1059300078F49C01F999FECF32BD21BDF89A80B56B
:10594000E80F4F5F5F4F2F5F3F4F4617570790F3AA
:105950008E2F9927089581E08093D10582E080936E
:10596000D00583E08093CF0584E08093D20585E065
:105970008093D30586E08093D40587E08093D50596
:1059800088E08093D60589E08093D7058AE08093EC
:10599000D8058BE08093D9058CE08093DA050895D3
:1059A00088E58093CE0580910201843150F08AE031
:1059B0008093EE05109212068BE18093EA058EE447
:1059C0000AC083E08093EE0580E2809312068EE1A8
:1059D0008093EA0585E580930F068093100680E2A8
:1059E000809311068AE68093DB0582E28093380675
:1059F00064E06093F5051092310610922E0648E09F
:105A00004093E80556EE5093E90530E43093EB05FA
:105A10009EE19093DC058FEF8093DE052FE02093CD
:105A2000DF059093DD051092E1054093E205309388
:105A3000E3051092E4052093E0051092F70510921B
:105A4000F8051092F9051092FA05109214061092BA
:105A50001506109216061092170690E89093FB0513
:105A600032E33093FC0582E0809337062093FD05F6
:105A70005093FE05609303068DE78093060680939E
:105A80000706809308069093FF0525E520930006FE
:105A900086E4809301068CED809302068CE380936C
:105AA0000406109205068FE58093180683EF809315
:105AB0001A068AEA80931C0680931D0684E180936F
:105AC000190680931B06309309069AE590930A06FF
:105AD00030930B06109236068EEF80931E0684E6F6
:105AE00080931F06909320069093210690932206A0
:105AF0008BE480932306209324068093250610923E
:105B0000260686E080932706409328069093290670
:105B10008AE280932A0685EF80932B068CE8809397
:105B20002C0685E080932D0610922F0610923006E9
:105B300081E28093F2058DE28093F3059093F40562
:105B400010923206109233061092340686E9809342
:105B5000350690930C0687E380930D060895CF9346
:105B6000DF930E94D02C8AE08093E50580E180934A
:105B7000E60526E02093E7059AE59093EC0588E793
:105B80008093ED059093EF058093F0052093F10548
:105B900080E28093F6058CE380930E068BE480937D
:105BA0001306A9E3B6E08CE0E1E2F1E0ED0101903B
:105BB00009928A95E1F767E770E0CD018B56904036
:105BC0000E94822C80934506DF91CF910895CF9358
:105BD000DF930E94D02C88E08093E50530E130937C
:105BE000E60526E02093E70594E69093EC0588E728
:105BF0008093ED059093EF058093F0052093F105D8
:105C00003093F60586E480930E0680931306A9E38D
:105C1000B6E08CE0E7E2F1E0ED01019009928A95AF
:105C2000E1F767E770E0CD018B5690400E94822C2F
:105C300080934506DF91CF910895CF93DF930E9423
:105C4000D02C26E02093E5058AE08093E60584E0E9
:105C50008093E70594E69093EC0588E78093ED0543
:105C60009093EF058093F0052093F10580E18093F8
:105C7000F60586E480930E0680931306A9E3B6E04A
:105C80008CE0EFE2F1E0ED01019009928A95E1F7F5
:105C900067E770E0CD018B5690400E94822C809384
:105CA0004506DF91CF910895F999FECF92BD81BD50
:105CB000F89A80B599270895F999FECF1FBA92BD39
:105CC00081BD60BD0FB6F894FA9AF99A0FBE089597
:105CD0006EE67CE20E94E988089546E75CE20E9455
:105CE00023890895EF92FF920F931F93CF93C82FAC
:105CF0008150853008F0C3E088E7C89F80011124F7
:105D00008CEEE82E8FEFF82EE00EF11E67E770E0C4
:105D1000C7010E94932C682F98012D593F4F8FB3D4
:105D20009927AC014270507081FDF9CF32BD21BD81
:105D3000F89A80B5861711F0CA0123C08FB399274E
:105D40009C012270307081FDF9CFF2BCE1BCF89A61
:105D500080B5883511F0C90114C088E7C89FC0011B
:105D6000112444972EE63CE248E750E0BC018EEC5B
:105D700095E00E94C4880E94DC690E942E8481E024
:105D800090E0CF911F910F91FF90EF900895282FF1
:105D9000863010F025E003C0882309F421E0F9994A
:105DA000FECF1FBA82E090E092BD81BD20BD0FB64C
:105DB000F894FA9AF99A0FBE0895CF93C82F80915C
:105DC000CE05883509F046C0C63010F0C5E003C0E6
:105DD000CC2309F43FC00E94468767E770E08EEC51
:105DE00095E00E94822C8093450688E7C89FC001F9
:105DF000112426E73CE248E750E06EEC75E044975A
:105E00000E94018926E73CE24CE050E06FEC75E02F
:105E100080E590E00E9401896CE070E08FEC95E0F5
:105E20000E94822C282FF999FECF1FBA8CE590E0B2
:105E300092BD81BD20BD0FB6F894FA9AF99A0FBEB3
:105E40008C2F0E94C72E0E94DC690E942E8481E064
:105E500090E002C080E090E0CF9108956DE470E0A2
:105E600088EE93E00E94932C482F8FB399279C01D2
:105E70002270307081FDF9CF85E394E092BD81BD41
:105E8000F89A80B5841779F48FB399279C01227012
:105E9000307081FDF9CF88EE93E092BD81BDF89A14
:105EA00080B5813011F0C90108952EE63CE24EE440
:105EB00050E068EE73E086E496E00E94C48881E0DA
:105EC00090E00895809146068130A9F46DE470E079
:105ED00086E496E00E94822C8093930626E73CE2BB
:105EE0004EE450E066E476E088EE93E00E9401899B
:105EF00081E090E0089580E090E00895CF93DF93F3
:105F000081E080934606E6E4F6E08FE0158616868B
:105F10001786108A8150349687FFF8CF80E48093EB
:105F2000530680935406109255068093560680932C
:105F3000570690EC909358061092590680935A0693
:105F400080935B0610925C0690935D0690935E06CC
:105F500080935F06109260068093610690936206BC
:105F6000A7E4B6E087E0E5E3F1E0ED0101900992F6
:105F70008A95E1F76DE470E0CD0101970E94822CD3
:105F800080939306DF91CF910895F999FECF82E037
:105F900090E092BD81BDF89A80B5282F863078F0C8
:105FA00023E0322FF999FECF1FBA82E090E092BD34
:105FB00081BD30BD0FB6F894FA9AF99A0FBE822FC0
:105FC000992708951F93CF93C82F162F863010F06E
:105FD000C5E003C0882309F4C1E08C2F99278230E3
:105FE000910541F08330910544F4019731F40E940A
:105FF000AF2D05C00E94E72D02C00E941D2E112367
:10600000E1F06CE070E080E590E00E94932C282F96
:10601000F999FECF8CE590E092BD81BDF89A80B5EC
:10602000821759F42EE63CE24CE050E060E570E067
:106030008FEC95E00E94C48802C00E94AB2C8C2F8C
:106040000E94DD2ECF911F910895DF92EF92FF9273
:106050000F931F93CF93FF24DF2CEF2C81E090E070
:106060000E94542E883511F031E0E32E6CE070E090
:1060700080E590E00E94932CC82FF999FECF8CE523
:1060800090E092BD81BDF89A80B58C1711F421E0A3
:10609000D22EC1E001E010E0EE2029F48C2F0E9406
:1060A000722E8823C9F591E0F92E1F930F9383EE8A
:1060B00098E09F938F9382E995E19F938F93E0916E
:1060C0008E03F0918F0309952DB73EB72A5F3F4F9E
:1060D0002DBF0230110549F0033011054CF4013099
:1060E000110531F40E94AF2D05C00E94E72D02C0BA
:1060F0000E941D2EDD2059F02EE63CE24CE050E0DF
:1061000060E570E08FEC95E00E94C48802C00E94B8
:10611000AB2C8C2F0E94DD2ECF5F0F5F1F4FC63040
:1061200008F4BACFFF2019F083E00E94C72E0E9426
:10613000C52FC82F0E94722E8C2F99279F938F9363
:1061400089E099E09F938F9302E915E11F930F93E4
:10615000E0918E03F0918F03099581E090E00E9419
:10616000542E2DB73EB72A5F3F4F2DBF8F3F21F0F2
:106170000E942E2F882399F482E299E09F938F93B7
:106180001F930F93E0918E03F0918F0309950E9466
:106190007E2F0E94622F0F900F900F900F90EE2095
:1061A00029F068E581E090E00E945C2E1092CD0518
:1061B00090E0E3E5F6E0CFE08081349618160CF429
:1061C0009F5FC150C7FFF8CF9093CD05892F9927C6
:1061D0009F938F9387E496E09F938F9383E499E056
:1061E0009F938F931F930F93E0918E03F0918F03F2
:1061F00009958DB79EB708968DBF84E699E09F9369
:106200008F931F930F93E0918E03F0918F03099565
:106210000F900F900F900F90CF911F910F91FF90C3
:10622000EF90DF900895982F2FB7F8943998389A07
:1062300088B1836088B98091B9008C7F8093B90060
:106240008AE28093B80010922A02109228021092DB
:106250002702992379F0ECE9F6E08BE010821182B5
:106260001282138214821582168217828150389608
:1062700087FFF4CF78942FBF089510922A0284E903
:106280008093BC0080E88093BC001092BD00109207
:10629000BA001092BB001092B9001092B800109290
:1062A000260280E00E9413311092BB0085E88093A3
:1062B000BC008091240282608093240208951F9282
:1062C0000F920FB60F9211242F933F934F935F932A
:1062D0008F939F93EF93FF9380912A02282F332768
:1062E000442755278F5F80932A02F9012731310512
:1062F00008F0C2C2E759FF4F0C94218B81E08093D4
:10630000260209C0809128028C3090F480912802E6
:106310008F5F8093280280912802E82FFF27EE0FDD
:10632000FF1FEE0FFF1FEA5BF94F8585181654F724
:10633000809128028C3070F0109223021092220279
:106340001092280285E080932A0280912702880F0C
:106350008D5A04C080912802880F8E5A8093BB000A
:1063600085E87FC280912802E82FFF2783E0EE0FA7
:10637000FF1F8A95E1F7E456F94F81818093BB00B6
:1063800085E88093BC0080912802E82FFF27EE0F5C
:10639000FF1FEE0FFF1FEE0FFF1FE456F94F808126
:1063A00080FF91C080912802E82FFF27EE0FFF1F8A
:1063B000EE0FFF1FEE0FFF1FE456F94F8281882377
:1063C00029F08091CD05873008F46CC280912202BB
:1063D00090912302892B09F065C28091200290914F
:1063E0002102892B09F05EC26EC08091280221E053
:1063F00030E002C0220F331F8A95E2F7809120021D
:106400009091210228233923232B79F080912802AF
:10641000E82FFF27EE0FFF1FEE0FFF1FEE0FFF1FEE
:10642000E456F94F80E184830DC080912802E82F63
:10643000FF27EE0FFF1FEE0FFF1FEE0FFF1FE456AB
:10644000F94F148280912802E82FFF2753E0EE0FC6
:10645000FF1F5A95E1F7E456F94F8481282F33271F
:1064600043E0220F331F4A95E1F780912802E82F7D
:10647000FF2793E0EE0FFF1F9A95E1F7E456F94FDF
:1064800082818770822B8093BB0085E88093BC005B
:106490002091280281E090E002C0880F991F2A9580
:1064A000E2F7209122023091230282239323892B49
:1064B00051F084E996E090932E0280932D0288E0BB
:1064C00080932F02EFC184E089C1E0912D02F09109
:1064D0002E0281918093BB0085E88093BC00F093ED
:1064E0002E02E0932D0280912F02815080932F0283
:1064F000882309F4D7C183E071C18091B90080334A
:1065000051F580912B02882329F4809128028F5F16
:1065100080932B0280912802E82FFF2783E0EE0F63
:10652000FF1F8A95E1F7E456F94F838199278F770A
:1065300090708F3791057CF480912802E82FFF2717
:10654000EE0FFF1FEE0FFF1FEE0FFF1FE456F94F78
:1065500083818F5F838310922A0284E98093BC0039
:106560008AE090E090933E0180933D018091280263
:106570008F5F8093280210922A026DC18091B9002A
:106580008034C9F180912702E82FFF27EE0FFF1F0B
:10659000EE0FFF1FEE0FFF1FE456F94F83818F7739
:1065A0008383809127028F5F809327028091270247
:1065B0008C30A0F01092270210922102109220023B
:1065C00080912C028F5F80932C028C3038F01092D7
:1065D0002C02809124028D7F8093240280912402DA
:1065E00081608093240210922A0284E98093BC0087
:1065F0001092260273C080912702E82FFF27EE0F2A
:10660000FF1FEE0FFF1FEE0FFF1FE456F94F8381B0
:106610008068838380912702E82FFF27EE0FFF1FFA
:10662000EE0FFF1FEE0FFF1FE456F94F808180FF32
:106630002FC080912702E82FFF2753E0EE0FFF1FA6
:106640005A95E1F7E456F94F84819927009751F064
:106650004097D9F584E996E090932E0280932D021D
:1066600088E031C080912702992743E0880F991F65
:106670004A95E1F78F55994F90932E0280932D0202
:106680009091270280912C029817E1F483E01BC0BF
:1066900080912702992733E0880F991F3A95E1F7F7
:1066A0008F55994F90932E0280932D028091240252
:1066B00081FD06C09091270280912C02981711F459
:1066C00082E001C081E080932F0280912F0281300F
:1066D00011F485E801C085EC8093BC0080912B0209
:1066E0008093250210922B02DDC0E0912D02F091E3
:1066F0002E028091BB00808380912D0290912E020A
:10670000019690932E0280932D0280912F0281504A
:1067100080932F02823010F085EC5DC0813011F43F
:1067200085E859C08091240281FF2DC080913602F6
:1067300080FD1DC080912702E82FFF2723E0EE0F88
:10674000FF1F2A95E1F7E456F94F86818A3F79F4D5
:1067500080912702E82FFF2793E0EE0FFF1F9A9505
:10676000E1F7E456F94F8081816080830CC080910D
:106770002702E82FFF2783E0EE0FFF1F8A95E1F73E
:10678000E456F94F1082809127028F5F8093270291
:10679000809127028C30A0F01092270210922102E3
:1067A0001092200280912C028F5F80932C028C30FB
:1067B00038F010922C02809124028D7F8093240265
:1067C00010922A0284E98093BC00809124028160A7
:1067D0008093240265C08093BC0086E080932A02E7
:1067E00061C088E9BBCD80912902880F805FB6CD5A
:1067F0008091290299278130910561F082309105BD
:106800001CF4892B21F04EC0029739F04BC08091C7
:106810001301A4CD80911201A1CD809111019ECDD3
:1068200080E89CCD10922A0284E98093BC001092EB
:1068300026028AE090E090933E0180933D01809192
:106840002902823088F4809129028F5F8093290287
:1068500082E180932A02809124028E7F8093240219
:1068600085EA8093BC001EC0109229028091240208
:1068700081608093240216C010922A0284E98093DA
:10688000BC00809124028160809324028AE090E021
:1068900090933E0180933D011092280210922702AE
:1068A00010922602FF91EF919F918F915F914F91EE
:1068B0003F912F910F900FBE0F901F9018951F932F
:1068C000CF93DF93182F80916B02882321F480915E
:1068D000BB01882319F081E090E097C01D3008F0DB
:1068E00092C01123B1F0E12FFF2723E0EE0FFF1F2D
:1068F0002A95E1F7E456F94F35978081359688233C
:106900000CF081C03897808180FD03C083E090E067
:106910007CC080919406823019F084E090E075C0CC
:1069200067E070E084E996E00E94822C90919B06DB
:10693000891719F085E090E068C080ED97E00E942B
:10694000A119EC018091240280FD05C0CE010E94B6
:10695000AA198823B9F3112319F48FEF90E00BC023
:10696000212F33272150304081E090E002C0880F72
:10697000991F2A95E2F79093230280932202A1E0C7
:10698000B0E0ECE9F6E040E050E06BE0CD01042E31
:1069900002C0880F991F0A94E2F7209122023091D9
:1069A000230282239323892B11F0118212826150DA
:1069B0004F5F5F4F389667FFE9CF10922802109221
:1069C0002A02809124028E7F8093240285EA80939C
:1069D000BC008091240280FD05C0CE010E94AA194E
:1069E0008823B9F38091220290912302892B29F008
:1069F000CE010E94AA19882311F38091220290915E
:106A00002302009711F082E090E0DF91CF911F9177
:106A100008950F931F93CF93DF93982F80916B026C
:106A2000882321F48091BB01882319F081E090E054
:106A300092C09D30A0F4992319F486E090E08BC0B9
:106A4000C92FDD27FE0133E0EE0FFF1F3A95E1F776
:106A5000E456F94F35978081359687FD03C082E073
:106A600090E079C03897808180FD03C083E090E09A
:106A700072C080ED97E00E94A1198C0180912402E0
:106A800080FD05C0C8010E94AA198823B9F3219787
:106A900021E030E0C90102C0880F991FCA95E2F7D2
:106AA0009093210280932002D901ECE9F6E040E0C6
:106AB00050E06BE0CD01042E02C0880F991F0A94AC
:106AC000E2F7209120023091210282239323892B27
:106AD00011F01182128261504F5F5F4F389667FF4D
:106AE000E9CF109227021092940610929B06109202
:106AF0002A02809124028E7F8093240285EA80936B
:106B0000BC008091240280FD05C0C8010E94AA1922
:106B10008823B9F38091200290912102892B29F0DA
:106B2000C8010E94AA19882311F38091940682302B
:106B300019F084E090E00FC067E070E084E996E02F
:106B40000E94822C90919B06891719F085E090E0B5
:106B500002C080E090E0DF91CF911F910F910895E6
:106B6000CF93DF9380E022E83FEFC1E3D7E0EDEF82
:106B7000F6E0DF01853020F411961C921E9202C0CF
:106B8000318320831982188222968F5F1296329663
:106B90008A3180F31092D8021092D7021092DA0252
:106BA0001092D9021092DC021092DB02DF91CF9199
:106BB00008951F920F920FB60F9211240F931F93F7
:106BC0002F933F934F935F936F937F938F939F93F5
:106BD000AF93BF93CF93DF93EF93FF9340918600E2
:106BE000509187008091310290913202481B590BDD
:106BF000CA0157FD0196AC015595479580918600D5
:106C0000909187009093320280933102CA01895992
:106C10009840A0913302B0913402875E954338F4D6
:106C2000149714F01092410181E090E081C0AD30E2
:106C3000B1050CF081C0CA018B5F9040835694402F
:106C400008F071C0425C5340FD01EA0FFB1FE350A6
:106C5000F94F80819181FA01E81BF90BCF01F7FF11
:106C600003C0909581959F4F06974CF480916C02DC
:106C7000883C28F480916C02865F80936C02FD0151
:106C8000EA0FFB1FE350F94F808191819C01220F95
:106C9000331F280F391F240F351F37FF02C02D5F08
:106CA0003F4FE901D595C795D595C795CA0101967E
:106CB0008C179D0714F4219706C041505040C4170B
:106CC000D5070CF4219680916C02833CD8F08D019D
:106CD0000A0F1B1FF801E350F94F808191819E013B
:106CE000281B390BC90163E070E00E949A8ACB012E
:106CF000880F991F860F971F0F5C184FF80191831B
:106D0000808307C0AA0FBB1FAF5CB84F11961C92BF
:106D10001E92E0913302F0913402EE0FFF1FE35018
:106D2000F94FD183C0838091330290913402019650
:106D30009093340280933302FF91EF91DF91CF91D2
:106D4000BF91AF919F918F917F916F915F914F9183
:106D50003F912F911F910F910F900FBE0F901F9099
:106D60001895EF92FF920F931F938091EA05992750
:106D7000880F991F880F991F7C010027F7FC009549
:106D8000102F8091C6029091C702A091C802B091C5
:106D9000C902BC01CD01A80197010E94CF8A30939E
:106DA0002A05209329058091BE029091BF02A091EF
:106DB000C002B091C102BC01CD01A80197010E949F
:106DC000CF8A30932C0520932B058091BA079091A0
:106DD000BB0797FD03969595879595958795909315
:106DE0002E0580932D058091CA079091CB0797FDC2
:106DF0000396959587959595879590933005809303
:106E00002F058091D7029091D8022091FB013091FB
:106E1000FC01821B930B9093320580933105809186
:106E2000660290916702A0916802B0916902BC016C
:106E3000CD0125E030E040E050E00E94CF8A309361
:106E40003405209333058091F5019091F6019093DC
:106E500036058093350580918F0190919001909334
:106E60003A058093390580911E0190911F019093FE
:106E70003C0580933B0580916C02992790933E05D9
:106E800080933D058091730790917407909340051E
:106E900080933F0580919D069927909342058093AA
:106EA00041058091A5069927909344058093430559
:106EB0008091AD0699279093460580934505809172
:106EC000B506992790934805809347058091D60190
:106ED0009091D701909352058093510580914B0872
:106EE00090914C08909356058093550580914F08DA
:106EF00090915008909358058093570580916202B5
:106F000090916302A0916402B0916502BC01CD0131
:106F100025E030E040E050E00E94CF8A30935A05EF
:106F20002093590580918402909185029093600589
:106F300080935F0580915108992790936405809311
:106F400063058091390390913A039093660580938D
:106F5000650580913703909138039093680580937D
:106F600067058091A703882321F48091A8038823D3
:106F700021F080912805816003C0809128058E7FD3
:106F8000809328051F910F91FF90EF9008951F9314
:106F9000CF93DF93182FEB0180916B02882309F5C3
:106FA000809102018C3010F4299801C0299A115067
:106FB0001F3F81F0D093DD01C093DC018091DC01A3
:106FC0009091DD01892BD1F7CE018C0F9D1F0E947E
:106FD000B619EDCF809102018C3010F4299A01C0CE
:106FE0002998DF91CF911F910895CF93DF938091DE
:106FF00002018D3011F40E94D61D10927A0080910A
:10700000FF019091000290937F0780937E0780910B
:10701000FD019091FE0190936F0780936E07809120
:10702000FB019091FC019093C0078093BF072091D2
:10703000F7013091F801C901880F991F880F991F36
:10704000820F931F820F931F9093BB078093BA0701
:107050002091F9013091FA01C901880F991F880F19
:10706000991F820F931F820F931F9093CB078093DA
:10707000CA078FEC80937A00ADE6B2E0C3EDD5E0AD
:1070800097E08991E82FFF27EE0FFF1FE350F94F9C
:107090000190F081E02DE158FF4F1E161F061CF0F5
:1070A000E0E0F0E005C0EF3FF10514F0EFEFF0E0B5
:1070B0008C91282F3327E217F30714F4815004C072
:1070C0002E173F0714F48F5F8C939150119697FF02
:1070D000D8CF80910F069927AA27BB27BC01CD01E5
:1070E00024EC39E040E050E00E945B8ADC01CB01F7
:1070F0008093870190938801A0938901B0938A01BE
:10710000809110069927AA27BB27BC01CD010E94B8
:107110005B8ADC01CB018093830190938401A0936F
:107120008501B0938601DF91CF910895A0E0B0E092
:10713000ECE9F8E30C94F08A882EC0E0D0E07E0100
:107140006E011092A703469AD093D202C093D10247
:10715000D093D002C093CF02D093CC02C093CB0285
:10716000D093DC02C093DB02D093DA02C093D90241
:10717000D093D802C093D70210926B0110926A018B
:107180001092EF010E94F53784E690E00E94C31947
:107190000E94F5378091DB0580FF10C080911401BB
:1071A00090911501875B934038F480911401909180
:1071B00015018E5E924010F40E94541D0FE18AE08A
:1071C00090E00E94C3198091FB019091FC01C80FCF
:1071D000D91F8091FF0190910002E80EF91E809165
:1071E000FD019091FE01C80ED91E015007FFE7CFA7
:1071F0009701205F3F4F3695279536952795309319
:10720000DC022093DB02C601409696958795969501
:1072100087959093DA028093D9026096F5E0D6952F
:10722000C795FA95E1F7D093D802C093D70290930F
:10723000D6028093D5023093D4022093D3028820C3
:1072400009F441C08091BA079091BB0797FF03C032
:10725000909581959F4F6CE070E00E949A8A9B0107
:107260007093D2026093D1028091CA079091CB07AC
:1072700097FF03C0909581959F4F6CE070E00E944E
:107280009A8A7093D0026093CF028091700590919A
:1072900071059093CC028093CB02B90184E090E019
:1072A0000E946D2E6091CF027091D00286E090E036
:1072B0000E946D2E6091CB027091CC0288E090E02C
:1072C0000E946D2E65C084E090E00E94682E90932D
:1072D000D2028093D10286E090E00E94682E9093C3
:1072E000D0028093CF0288E090E00E94682E9C013B
:1072F0009093CC028093CB028091D1029091D202E4
:107300008150984050F48091CF029091D0028150EA
:10731000984018F421503440D8F185E899E09F93C3
:107320008F9382E995E19F938F93E0918E03F09183
:107330008F0309958091BA079091BB0797FF03C00F
:10734000909581959F4F6CE070E00E949A8A7093AF
:10735000D2026093D1028091CA079091CB0797FF28
:1073600003C0909581959F4F6CE070E00E949A8ACF
:107370007093D0026093CF02809170059091710557
:107380009093CC028093CB020F900F900F900F90B0
:1073900010927F0710927E0710926F0710926E076F
:1073A0001092C0071092BF0784E690E00E94C319B4
:1073B0008091F7019091F8019C01220F331F220F59
:1073C000331F280F391F280F391F3093BB07209315
:1073D000BA078091F9019091FA018C01000F111FF9
:1073E000000F111F080F191F080F191F1093CB074B
:1073F0000093CA078091EA05C82EDD24EE24FF24FD
:10740000442737FD4095542FC701B6010E945B8A7F
:107410004B015C016093C6027093C7028093C8025F
:107420009093C9029801442737FD4095542FC70116
:10743000B6010E945B8ADC01CB018093BE0290936F
:10744000BF02A093C002B093C1028092A2029092A8
:10745000A302A092A402B092A50280939A029093F4
:107460009B02A0939C02B0939D02109296021092F0
:1074700097021092980210929902809116019091B1
:107480001701A0911801B091190190937305809391
:1074900072051092EE011092ED0110928602109288
:1074A0008702109288021092890200918F01109138
:1074B0009001109385020093840284E690E09093FB
:1074C0008C0180938B0182E390E09093DD018093A7
:1074D000DC0180910F069927AA27BB27BC01CD01AB
:1074E00024EC39E040E050E00E945B8ADC01CB01F3
:1074F0008856954CAF4FBF4F80938701909388017A
:10750000A0938901B0938A01809110069927AA2738
:10751000BB27BC01CD010E945B8ADC01CB018856F0
:10752000954CAF4FBF4F8093830190938401A093FC
:107530008501B09386011092480110924701C8015D
:10754000AA2797FDA095BA2F2091430130914401BD
:107550004091450150914601BC01CD010E945B8ADA
:10756000DC01CB018093C6079093C707A093C8079F
:10757000B093C907109281021092800281E080933B
:1075800001010E94DC69809136028460809336029A
:107590008FEF809346081092470880E28093480856
:1075A000CDE6D2E0A3EDB5E007E08D91E82FFF270F
:1075B000EE0FFF1FE350F94F80819181815889932D
:1075C000015007FFF2CF84E680936C028091DA01CC
:1075D000882311F0469A579A8091DB029091DC0241
:1075E00080569940815C9B4228F08091A70381607E
:1075F0008093A7038091D9029091DA028056994036
:10760000815C9B4228F08091A70382608093A7034E
:107610008091D7029091D8028C5291408957954021
:1076200028F08091A70384608093A7038091D10202
:107630009091D2028C529140835C914028F08091CD
:10764000A70388608093A7038091CF029091D00216
:107650008C529140835C914028F08091A703806117
:107660008093A7038091CB029091CC0280509240EE
:107670008355914028F08091A70380628093A703EF
:1076800086E480937E010E942E84ECE0CDB7DEB7C5
:107690000C940C8BA3E1B0E0E0E5FBE30C94EA8AE8
:1076A0008091D7029091D8022091FB013091FC018A
:1076B000821B930B9093C0078093BF0780910502B4
:1076C0009091060297FD07969C0113E0359527954A
:1076D0001A95E1F730937F0720937E07809103028C
:1076E0009091040297FD0796B3E095958795BA951A
:1076F000E1F790936F0780936E0730938A0720938A
:10770000890790938207809381078091BA079091AF
:10771000BB07AC01440F551F480F591F2091F701BB
:107720003091F801C901880F991F880F991F820FA6
:10773000931F820F931F480F591F57FF02C04D5FC1
:107740005F4F55954795559547955093BB07409387
:10775000BA078091CA079091CB07AC01440F551F1F
:10776000480F591F2091F9013091FA01C901880F82
:10777000991F880F991F820F931F820F931F480F25
:10778000591F57FF02C04D5F5F4F5595479555955F
:1077900047955093CB074093CA072091F70130914A
:1077A000F801C901880F991F880F991F820F931F35
:1077B000820F931F9C01442737FD4095542F8091E1
:1077C000B6029091B702A091B802B091B902820FAF
:1077D000931FA41FB51F8093B6029093B702A09386
:1077E000B802B093B9022091F9013091FA01C901B0
:1077F000880F991F880F991F820F931F820F931F65
:107800009C01442737FD4095542F8091B2029091FE
:10781000B302A091B402B091B502820F931FA41FCE
:10782000B51F8093B2029093B302A093B402B093B9
:10783000B50280919307909194072091F7013091C0
:10784000F801820F931F9093940780939307809180
:10785000C2079091C3072091F9013091FA01820F7C
:10786000931F9093C3078093C2078091CD0290919C
:10787000CE0201969093CE028093CD028091700546
:10788000909171052091CB023091CC02821B930B19
:107890009C01442737FD4095542F8091AE02909172
:1078A000AF02A091B002B091B102820F931FA41F4A
:1078B000B51F8093AE029093AF02A093B002B09335
:1078C000B1028FEC80937A001092100120919E02F9
:1078D00030919F024091A0025091A10229873A87DE
:1078E0004B875C8729543B46414050402CF028E4AC
:1078F0003BE641E050E00DC089859A85AB85BC85AB
:10790000885B9449AE4FBF4F4CF428EB34E94EEFFF
:107910005FEF2D833E834F83588708C089859A8502
:10792000AB85BC858D839E83AF83B8872091A602EB
:107930003091A7024091A8025091A9022D873E875D
:107940004F87588B29543B46414050402CF028E447
:107950003BE641E050E00DC08D859E85AF85B8893E
:10796000885B9449AE4FBF4F4CF428EB34E94EEF9F
:107970005FEF29833A834B835C8308C08D859E85A6
:10798000AF85B88989839A83AB83BC83A091BF07F5
:10799000B091C007BB8BAA8BFD01CF01AA2797FD31
:1079A000A095BA2FA0909602B0909702C09098022E
:1079B000D0909902A80EB91ECA1EDB1EA092960294
:1079C000B0929702C0929802D0929902E090C607B6
:1079D000F090C7070091C8071091C907E80EF91E7B
:1079E0000A1F1B1FE092C607F092C7070093C80743
:1079F0001093C907F0915102F98BFF2309F098C148
:107A000080915002882309F093C18091B60786FFC8
:107A10008FC180916E0790916F07AA2797FDA0955F
:107A2000BA2FBC01CD0129813A814B815C810E9432
:107A30005B8A9B01AC0197FF04C02150384F4F4F28
:107A40005F4FBBE05595479537952795BA95D1F788
:107A500080916A01682E772488249924CA01B9018B
:107A6000A40193010E945B8ADC01CB018093E702B1
:107A70009093E802A093E902B093EA02B7FF04C032
:107A80008150904FAF4FBF4F1C012D01ACE055947A
:107A9000479437942794AA95D1F72092E702309221
:107AA000E8024092E9025092EA0280917E079091AA
:107AB0007F07AA2797FDA095BA2FBC01CD012D8184
:107AC0003E814F8158850E945B8A97FF04C06150B8
:107AD000784F8F4F9F4FFBE09595879577956795EA
:107AE000FA95D1F7A40193010E945B8ADC01CB01D6
:107AF0008093EB029093EC02A093ED02B093EE0220
:107B0000B7FF04C08150904FAF4FBF4F9C01AD01F4
:107B1000ECE05595479537952795EA95D1F7209351
:107B2000EB023093EC024093ED025093EE02809111
:107B3000E7029091E8029093660780936507809131
:107B4000EB029091EC0290936A07809369072219E7
:107B50003309440955092093EB023093EC0240931A
:107B6000ED025093EE02E20EF31E041F151FE09289
:107B7000C607F092C7070093C8071093C907809102
:107B800069018823B1F457FF04C02F5F3F4F4F4F67
:107B90005F4F5595479537952795A21AB30AC40AA2
:107BA000D50AA0929602B0929702C0929802D09203
:107BB00099022A893B8979010027F7FC0095102F4B
:107BC0008091EB029091EC02A091ED02B091EE0257
:107BD000E80EF91E0A1F1B1FC801B70129813A814F
:107BE0004B815C810E945B8A9B01AC0197FF04C0C2
:107BF0002150384F4F4F5F4F6BE055954795379564
:107C000027956A95D1F780916B01A82EBB24CC24CF
:107C1000DD24CA01B901A60195010E945B8ADC013D
:107C2000CB018093DF029093E002A093E102B09336
:107C3000E202B7FF04C08150904FAF4FBF4F3C01ED
:107C40004D013CE095948794779467943A95D1F7E9
:107C50006092DF027092E0028092E1029092E20272
:107C6000C801B7012D813E814F8158850E945B8AF2
:107C700097FF04C06150784F8F4F9F4F2BE0959531
:107C80008795779567952A95D1F7A60195010E946A
:107C90005B8ADC01CB018093E3029093E402A09322
:107CA000E502B093E602B7FF04C08150904FAF4F9A
:107CB000BF4FAC01BD018CE0759567955795479511
:107CC0008A95D1F74093E3025093E4026093E50272
:107CD0007093E6022A893B8937FF03C030952195CE
:107CE0003F4F21343105E4F1D401C30197FE07C0B1
:107CF000B095A095909581959F4FAF4FBF4F81381C
:107D00009105A105B10584F4DB01CA0177FF07C025
:107D1000B095A095909581959F4FAF4FBF4F8138FB
:107D20009105A105B105E4F081E08093820218C0BD
:107D300010926A0710926907109266071092650701
:107D40001092E3021092E4021092E5021092E60211
:107D50001092DF021092E0021092E1021092E20211
:107D60008091E3029091E402A091E502B091E602D5
:107D7000BC01CD0124E630E040E050E00E94CF8A13
:107D8000E090DF02F090E002E21AF30AF0927D0741
:107D9000E0927C078091DF029091E002A091E102E5
:107DA000B091E202BC01CD0124E630E040E050E0B9
:107DB0000E94CF8ADA01C9012091E3023091E402E6
:107DC0008C01021B130B10937107009370078091B5
:107DD000430190914401A0914501B0914601BC013D
:107DE000CD0128E631E040E050E00E945B8A20911E
:107DF000C6073091C7074091C8075091C907261799
:107E000037074807590764F0261B370B480B590BF7
:107E10002093C6073093C7074093C8075093C907FC
:107E20002091C6073091C7074091C8075091C907F4
:107E300057FF0CC0260F371F481F591F2093C60736
:107E40003093C7074093C8075093C90760916E07E6
:107E500070916F076E0D7F1D9B01442737FD409584
:107E6000542F80919A0290919B02A0919C02B09114
:107E70009D02820F931FA41FB51F80939A029093B7
:107E80009B02A0939C02B0939D0280915602909118
:107E90005702681B790BCB01AA2797FDA095BA2F33
:107EA00029853A854B855C85820F931FA41FB51FDA
:107EB00080939E0290939F02A093A002B093A10290
:107EC000C0908301D0908401E0908501F0908601FC
:107ED000C816D906EA06FB06C4F488EA91E6A0E0D3
:107EE000B0E08C199D09AE09BF0980939E02909362
:107EF0009F02A093A002B093A10280939A02909354
:107F00009B02A0939C02B0939D0222273327A901D4
:107F10002C193D094E095F0980919E0290919F02A4
:107F2000A091A002B091A10282179307A407B50700
:107F3000B4F4D701C601885A9146A040B04080935E
:107F40009E0290939F02A093A002B093A1028093FF
:107F50009A0290939B02A0939C02B0939D02609121
:107F60007E0770917F07600F711F9B01442737FDCB
:107F70004095542F8091A2029091A302A091A40257
:107F8000B091A502820F931FA41FB51F8093A20278
:107F90009093A302A093A402B093A50280915402EF
:107FA00090915502681B790BCB01AA2797FDA095EC
:107FB000BA2F2D853E854F855889820F931FA41FA8
:107FC000B51F8093A6029093A702A093A802B09336
:107FD000A902E0908701F090880100918901109139
:107FE0008A01E816F9060A071B07C4F488EA91E635
:107FF000A0E0B0E08E199F09A00BB10B8093A60200
:108000009093A702A093A802B093A9028093A20222
:108010009093A302A093A402B093A5022227332732
:10802000A9012E193F09400B510B8091A602909196
:10803000A702A091A802B091A90282179307A407F2
:10804000B507B4F4D801C701885A9146A040B040A2
:108050008093A6029093A702A093A802B093A902CE
:108060008093A2029093A302A093A402B093A502CE
:108070008091960290919702A0919802B0919902F6
:108080008093AA029093AB02A093AC02B093AD028E
:108090008091A6029091A702A091A802B091A90296
:1080A0008093C6029093C702A093C802B093C902FE
:1080B00080919E0290919F02A091A002B091A10296
:1080C0008093BE029093BF02A093C002B093C102FE
:1080D0008091A2029091A302A091A402B091A50266
:1080E0008093C2029093C302A093C402B093C502CE
:1080F00080919A0290919B02A0919C02B0919D0266
:108100008093BA029093BB02A093BC02B093BD02CD
:1081100080911C0190911D0197FD079603E09595B4
:1081200087950A95E1F790937F0780937E0780916A
:108130001A0190911B0197FD079613E0959587957D
:108140001A95E1F790936F0780936E078091FF0176
:10815000909100020F9734F488E19CEF90937F0791
:1081600080937E078091FF0190910002079734F47D
:1081700080E398EF90937F0780937E072091020120
:108180002A30A9F48091FF0190910002835F93400F
:1081900034F088EE93E090937F0780937E07809180
:1081A000FF01909100028A5F9340DCF014C080913F
:1081B000FF0190910002815D974034F088EE93E0DA
:1081C00090937F0780937E078091FF01909100023A
:1081D000805E974034F080ED97E090937F07809326
:1081E0007E078091FD019091FE010F9734F488E1A4
:1081F0009CEF90936F0780936E078091FD019091A3
:10820000FE01079734F480E398EF90936F07809313
:108210006E072A30A9F48091FD019091FE01835FE1
:10822000934034F088EE93E090936F0780936E074D
:108230008091FD019091FE018A5F9340DCF014C0B3
:108240008091FD019091FE01815D974034F088EEB0
:1082500093E090936F0780936E078091FD0190915A
:10826000FE01805E974034F080ED97E090936F07B9
:1082700080936E0760917501662309F4AFC0409149
:108280001C0150911D018091EF029091F002481B5A
:10829000590B5093F6024093F50220911C01309146
:1082A0001D01280F391F37FF02C02F5F3F4F359543
:1082B00027953093F0022093EF02413851051CF0CE
:1082C00080E890E005C040585F4F34F480E89FEFAD
:1082D0009093F6028093F50240911A0150911B0190
:1082E0008091F1029091F202481B590B5093F402D5
:1082F0004093F30220911A0130911B01280F391F7E
:1083000037FF02C02F5F3F4F359527953093F2021C
:108310002093F102413851051CF080E890E005C03F
:1083200040585F4F34F480E89FEF9093F4028093BD
:10833000F302462F55278091F5029091F602849F13
:10834000B001859F700D949F700D11249B0177FFE4
:1083500002C0215F3F4FF4E035952795FA95E1F78C
:1083600080917E0790917F07820F931F90937F07E4
:1083700080937E078091F3029091F402849FD00154
:10838000859FB00D949FB00D1124AD019D01B7FFE5
:1083900002C0215F3F4FE4E035952795EA95E1F76C
:1083A00080916E0790916F07820F931F90936F07D4
:1083B00080936E0780911C0190911D01860F971F7D
:1083C00090931D0180931C0180911A0190911B01D3
:1083D000840F951F90931B0180931A0100918107D0
:1083E000109182078091650790916607101611061B
:1083F0005CF59C0197FF04C022273327281B390B0B
:10840000C901AA2797FDA095BA2F209169013327AA
:1084100044275527BC01CD010E945B8A9B01AC011A
:1084200097FF04C0215C3F4F4F4F5F4F76E055955B
:108430004795379527957A95D1F780917C0790914C
:108440007D07820F931F27C097FF03C090958195EA
:108450009F4FAA2797FDA095BA2F20916901332736
:1084600044275527BC01CD010E945B8A9B01AC01CA
:1084700097FF04C0215C3F4F4F4F5F4F66E055951B
:108480004795379527956A95D1F780917C0790910C
:108490007D07821B930B90937D0780937C07E09070
:1084A0008907F0908A078091690790916A071E14E6
:1084B0001F045CF59C0197FF04C022273327281B6B
:1084C000390BC901AA2797FDA095BA2F2091690100
:1084D000332744275527BC01CD010E945B8A9B01AD
:1084E000AC0197FF04C0215C3F4F4F4F5F4F96E0B8
:1084F00055954795379527959A95D1F780917007AF
:1085000090917107820F931F27C097FF03C090952A
:1085100081959F4FAA2797FDA095BA2F20916901B9
:10852000332744275527BC01CD010E945B8A9B015C
:10853000AC0197FF04C0215C3F4F4F4F5F4F86E077
:1085400055954795379527958A95D1F7809170076E
:1085500090917107821B930B909371078093700722
:108560008091B60787FF44C0B989BB2309F040C09A
:10857000809150028823E1F5E1E0EE16E1E0FE068D
:108580004CF080917E0790917F078E0D9F1D80504B
:1085900091400DC0F0E0EF16FFEFFF0664F480910C
:1085A0007E0790917F078E0D9F1D80509F4F909367
:1085B0007F0780937E0721E0013012074CF0809105
:1085C0006E0790916F07800F911F805091400CC0F3
:1085D0003FEF0030130764F480916E0790916F07AE
:1085E000800F911F80509F4F90936F0780936E076D
:1085F000E2E1CD5E0C94068B80916B02882301F53D
:10860000809136028C7F80933602ACEAB3E0ECE9CD
:10861000F6E09BE08091BB01882309F48C938D9157
:10862000818312829150389697FFF4CF8091BB01DD
:10863000882359F08091BB0181508093BB0105C014
:1086400080913602816080933602809126028823D1
:1086500019F01092260208958093280280932A022E
:10866000809124028E7F8093240285EA8093BC004F
:108670000895CF93DF93ADE6B2E0C3EDD5E057E0C8
:108680009991E92FFF27EE0FFF1FE350F94F01905B
:10869000F081E02DE158FF4FEF3FF10521F01CF094
:1086A000EFEFF0E004C0F7FF02C0E0E0F0E0993146
:1086B00011F4EC931BC04C91242F3327E217F307DE
:1086C000A9F0CF01821B930B97FD03969595879593
:1086D00095958795242F280F2C93822F9927E8179B
:1086E000F90714F4215001C02F5F2C9351501196BB
:1086F00057FFC6CF8091DD05883F38F0EFEFF0E0FF
:10870000E81BF109E359FD4F808180937B01809143
:108710007B01882329F0843618F084E680937B015E
:108720008091DF05883F38F0EFEFF0E0E81BF109BA
:10873000E359FD4F808180937901809179018823ED
:1087400029F0843618F084E6809379018091EC0555
:10875000883F38F0EFEFF0E0E81BF109E359FD4FF7
:10876000808180937401809174018B3010F48AE0D1
:1087700002C08F3F11F48093740180911906883FE5
:1087800038F0EFEFF0E0E81BF109E359FD4F80818D
:108790008093950780919507863010F485E002C09C
:1087A0008F3F11F48093950780911B06883F38F026
:1087B000EFEFF0E0E81BF109E359FD4F8081809372
:1087C000BD078091BD07863010F485E002C08F3F61
:1087D00011F48093BD0780910606883F38F0EFEFD3
:1087E000F0E0E81BF109E359FD4F80818093920787
:1087F00080910706883F38F0EFEFF0E0E81BF109C1
:10880000E359FD4F808180936B0780910806883F74
:1088100038F0EFEFF0E0E81BF109E359FD4F8081FC
:1088200080939B078091DE05883F38F0EFEFF0E002
:10883000E81BF109E359FD4F808180937A01809113
:10884000E105883F38F0EFEFF0E0E81BF109E3596C
:10885000FD4F8081809378018091E305883F38F057
:10886000EFEFF0E0E81BF109E359FD4F80818093C1
:1088700076018091EB05883F38F0EFEFF0E0E81BE0
:10888000F109E359FD4F8081809377018091ED05D7
:10889000883F38F0EFEFF0E0E81BF109E359FD4FB6
:1088A0008081809373018091EE05883F38F0EFEF6F
:1088B000F0E0E81BF109E359FD4F808180937501D9
:1088C0008091EF05883F38F0EFEFF0E0E81BF10909
:1088D000E359FD4F8081809372018091F005883FBC
:1088E00038F0EFEFF0E0E81BF109E359FD4F80812C
:1088F000809371018091F605883F38F0EFEFF0E04A
:10890000E81BF109E359FD4F808180936F0180914D
:10891000F705883F38F0EFEFF0E0E81BF109E35985
:10892000FD4F808180934B028091F805883F38F09D
:10893000EFEFF0E0E81BF109E359FD4F80818093F0
:108940004A028091F905883F38F0EFEFF0E0E81B2C
:10895000F109E359FD4F8081809349028091FA0526
:10896000883F38F0EFEFF0E0E81BF109E359FD4FE5
:1089700080818093480280911406883F38F0EFEFA1
:10898000F0E0E81BF109E359FD4F80818093470235
:1089900080911506883F38F0EFEFF0E0E81BF10911
:1089A000E359FD4F80818093460280911606883FEF
:1089B00038F0EFEFF0E0E81BF109E359FD4F80815B
:1089C0008093450280911706883F38F0EFEFF0E082
:1089D000E81BF109E359FD4F8081809344028091A7
:1089E000FB05883F38F0EFEFF0E0E81BF109E359B1
:1089F000FD4F808180936E018091FF05883F38F0A4
:108A0000EFEFF0E0E81BF109E359FD4F808180931F
:108A10006D0180910906883F38F0EFEFF0E0E81B28
:108A2000F109E359FD4F808180936C0180910C0620
:108A3000883F38F0EFEFF0E0E81BF109E359FD4F14
:108A4000808180936B0180910D06883F38F0EFEFB5
:108A5000F0E0E81BF109E359FD4F808180936A0142
:108A600080910E06883F38F0EFEFF0E0E81BF10947
:108A7000E359FD4F80818093690180913506883FDD
:108A800038F0EFEFF0E0E81BF109E359FD4F80818A
:108A900080937A078091DB058093B6078091380632
:108AA00080939A0780911306883F38F0EFEFF0E04B
:108AB000E81BF109E359FD4F8081809368018091A3
:108AC0002E06883F38F0EFEFF0E0E81BF109E3599C
:108AD000FD4F80818093CD0780916F01282F332730
:108AE0002F5F3F4F8CE398E2B9010E949A8A7093FE
:108AF0007D0160937C018091E9058093BE078091A0
:108B0000E80580938307909130069333C8F181E0A4
:108B100080934302983F58F0EFEFF0E0E91BF10932
:108B2000E359FD4F8081823310F41092430280910B
:108B30007E0120914302821799F0833070F4222342
:108B400019F08CED95E002C088EC90E09093DD0187
:108B50008093DC0120937E0103C0815080937E01CD
:108B600080910D0890910E0897FF0FC080914302ED
:108B7000882359F08091A70380688093A70305C0DC
:108B8000109243028AE080937E0180910D089091BB
:108B90000E0897FF1DC080916B028823C9F0809159
:108BA00043028823A9F080910801909109018F5F09
:108BB0009F4F71F488E99AE39093DD018093DC0183
:108BC00080E094EA90930901809308011092430297
:108BD00080914302882369F08091350281608093FF
:108BE000350280916B01823D48F4825E80936B0177
:108BF00005C0809135028E7F80933502DF91CF9141
:108C00000895A7E1B0E0E7E0F6E40C94EA8A0E9458
:108C10004A3BE0907602F0907702FA82E9828091F6
:108C2000830799270A96E816F90614F49A8389832C
:108C300080916C02843608F066C08091350282FD16
:108C400062C080910B0390910C03009731F0019763
:108C500090930C0380930B030BC010926B029093C4
:108C6000380280933702809136028D7E80933602DF
:108C7000809102018A3011F0843110F0289A01C0ED
:108C800028988091370290913802895E9340C0F114
:108C90008091F305282F33273A8329838091360268
:108CA0008061809336028091CF05A82FBB27AA0F41
:108CB000BB1FFD01EF5CF84F118210828091D0053F
:108CC000282F3327220F331FC9018F5C984FFC01D7
:108CD00011821082A350B94F11961C921E922350FC
:108CE000394FD90111961C921E928091D205E82F1E
:108CF000FF27EE0FFF1FE350F94F11821082A9C228
:108D000010926B02A6C280916C028D3808F4A1C249
:108D1000809136028F7E809336029091F40582E333
:108D2000989FC001112490930C0380930B03E98159
:108D3000FA81B9978CF080916B02882369F0809159
:108D4000370290913802FFEF8F3F9F0729F001967D
:108D500090933802809337028091370290913802C5
:108D60008F3F910509F008F510928E0210928F0244
:108D7000109290021092910210928A0210928B022D
:108D800010928C0210928D021092F7021092F8024B
:108D90001092F9021092FA02109296021092970223
:108DA000109298021092990205C08091360282605A
:108DB000809336028091D105E82FFF27EE0FFF1F29
:108DC000E350F94F80819181813591050CF435C1D3
:108DD00020916B02222309F030C18091D205E82F47
:108DE000FF27EE0FFF1FE350F94F808191818C34F4
:108DF00091050CF4FFC080910D038F5F80930D03EC
:108E0000893C08F41AC120930D0310923802109285
:108E100037023091CF05E32FFF27EE0FFF1FE350FE
:108E2000F94F8081918187349105B4F48091D00508
:108E3000E82FFF27EE0FFF1FE350F94F808191814C
:108E40000190F081E02DF7FF03C0F095E195FF4F11
:108E5000E734F1050CF478C041E02091D005A22F51
:108E6000BB27AA0FBB1FA350B94F8D919C9111979F
:108E70008734910544F0E32FFF27EE0FFF1FE350E7
:108E8000F94F808191818D919C918734910574F087
:108E90008091CF05E82FFF27EE0FFF1FE350F94F1A
:108EA00080819181873491050CF042E0E22FFF2709
:108EB000EE0FFF1FE350F94F8081918186349105B9
:108EC00074F48091CF05E82FFF27EE0FFF1FE350CA
:108ED000F94F80819181873491050CF043E0E22FB6
:108EE000FF27EE0FFF1FE350F94F808191818A5BCE
:108EF0009F4F74F48091CF05E82FFF27EE0FFF1FDF
:108F0000E350F94F80819181873491050CF044E062
:108F1000E22FFF27EE0FFF1FE350F94F8081918171
:108F20008A5B9F4F74F48091CF05E82FFF27EE0FE7
:108F3000FF1FE350F94F80819181863491050CF435
:108F400045E0842F0E94C72E8091D005E82FFF278F
:108F5000EE0FFF1FE350F94F808191810190F08166
:108F6000E02DF7FF03C0F095E195FF4F7E97BCF42D
:108F70008091CF05E82FFF27EE0FFF1FE350F94F39
:108F8000808191818A5B9F4F54F481E08093C2037A
:108F900088EE93E09093DD018093DC014EC00E9447
:108FA000C52F0E94722E80E00E94E7098091F5058E
:108FB0000E94CF858091B60780FF10C08091140178
:108FC00090911501875B934038F480911401909142
:108FD00015018E5E924010F40E94541D1092DA0129
:108FE00080E00E94963881E0809310038093DA013C
:108FF000579A1AC080819181855B9F4FE4F48091DC
:109000000D038F5F80930D03893CB8F020936B02B2
:1090100020930D03109238021092370281E00E94D3
:10902000963881E0809310030E94C52F68E770E0B6
:109030000E94C73702C020930D038091D105E82F0D
:10904000FF27EE0FFF1FE350F94F808191818B5A6C
:109050009F4F0CF0FEC030916B02E091D20533239C
:1090600009F0CCC0FF27EE0FFF1FE350F94F8081BE
:109070009181855B9F4F0CF0BEC020913106E22F9D
:10908000FF27EE0FFF1FE350F94F80819181855B31
:109090009F4F1CF0222309F0AEC080910E038F5F1A
:1090A00080930E03893C08F4D4C030930E03809162
:1090B000A703882309F098C080911003882309F43E
:1090C00093C080914603882309F08EC081E090E030
:1090D000909338028093370281E080936B02109264
:1090E000F7021092F8021092F9021092FA0210920E
:1090F0009602109297021092980210929902109282
:109100009202109293021092940210929502809112
:10911000EA05E82EFF24002711278091BA079091D5
:10912000BB079C01442737FD4095542FC801B70168
:109130000E945B8ADC01CB018093A6029093A70278
:10914000A093A802B093A9028091CA079091CB077F
:109150009C01442737FD4095542FC801B7010E9458
:109160005B8ADC01CB0180939E0290939F02A093C7
:10917000A002B093A1028091C6029091C702A09173
:10918000C802B091C9028093A2029093A302A09357
:10919000A402B093A5028091BE029091BF02A0915B
:1091A000C002B091C10280939A0290939B02A09357
:1091B0009C02B0939D0210928E0210928F02109228
:1091C00090021092910210928A0210928B021092D9
:1091D0008C0210928D028091360288608093360254
:1091E00084E68093110335C08CED95E09093DD010A
:1091F0008093DC012EC010920E032BC0FF27EE0FD0
:10920000FF1FE350F94F808191818C349105FCF070
:1092100020913106E22FFF27EE0FFF1FE350F94F99
:1092200080819181855B9F4F14F0222381F480918E
:109230000F038F5F80930F03893C58F010926B02ED
:1092400010920F03109238021092370202C010924F
:109250000F03809141018150809341018091410130
:109260008F3F21F08091360284FFA9C30E943943C9
:10927000B090E50580911A0390911B039C01220F89
:10928000331F280F391FC090CF05AC2DBB27AA0F65
:10929000BB1FFD01E350F94F4B2D55278081918174
:1092A000849FF001859FF00D949FF00D11242E0FE7
:1092B0003F1F37FF02C02D5F3F4FB901759567957E
:1092C00075956795AF5CB84F8091E605082F11271B
:1092D0008D919C91809F7001819FF00C909FF00C6C
:1092E00011246E0D7F1D70931B0360931A038091F0
:1092F0001C0390911D039C01220F331F280F391F5F
:10930000D090D005AD2DBB27AA0FBB1FFD01E350A8
:10931000F94F80819181849FF001859FF00D949F8A
:10932000F00D11242E0F3F1F37FF02C02D5F3F4F5E
:10933000A9015595479555954795AF5CB84F8D91C7
:109340009C91809F7001819FF00C909FF00C1124E4
:109350004E0D5F1D50931D0340931C0380914302EB
:10936000882309F448C0CB0177FD0396DC01B5954D
:10937000A795B595A795CA0157FD0396FC01F595EC
:10938000E795F595E79580919D01682F772767FD13
:1093900070956A9F90016B9F300D7A9F300D11245C
:1093A00080914803482F552747FD50954E9FC00197
:1093B0004F9F900D5E9F900D1124280F391F37FF8E
:1093C00002C0295F3F4F93E0359527959A95E1F7C5
:1093D00030937D0220937C026E9F90016F9F300D31
:1093E0007E9F300D11244A9FC0014B9F900D5A9FC4
:1093F000900D11243FC080912F06E82FFF27E75BD7
:10940000FE4F868180939D01908190934803A82F01
:10941000BB27A7FDB095A69F9001A79F300DB69FD3
:10942000300D1124E92FFF27E7FDF095E49FC001DF
:10943000E59F900DF49F900D1124280F391F37FFE1
:1094400002C0295F3F4F83E0359527958A95E1F764
:1094500030937D0220937C02A49F9001A59F300D44
:10946000B49F300D1124E69FC001E79F900DF69F39
:10947000900D1124281B390B37FF02C0295F3F4F85
:1094800003E0359527950A95E1F730937B02209309
:109490007A028091D205E82FFF27EE0FFF1FE350DD
:1094A000F94F80819181909581959F4F909379029A
:1094B000809378028530910514F0049705C00FEF72
:1094C0008C3F900734F4049690937902809378024D
:1094D00004C010927902109278028091360388239A
:1094E00009F43EC0282F332780917C0290917D02A1
:1094F00097FD079613E0959587951A95E1F7289FB4
:10950000A001299F500D389F500D1124CA0157FD0D
:109510000F96B4E095958795BA95E1F790937D0203
:1095200080937C0280917A0290917B0297FD07964E
:10953000A3E095958795AA95E1F7289FB001299F0B
:10954000700D389F700D1124CB0177FD0F96F4E05C
:1095500095958795FA95E1F790937B0280937A022F
:1095600080907C0290907D028091390390913A0323
:10957000881A990A90927D0280927C0200917A0268
:1095800010917B028091370390913803081B190BCF
:1095900010937B0200937A028091D105E82FFF2778
:1095A000EE0FFF1FE350F94FE080F1808FE790E06E
:1095B000E80EF91EF0927702E09276028091740133
:1095C0009927AA2797FDA095BA2FBC01CD010E942B
:1095D000CF89DC01CB0120E030E040E251E4BC0166
:1095E000CD010E943D89DC01CB01BC01CD010E946F
:1095F000A189DC01CB018093C40780917301809322
:109600009C07809172019927AA2797FDA095BA2FF0
:10961000BC01CD010E94CF89DC01CB0120E030E00C
:1096200040E251E4BC01CD010E943D89DC01CB0147
:10963000BC01CD010E94A189DC01CB01809375079B
:109640008091710180938B078091CE0380FF59C078
:109650008091CD07813808F454C08091C7039927C1
:1096600087FD90952B2D3327829FD001839FB00DCE
:10967000929FB00D11248A0E9B1E90927D028092C3
:109680007C028091C803992787FD9095829FF00105
:10969000839FF00D929FF00D11240E0F1F1F10934A
:1096A0007B0200937A028091C903282F332727FD7C
:1096B00030958091780290917902820F931F909358
:1096C0007902809378028091CB03282F332727FDDE
:1096D00030958091E0059927289F8001299F100DE2
:1096E000389F100D11241093480100934701809179
:1096F000CA0399278E159F0524F4909377028093CF
:109700007602809176029091770297FF04C01092C2
:109710007702109276028091B60782FF02C0109203
:109720009C0740917C0250917D02CA0157FD03962F
:109730009C01359527953595279537FF03C03095C2
:1097400021953F4F80913B0290913C0282179307F5
:10975000B4F4CA0157FF03C0909581959F4F97FDC0
:109760000396959587959595879590933C02809360
:109770003B028536910544F084E690E001C00197F4
:1097800090933C0280933B0240917A0250917B027D
:10979000CA0157FD03969C01359527953595279568
:1097A00037FF03C0309521953F4F8091390290914A
:1097B0003A0282179307B4F4CA0157FF03C0909589
:1097C00081959F4F97FD03969595879595958795DC
:1097D00090933A02809339028536910544F084E6ED
:1097E00090E001C0019790933A02809339028091F2
:1097F000360284FF08C010923C0210923B02109285
:109800003A0210923902ED2DFF27EE0FFF1FE350B1
:10981000F94F40910A06242F332780819181281720
:10982000390744F48091360682FF04C081E08093BA
:109830004F0213C0ED2DFF27EE0FFF1FE350F94F2E
:10984000842F992720910B06821B91092081318159
:109850002817390714F410924F024091D005E42FD5
:10986000FF27EE0FFF1FE350F94F50910A06852F97
:10987000992722273327281B390B80819181821752
:10988000930744F48091360683FF04C081E08093FF
:109890004E0216C080914E02882391F0E42FFF27DC
:1098A000EE0FFF1FE350F94F80910B069927851BA0
:1098B0009109208131818217930714F410924E028E
:1098C000EC2DFF27EE0FFF1FE350F94F40910A06E2
:1098D000242F3327808191812817390744F4809100
:1098E000360680FF04C081E080934C0217C080914F
:1098F0004C02882399F0EC2DFF27EE0FFF1FE35059
:10990000F94F842F992720910B06821B9109208102
:1099100031812817390714F410924C024091CF0579
:10992000E42FFF27EE0FFF1FE350F94F50910A0677
:10993000852F992722273327281B390B8081918176
:109940008217930744F48091360681FF04C081E0BA
:1099500080934D0216C080914D02882391F0E42F30
:10996000FF27EE0FFF1FE350F94F80910B06992759
:10997000851B9109208131818217930714F410927D
:109980004D0280914F02882319F480914E0281117B
:1099900081E08093500280914C02882321F48091D1
:1099A0004D02882351F081E08093510210925002C1
:1099B00010924F0210924E0202C080935102809189
:1099C0005002882321F480915102882369F080910C
:1099D0000906992729813A818217930714F49A83FB
:1099E000898381E0809382028091350299279C01CE
:1099F0002470307082FF2DC08091390390913A031A
:109A0000909581959F4F90937D0280937C028091E9
:109A1000370390913803909581959F4F90937B02E7
:109A200080937A02809181019091820190937702D4
:109A3000809376028091B6078B778B668093B6070A
:109A400080919A078C7B80939A0788EC80937A01A7
:109A50001EC08091360284FF1AC030937902209391
:109A6000780230937D0220937C0230937B02209316
:109A70007A029AE59093C40788E780939C079093B5
:109A8000750780938B0710925002109251028091BB
:109A90008E0790918F07A0919007B0919107209128
:109AA000C6023091C7024091C8025091C902820F8C
:109AB000931FA41FB51F80938E0790938F07A093C9
:109AC0009007B09391078091960790919707A09186
:109AD0009807B0919907E090BE02F090BF02009104
:109AE000C0021091C102EB82FC820D831E838E0D99
:109AF0009F1DA01FB11F8093960790939707A09377
:109B00009807B09399078091850790918607A09157
:109B10008707B0918807E090C202F090C3020091DD
:109B2000C4021091C502EF82F88609871A878E0D4C
:109B30009F1DA01FB11F8093850790938607A09358
:109B40008707B09388078091760790917707A09157
:109B50007807B0917907E090BA02F090BB020091CB
:109B6000BC021091BD02EB86FC860D871E878E0D10
:109B70009F1DA01FB11F8093760790937707A09336
:109B80007807B0937907F0905102FF86FF2029F4FF
:109B900080915002882309F460C01092B60210929E
:109BA000B7021092B8021092B9021092B20210924B
:109BB000B3021092B4021092B50210928E07109266
:109BC0008F071092900710929107109296071092AB
:109BD0009707109298071092990710928507109294
:109BE00086071092870710928807109276071092C6
:109BF000770710927807109279078091A6029091CA
:109C0000A702A091A802B091A9028093A20290930A
:109C1000A302A093A402B093A50280919E0290910A
:109C20009F02A091A002B091A10280939A0290930A
:109C30009B02A0939C02B0939D021092EC011092A3
:109C4000EB0110925502109254021092570210929A
:109C500056020F85002309F0F8C180915002882335
:109C600009F0F3C180917005909171058150924087
:109C70002CF480916B02882309F4E7C19090460888
:109C8000A090EA052090BA073090BB074090CA0721
:109C90005090CB0719140CF0E3C0BB24CC24DD2476
:109CA000CA01B901A60195010E94CF8A79018A01F2
:109CB00080910F0890911008281A390AC101AA272B
:109CC00097FDA095BA2FE81AF90A0A0B1B0B6B81B6
:109CD0007C818D819E81A60195010E94CF8A5901C8
:109CE0006A018091110890911208481A590AC2011C
:109CF000AA2797FDA095BA2FA81AB90ACA0ADB0AA3
:109D0000292C332427FC3094432C532CC801B70151
:109D1000A20191010E945B8A97FF04C061507E4FAF
:109D20008F4F9F4F3B014C0109E0959487947794A6
:109D300067940A95D1F7C601B501A20191010E946D
:109D40005B8A97FF04C061507E4F8F4F9F4F5B012E
:109D50006C0119E0D594C794B794A7941A95D1F7DC
:109D600080913B0290913C02813491053CF48091BA
:109D7000390290913A0281349105D4F0D401C301A3
:109D800097FE03C00196A11DB11D3C014D019594A4
:109D9000879477946794D601C501D7FE03C00196D6
:109DA000A11DB11D5C016D01D594C794B794A79412
:109DB0008091D205E82FFF27EE0FFF1FE350F94FE8
:109DC000808191810190F081E02DF7FF03C0F09533
:109DD000E195FF4F7A97A4F0C401B30123E030E08E
:109DE00040E050E00E94CF8A39014A01C601B50126
:109DF00023E030E040E050E00E94CF8A59016A0140
:109E000080914808282F332727FD3095432F532F63
:109E1000261537054805590514F439014A019927D3
:109E200087FD9095909581959F4FAA2797FDA095C6
:109E3000BA2F681679068A069B0614F43C014D0178
:109E40002A153B054C055D0514F459016A01A81655
:109E5000B906CA06DB060CF0D0C05C016D01CDC0AE
:109E6000EA2CFF2400271127CA01B901A801970194
:109E70000E94CF8A39014A01C101AA2797FDA09506
:109E8000BA2F681A790A8A0A9B0A6B817C818D81B4
:109E90009E81A80197010E94CF8A59016A01C201DF
:109EA000AA2797FDA095BA2FA81AB90ACA0ADB0AF1
:109EB000D401C30197FE03C00F96A11DB11D3C0143
:109EC0004D01F4E09594879477946794FA95D1F7CF
:109ED000D601C501D7FE03C00F96A11DB11D5C01BF
:109EE0006D01E4E0D594C794B794A794EA95D1F7AF
:109EF00080913B0290913C02813491053CF4809129
:109F0000390290913A0281349105A4F0C401B30161
:109F100023E030E040E050E00E94CF8A39014A015E
:109F2000C601B50123E030E040E050E00E94CF8A56
:109F300059016A018091D205E82FFF27EE0FFF1F1C
:109F4000E350F94F808191810190F081E02DF7FF7E
:109F500003C0F095E195FF4F7A97A4F0C401B301D7
:109F600023E030E040E050E00E94CF8A39014A010E
:109F7000C601B50123E030E040E050E00E94CF8A06
:109F800059016A0189E180938D0121E26216710411
:109F9000810491042CF070E2672E712C812C912C9D
:109FA00030EE63163FEF73063FEF83063FEF9306F5
:109FB00044F460EE662E6FEF762E6FEF862E6FEF15
:109FC000962E41E2A416B104C104D1042CF050E253
:109FD000A52EB12CC12CD12C50EEA5165FEFB506E5
:109FE0005FEFC5065FEFD50644F440EEA42E4FEFB9
:109FF000B42E4FEFC42E4FEFD42E8091A602909135
:10A00000A702A091A802B091A90286199709A809F0
:10A01000B9098093A6029093A702A093A802B093D7
:10A02000A90280919E0290919F02A091A002B091FE
:10A03000A1028A199B09AC09BD0980939E029093E5
:10A040009F02A093A002B093A1028091EB01909196
:10A05000EC018F3F910509F008F4C4C56F856623B4
:10A0600009F04EC580915002882309F049C58091BE
:10A070008202882309F044C570911206788B7723F9
:10A0800009F43EC580918E0790918F07A0919007AB
:10A09000B0919107B7FF04C081509F4FAF4FBF4FA2
:10A0A000E92EFA2E0B2F112707FD1A95E0928E0745
:10A0B000F0928F0700939007109391078091960775
:10A0C00090919707A0919807B0919907B7FF04C0A6
:10A0D00081509F4FAF4FBF4F892F9A2FAB2FBB2778
:10A0E000A7FDBA95898B9A8BAB8BBC8B8093960717
:10A0F00090939707A0939807B09399078091EA05EA
:10A10000A82EBB24CC24DD242091B6023091B702C6
:10A110004091B8025091B902C601B5010E945B8A14
:10A1200097FF04C061507F4F8F4F9F4F672E782E4F
:10A13000892E992487FC9A946092B6027092B70295
:10A140008092B8029092B9022091B2023091B3028B
:10A150004091B4025091B502C601B5010E945B8ADC
:10A1600097FF04C061507F4F8F4F9F4F272E382E8F
:10A17000492E552447FC5A942092B2023092B302E1
:10A180004092B4025092B5028091AE029091AF021B
:10A19000A091B002B091B102B7FF04C081509F4FAF
:10A1A000AF4FBF4F892F9A2FAB2FBB27A7FDBA9573
:10A1B0008093AE029093AF02A093B002B093B1022D
:10A1C000D801C70186199709A809B9098093030323
:10A1D00090930403A0930503B09306032091110606
:10A1E000E22EFF2400271127BC01CD01A801970111
:10A1F0000E94CF8A59016A012093120330931303FE
:10A20000409314035093150389899A89AB89BC89BB
:10A2100082199309A409B509809307039093080351
:10A22000A0930903B0930A03BC01CD01A8019701D3
:10A230000E94CF8A2093160330931703409318038C
:10A2400050931903D601C501D7FE04C081509F4F1A
:10A25000AF4FBF4F892F9A2FAB2FBB27A7FDBA95C2
:10A26000909355028093540257FF04C021503F4FF2
:10A270004F4F5F4FBB2757FDBA95A52F942F832FC4
:10A28000909357028093560280913B0290913C023A
:10A2900081349105DCF48091390290913A02813445
:10A2A0009105A4F48091D205E82FFF27EE0FFF1F40
:10A2B000E350F94F808191810190F081E02DF7FF0B
:10A2C00003C0F095E195FF4F7A97E4F0809146083E
:10A2D0008F3FC1F4809154029091550297FD0196F1
:10A2E00095958795909355028093540280915602DC
:10A2F0009091570297FD01969595879590935702F7
:10A30000809356028091850790918607A0918707D8
:10A31000B0918807B7FF04C081509F4FAF4FBF4F28
:10A32000892F9A2FAB2FBB27A7FDBA95809385075E
:10A3300090938607A0938707B0938807809176074C
:10A3400090917707A0917807B0917907B7FF04C083
:10A3500081509F4FAF4FBF4F892F9A2FAB2FBB27F5
:10A36000A7FDBA958093760790937707A093780717
:10A37000B09379078091C6029091C702A091C8025C
:10A38000B091C9022F81388549855A85281B390B20
:10A390004A0B5B0B2093FB023093FC024093FD02BF
:10A3A0005093FE028091BE029091BF02A091C00224
:10A3B000B091C102EB84FC840D851E85E81AF90A70
:10A3C0000A0B1B0BE092FF02F092000300930103C3
:10A3D0001093020320930303309304034093050377
:10A3E00050930603E0920703F092080300930903D9
:10A3F00010930A038091A2029091A302A091A4025B
:10A40000B091A502821B930BA40BB50B8093A20203
:10A410009093A302A093A402B093A50280919A0204
:10A4200090919B02A0919C02B0919D028E199F0970
:10A43000A00BB10B80939A0290939B02A0939C0275
:10A44000B0939D0288898823E1F0209180023091A9
:10A450008102213831054CF08091D7029091D802C9
:10A4600001969093D8028093D70220583F4F4CF426
:10A470008091D7029091D80201979093D80280934F
:10A48000D702109281021092800281E090E09093B6
:10A490001F0380931E03E0900303F09004030091D8
:10A4A000050310910603D801C70117FF07C08827CD
:10A4B0009927DC018E199F09A00BB10B81509240A6
:10A4C000A040B04034F084E090E090931F0380936C
:10A4D0001E038091240390912503A0912603B0913F
:10A4E000270320918E0730918F074091900750915C
:10A4F0009107821B930BA40BB50B815E914BAF4F61
:10A50000BF4F8F539C49A040B04028F0809147082E
:10A5100089310CF4FFC021E0E21620E1F20620E0D0
:10A52000020720E012070CF473C0809120038823F7
:10A5300009F46AC0D801C70117FF07C08827992707
:10A54000DC018E199F09A00BB10B9C01AD01B7FF77
:10A5500004C021503E4F4F4F5F4FF9E0559547954E
:10A5600037952795FA95D1F780911E0390911F0397
:10A57000820F931F90931F0380931E03D801C7017E
:10A5800017FF03C00796A11DB11DE3E0B595A79580
:10A5900097958795EA95D1F78093120390931303CB
:10A5A000A0931403B093150389589341A040B04081
:10A5B00064F088E893E1A0E0B0E080931203909308
:10A5C0001303A0931403B093150320911203309149
:10A5D0001303409114035091150357FF04C02150F9
:10A5E0003F4F4F4F5F4F232F342F452F552747FDA8
:10A5F0005A958091540290915502820F931F909327
:10A6000055028093540206C081E08093200302C06B
:10A610001092200340E0E41640EFF4064FEF0407E9
:10A620004FEF14070CF073C080912103882309F4C5
:10A630006AC0D801C70117FF07C088279927DC0126
:10A640008E199F09A00BB10B9C01AD01B7FF04C08F
:10A6500021503E4F4F4F5F4F69E0559547953795D5
:10A6600027956A95D1F780911E0390911F03820F61
:10A67000931F90931F0380931E03D801C70117FFF8
:10A6800003C00796A11DB11D23E0B595A795979529
:10A6900087952A95D1F78093120390931303A09383
:10A6A0001403B093150388579C4EAF4FBF4F64F40B
:10A6B00088E79CEEAFEFBFEF8093120390931303F4
:10A6C000A0931403B0931503209112033091130348
:10A6D000409114035091150357FF04C021503F4F80
:10A6E0004F4F5F4F232F342F452F552747FD5A9546
:10A6F0008091540290915502820F931F90935502BE
:10A700008093540211C081E0809321030DC0109208
:10A7100021030AC010921F0310921E0384E690E0EA
:10A7200090938C0180938B016889262F3327809129
:10A730001E0390911F032817390724F430931F0339
:10A7400020931E0310914708112379F0212F3327FE
:10A7500027FD309580911E0390911F03281739071C
:10A7600024F430931F0320931E0340910303509160
:10A77000040360910503709106034138510561059A
:10A78000710574F08091DB029091DC0220911E0330
:10A7900030911F03820F931F9093DC028093DB02A2
:10A7A00040585F4F6F4F7F4F74F48091DB02909160
:10A7B000DC0220911E0330911F03821B930B9093A8
:10A7C000DC028093DB0281E090E090931F03809392
:10A7D0001E03C0900703D0900803E0900903F09097
:10A7E0000A03D701C601F7FE07C088279927DC01B5
:10A7F0008C199D09AE09BF0981509240A040B0401C
:10A8000034F084E090E090931F0380931E038091C6
:10A81000280390912903A0912A03B0912B03209142
:10A820009607309197074091980750919907821B9E
:10A83000930BA40BB50B815E914BAF4FBF4F8F5362
:10A840009C49A040B04018F019310CF4FFC001E061
:10A85000C01600E1D00600E0E00600E0F0060CF4CF
:10A8600073C080912203882309F46AC0D701C6010E
:10A87000F7FE07C088279927DC018C199D09AE09CE
:10A88000BF099C01AD01B7FF04C021503E4F4F4F9F
:10A890005F4F09E055954795379527950A95D1F76C
:10A8A00080911E0390911F03820F931F90931F03AB
:10A8B00080931E03D701C601F7FE03C00796A11DB2
:10A8C000B11D13E0B595A795979587951A95D1F782
:10A8D0008093160390931703A0931803B093190362
:10A8E00089589341A040B04064F088E893E1A0E02B
:10A8F000B0E08093160390931703A0931803B093CE
:10A9000019032091160330911703409118035091B9
:10A91000190357FF04C021503F4F4F4F5F4F232F64
:10A92000342F452F552747FD5A9580915602909117
:10A930005702820F931F909357028093560206C0CE
:10A9400081E08093220302C01092220320E0C2160D
:10A9500020EFD2062FEFE2062FEFF2060CF073C0C5
:10A9600080912303882309F46AC0D701C601F7FE4A
:10A9700007C088279927DC018C199D09AE09BF09FA
:10A980009C01AD01B7FF04C021503E4F4F4F5F4FB8
:10A99000E9E05595479537952795EA95D1F7809148
:10A9A0001E0390911F03820F931F90931F038093A8
:10A9B0001E03D701C601F7FE03C00796A11DB11DF6
:10A9C00073E0B595A795979587957A95D1F780937C
:10A9D000160390931703A0931803B0931903885795
:10A9E0009C4EAF4FBF4F64F488E79CEEAFEFBFEFD4
:10A9F0008093160390931703A0931803B093190341
:10AA000020911603309117034091180350911903B8
:10AA100057FF04C021503F4F4F4F5F4F232F342F1C
:10AA2000452F552747FD5A95809156029091570220
:10AA3000820F931F909357028093560211C081E0BA
:10AA4000809323030DC0109223030AC010921F03AA
:10AA500010921E0384E690E090938C0180938B010A
:10AA60004889242F332780911E0390911F032817B4
:10AA7000390724F430931F0320931E038091470865
:10AA8000882379F0282F332727FD309580911E03E6
:10AA900090911F032817390724F430931F03209344
:10AAA0001E034091070350910803609109037091C0
:10AAB0000A03413851056105710574F08091D9028E
:10AAC0009091DA0220911E0330911F03820F931F91
:10AAD0009093DA028093D90240585F4F6F4F7F4FB7
:10AAE000CCF48091D9029091DA0220911E0330912A
:10AAF0001F03821B930B9093DA028093D9020AC042
:10AB0000109257021092560210925502109254025F
:10AB10001092820280919C07882341F41092570280
:10AB200010925602109255021092540280918E0794
:10AB300090918F07A0919007B09191078093240383
:10AB400090932503A0932603B09327038091960743
:10AB500090919707A0919807B09199078093280347
:10AB600090932903A0932A03B0932B031092B6026B
:10AB70001092B7021092B8021092B9021092B2026B
:10AB80001092B3021092B4021092B5021092AE026B
:10AB90001092AF021092B0021092B10210928E0782
:10ABA00010928F07109290071092910710929607BB
:10ABB00010929707109298071092990710928507A4
:10ABC00010928607109287071092880710927607D6
:10ABD0001092770710927807109279071092EC0183
:10ABE0001092EB01E0907802F0907902C701F7FE35
:10ABF00004C0882799278E199F0904973CF08091FB
:10AC0000B60784FD03C082E3809311031091E7052A
:10AC1000A12EBB24CC24DD24B701882777FD8095A5
:10AC2000982F9701F7FE04C0222733272E193F09DA
:10AC3000442737FD4095542F0E945B8A9B01AC014D
:10AC4000C601B5010E945B8A97FF04C061507E4F28
:10AC50008F4F9F4F59E095958795779567955A95B2
:10AC6000D1F79B01812F99278E9DD0018F9DB00D2B
:10AC70009E9DB00D1124CD01B7FD03969595879546
:10AC800095958795280F391F809158029091590208
:10AC9000280F391F442737FD4095542F2093F70282
:10ACA0003093F8024093F9025093FA028091960291
:10ACB00090919702A0919802B0919902821B930BF8
:10ACC000A40BB50B8093960290939702A0939802E1
:10ACD000B09399028155934CA040B04064F080E558
:10ACE00093ECA0E0B0E08093960290939702A0933B
:10ACF0009802B09399028091960290919702A09148
:10AD00009802B0919902805B9C43AF4FBF4F64F4AF
:10AD100080EB9CE3AFEFBFEF809396029093970296
:10AD2000A0939802B093990200918F011091900125
:10AD300017FDFCC08091B60783FFF8C080918E019B
:10AD4000815080938E01882309F0F4C08DE08093B8
:10AD50008E018091C6029091C702A091C802B09165
:10AD6000C902B7FF04C081509E4FAF4FBF4F39E0BB
:10AD7000B595A795979587953A95D1F77C0197FF5B
:10AD800004C0F094E194F108F3948091BE02909194
:10AD9000BF02A091C002B091C102B7FF04C08150B0
:10ADA0009E4FAF4FBF4F29E0B595A79597958795D3
:10ADB0002A95D1F79C0197FF03C0309521953F4F0D
:10ADC000E216F3060CF47901B701F7FE02C0695FE1
:10ADD0007F4F2B01A3E055944794AA95E1F722E019
:10ADE00030E0420E531E6090C6077090C7078090F7
:10ADF000C8079090C90720914301309144014091C8
:10AE0000450150914601C401B3010E94CF8A590106
:10AE10006A013093740720937307021B130BC80158
:10AE2000845E9D4F68E671E00E949A8A9C01245BD3
:10AE3000304080918B0190918C01009731F0019707
:10AE400090938C0180938B011BC049E1E416F104BF
:10AE5000BCF48091800290918102820F931F9093A5
:10AE600081028093800280911103882349F08150F0
:10AE700080931103882321F4B0928502A09284026A
:10AE800080918B0190918C01892BF9F480918D0137
:10AE90009927289FB001299F700D389F700D1124AC
:10AEA000CB01B2010E949A8ACB01AA2797FDA095F7
:10AEB000BA2F680E791E8A1E9B1E6092C60770927A
:10AEC000C7078092C8079092C90780911103882311
:10AED00069F58091840290918502209173073091E9
:10AEE0007407821B930B845E9D4F68E671E00E949D
:10AEF0009A8A9C01245B304080917701869599273E
:10AF0000289FD001299FB00D389FB00D11249D01BD
:10AF1000B7FF02C0215F3F4FF4E035952795FA95C2
:10AF2000E1F7309359022093580204C0109259025D
:10AF30001092580280918202882381F010928A0236
:10AF400010928B0210928C0210928D0210928E023F
:10AF500010928F021092900210929102F090510282
:10AF6000FF20F1F480919C07282F33274427552791
:10AF70008091C6029091C702A091C802B091C90207
:10AF8000BC01CD010E945B8ADC01CB01BC01CD017B
:10AF900028EF3AE240E050E00E94CF8A390102C037
:10AFA00066247724E0905002EE20F1F480919C0713
:10AFB000282F3327442755278091BE029091BF0246
:10AFC000A091C002B091C102BC01CD010E945B8A78
:10AFD000DC01CB01BC01CD0128EF3AE240E050E0BA
:10AFE0000E94CF8A290102C0442455248091700711
:10AFF00090917107893C91051CF088EC90E005C0A8
:10B0000088539F4F34F488E39FEF909371078093A8
:10B01000700780917C0790917D07893C91051CF019
:10B0200088EC90E005C088539F4F34F488E39FEF8D
:10B0300090937D0780937C0780917E0790917F0796
:10B04000AA2797FDA095BA2F2091C407A22EBB2452
:10B05000CC24DD24BC01CD01A60195010E945B8AB0
:10B060009B01AC018091700790917107AA2797FD11
:10B07000A095BA2FE7E0880F991FAA1FBB1FEA957A
:10B08000D1F7280F391F4A1F5B1F57FF04C0215CEF
:10B090003F4F4F4F5F4F76E0559547953795279532
:10B0A0007A95D1F78301020F131F10937F07009346
:10B0B0007E0780916E0790916F07AA2797FDA09554
:10B0C000BA2FBC01CD01A60195010E945B8A9B01AC
:10B0D000AC0180917C0790917D07AA2797FDA095F0
:10B0E000BA2F67E0880F991FAA1FBB1F6A95D1F777
:10B0F000280F391F4A1F5B1F57FF04C0215C3F4FB9
:10B100004F4F5F4FF6E05595479537952795FA9540
:10B11000D1F74201820E931E90926F0780926E07C4
:10B120008091BF079091C007880F991FAA2797FDAC
:10B13000A095BA2F20917507332744275527BC01C6
:10B14000CD010E945B8A5B016C0197FF08C02FE371
:10B1500030E040E050E0A20EB31EC41ED51EE6E073
:10B16000D594C794B794A794EA95D1F780918B07AB
:10B17000282F3327442755278091AA029091AB02AC
:10B18000A091AC02B091AD02BC01CD010E945B8ADE
:10B19000DC01CB01BC01CD0120EF35E540E050E002
:10B1A0000E94CF8AB501620F731F7093C00760932E
:10B1B000BF070150104134F080E090E190937F0789
:10B1C00080937E0780917E0790917F078050904FFB
:10B1D00034F480E090EF90937F0780937E0751E0F6
:10B1E000851650E1950634F080E090E190936F076A
:10B1F00080936E0780916E0790916F078050904FFB
:10B2000034F480E090EF90936F0780936E07615065
:10B21000704134F080E090E19093C0078093BF07C5
:10B220008091BF079091C0078050904F34F480E028
:10B2300090EF9093C0078093BF0780910001482F43
:10B24000552780911E0190911F014817590794F4CA
:10B2500020911E0130911F0109811A81049FC001B4
:10B26000059F900D149F900D1124B9010E94868AAC
:10B270007A83698329813A81220F331F220F331F7A
:10B280003A8329834091B60740FD02C00C94366191
:10B29000EE2009F0EBC7FF2009F0E8C700E010E05E
:10B2A00048018091520290915302909354058093EB
:10B2B00053052091DD023091DE022115310509F0A0
:10B2C0003FC080911401909115018959934058F025
:10B2D00087B5803F20F48091EF01815011C081E05B
:10B2E000809335034EC080911401909115018436EE
:10B2F000910508F587B58031D0F08091EF018F5F1F
:10B300008093EF019FE089029001112480917A05DA
:10B31000821B87BD8CE291E09093DD018093DC017C
:10B320008EE591E09093DE028093DD022AC081E0F9
:10B330008093340326C0F0923403F092350321C089
:10B340008091660290916702A0916802B0916902B3
:10B3500064E0880F991FAA1FBB1F6A95D1F78093DD
:10B36000F0019093F101A093F201B093F3011093D7
:10B37000EE010093ED01215030403093DE02209326
:10B38000DD0220917A0141FF24C02233D8F480915C
:10B3900091018150809391018F3FD9F510928302E2
:10B3A0008091660290916702A0916802B091690253
:10B3B0008093620290936302A0936402B09365024B
:10B3C00081E004C081E08093830288EC8093910146
:10B3D00020C08091470190914801820F911D2091DA
:10B3E000E0053327829FA001839F500D929F500D4F
:10B3F0001124CA01AA2797FDA095BA2F8093620253
:10B4000090936302A0936402B093650281E08093FD
:10B4100083028091C6029091C702A091C802B091A8
:10B42000C902E0904301F090440100914501109160
:10B430004601BC01CD01A80197010E94CF8A5901A4
:10B440006A018091BE029091BF02A091C002B091AA
:10B45000C102BC01CD01A80197010E94CF8AB901A8
:10B46000C5010E9484885C01CC971CF05CE3A52E8A
:10B47000B12CC5010E94DE6C5C0180E28093420128
:10B48000109261021092600280918302882309F475
:10B490005FC58091360299279C012071307084FD30
:10B4A00057C58091350282608093350270919A076A
:10B4B000872F992741E0C42ED12CC822D92280FDA4
:10B4C00004C08091B60781FD10C0C980DA80309336
:10B4D0002D0320932C03309361022093600280910E
:10B4E0003602806C80933602ABC28091360281FFB7
:10B4F0007AC20091810110918201C8010F962090BB
:10B50000760230907702821593050CF058C0809136
:10B510003403882309F053C08091360287FF15C099
:10B52000809136028F7780933602809166029091E7
:10B530006702A0916802B0916902809362029093C1
:10B540006302A0936402B093650280913602806426
:10B5500080933602E0907A07EE20F1F0809162024B
:10B5600090916302A0916402B0916502BC01CD018B
:10B5700024E630E040E050E00E94CF8A8E2D9927EB
:10B58000AA27BB2782179307A407B5072CF4D092EC
:10B590006102C092600210C0C101801B910B0F9725
:10B5A00097FF03C0909581959F4F90936102809380
:10B5B00060028BE28093420110925A0216C1C801C8
:10B5C0000F9728163906C4F5209135032223A1F5DB
:10B5D0008091360286FF15C0809136028F7B809362
:10B5E00036028091660290916702A0916802B09144
:10B5F00069028093620290936302A0936402B09305
:10B60000650280913602806880933602C101801BFA
:10B61000910B0F9697FF03C0909581959F4F909542
:10B6200081959F4F90936102809360028DE2809399
:10B63000420120935A02D9C08DE380934201609168
:10B640005B02662371F120915C0230915D024091B2
:10B650005E0250915F028091620290916302A0911C
:10B660006402B091650282179307A407B507CCF472
:10B6700080913602806480933602862F99279093BA
:10B680006102809360028AE080935A028EE5809383
:10B6900042018091360287FFA8C0809136028F77E1
:10B6A00033C0662309F443C020915C0230915D02EF
:10B6B00040915E0250915F0280916202909163021C
:10B6C000A0916402B0916502281739074A075B0709
:10B6D00074F580913602806880933602862F992710
:10B6E000909581959F4F909361028093600286EFC1
:10B6F00080935A0286E7809342018091360286FF4A
:10B7000074C0809136028F7B8093360280916602EE
:10B7100090916702A0916802B091690280936202E1
:10B7200090936302A0936402B09365025EC080911F
:10B730003602807C09F459C080915A02882379F539
:10B74000E0906602F0906702009168021091690231
:10B75000D801C70180589040A040B04020916202BB
:10B760003091630240916402509165028217930701
:10B77000A407B5075CF4D801C70180589F4FAF4FAD
:10B78000BF4F281739074A075B075CF080936202B6
:10B7900090936302A0936402B093650202C010927A
:10B7A0005A02809136028F738093360210922D03D5
:10B7B00010922C0371FF06C084EF91E09093DD019D
:10B7C0008093DC0180916A02882379F4809166027B
:10B7D00090916702A0916802B0916902C397A10598
:10B7E000B1051CF081E080936A0260912C03709196
:10B7F0002D038091600290916102680F791F709310
:10B800002D0360932C03CB0177FF04C08827992771
:10B81000861B970B855F91400CF4CEC040915A0275
:10B82000442389F180915C0290915D022091620233
:10B8300030916302821B930B0996439748F48091E1
:10B840005C0290915D02A0915E02B0915F0212C015
:10B85000242F332727FD3095432F532F80916202E9
:10B8600090916302A0916402B0916502820F931FD0
:10B87000A41FB51F8093620290936302A093640299
:10B88000B093650224C08091E0052091620230915E
:10B89000630240916402509165021616170644F443
:10B8A00063E00E947A8A280F311D411D511D07C097
:10B8B00063E00E947A8A281B3109410951092093CB
:10B8C00062023093630240936402509365021092C7
:10B8D0002D0310922C03E0906602F0906702009115
:10B8E000680210916902D801C70180509440A040BD
:10B8F000B040209162023091630240916402509105
:10B90000650282179307A407B5075CF4D801C70145
:10B9100080509C4FAF4FBF4F281739074A075B072E
:10B9200044F08093620290936302A0936402B09308
:10B93000650280919A0781FF06C084E690E09093AB
:10B94000DD018093DC018091E4058823A9F58091D5
:10B950005B02882389F5409152025091530257FFB0
:10B9600002C04D5F5F4F559547955595479580911E
:10B970001E0190911F01209100013327489FF00183
:10B98000499FF00D589FF00D1124CF01B9010E947D
:10B990009A8A7093820160938101663471051CF468
:10B9A00086E490E005C06739710534F086E990E0DF
:10B9B00090938201809381018091DD029091DE025B
:10B9C000892BD1F18091660290916702A091680263
:10B9D000B09169028093620290936302A093640223
:10B9E000B093650229C08091660290916702A09190
:10B9F0006802B091690280599140A040B0408093A4
:10BA0000620290936302A0936402B09365028091F6
:10BA1000E405882311F0992702C088E790E090930D
:10BA2000820180938101E980FA80F0925302E092D2
:10BA300052028EE280934201C0905202D090530293
:10BA4000E0906602F090670200916802109169022E
:10BA5000209162023091630240916402509165022C
:10BA60002E153F054007510724F080919A0780FD6D
:10BA7000BBC28091DD029091DE02892B39F0C0902B
:10BA80005202D090530200E010E0D7C0D801C701A5
:10BA9000821B930BA40BB50B8093FB029093FC02CB
:10BAA000A093FD02B093FE02823000E890070FEFF2
:10BAB000A0070FEFB0072CF481E090E8AFEFBFEFE5
:10BAC00009C08F5F9F47A040B04064F08FEF9FE7B1
:10BAD000A0E0B0E08093FB029093FC02A093FD02F3
:10BAE000B093FE020091FB021091FC02809179015B
:10BAF000282F3327442755278091FB029091FC0281
:10BB0000A091FD02B091FE02BC01CD010E945B8AB2
:10BB100097FF04C0615E7F4F8F4F9F4F25E0959543
:10BB20008795779567952A95D1F76093FB02709377
:10BB3000FC028093FD029093FE0265302EEF7207A7
:10BB40002FEF82072FEF92072CF484E09EEFAFEFE8
:10BB5000BFEF09C0605074408040904064F080E0C6
:10BB600094E0A0E0B0E08093FB029093FC02A093ED
:10BB7000FD02B093FE028090FB029090FC022091A7
:10BB8000ED013091EE0137FF02C0295F3F4F83E0A6
:10BB9000359527958A95E1F74FEF223834071CF445
:10BBA00021E83FEF05C02038310514F020E830E0EF
:10BBB000C901AA2797FDA095BA2F20917B013327B1
:10BBC00044275527BC01CD010E945B8A97FF04C022
:10BBD0006D5F7F4F8F4F9F4FB2E09595879577951B
:10BBE0006795BA95D1F79B015FEF613075071CF43B
:10BBF00020E03FEF06C06F3F710519F014F020E020
:10BC000031E080913602807C49F0C90137FD03960E
:10BC10009C0135952795359527950DC080919A07FC
:10BC200080FF09C0C90137FD07969C01F3E03595F7
:10BC30002795FA95E1F7820E931E20917801222331
:10BC400009F454C060918602709187028091880245
:10BC50009091890297FF04C061587F4F8F4F9F4F8B
:10BC6000E7E09595879577956795EA95D1F733271E
:10BC7000442755270E945B8A97FF04C0615E7F4F6F
:10BC80008F4F9F4F55E095958795779567955A9576
:10BC9000D1F76093FB027093FC028093FD029093B6
:10BCA000FE026138AFEF7A07AFEF8A07AFEF9A076E
:10BCB0002CF480E89FEFAFEFBFEF0AC06F3F710534
:10BCC0008105910569F064F080E091E0A0E0B0E0CA
:10BCD0008093FB029093FC02A093FD02B093FE02BE
:10BCE0008091FB029091FC02880E991E8091760152
:10BCF000282F332780914A08992787FD9095289F00
:10BD0000F001299FF00D389FF00D11249F01F7FFDE
:10BD100002C021583F4F220F232F221F330BFFEF6A
:10BD200021383F071CF420E83FEF06C02F3F3105C4
:10BD300019F014F020E031E0820E931EC401AA270E
:10BD400097FDA095BA2FE0905202F0905302970110
:10BD5000442737FD4095542FBC01CD010E945B8ADA
:10BD600097FF04C061507E4F8F4F9F4F29E09595FC
:10BD70008795779567952A95D1F7C61AD70A809146
:10BD8000600290916102892B09F060C01E141F04AB
:10BD90000CF05CC0980117FF03C0309521953F4F10
:10BDA0002D33310540F480917E0290917F028C15F5
:10BDB0009D0574F526C02C53304085E036952795B7
:10BDC0008A95E1F72031310510F02FE030E0409105
:10BDD0007E0250917F0210161106E4F480E190E09B
:10BDE000821B930B489F9001499F300D589F300D47
:10BDF0001124B4E036952795BA95E1F72C153D0549
:10BE000020F580917F0190918001C816D906F4F049
:10BE10006C011CC0205F3F4F80917F019091800199
:10BE2000829F8001839F100D929F100D1124980115
:10BE3000A4E036952795AA95E1F74C155D0514F019
:10BE40006A0104C0C216D30608F06901C601AA2718
:10BE500097FDA095BA2FFDE0880F991FAA1FBB1F61
:10BE6000FA95D1F79501442737FD4095542FBC0131
:10BE7000CD010E94CF8A2093FF02309300034093AC
:10BE8000010350930203C090FF02D0900003809101
:10BE90002E0390912F039C01220F331F280F391F6F
:10BEA0002C0D3D1D37FF02C02D5F3F4FA901559559
:10BEB00047955595479550932F0340932E038091B6
:10BEC000DC05282F3327220F331F220F331F24179F
:10BED00035076CF48091BE07282F3327220F331FBC
:10BEE000220F331F205530404217530724F0309360
:10BEF0002F0320932E0380919A0780FF14C0809116
:10BF00002E0390912F0329813A818217930724F001
:10BF100030932F0320932E0340912E0350912F0333
:10BF20005A83498361C029813A812E193F0937FF1D
:10BF300002C02D5F3F4F3595279535952795609128
:10BF40002E0370912F03620F731F7A8369834CC095
:10BF50008091E405882301F56091520270915302AB
:10BF600077FF02C06D5F7F4F7595679575956795F3
:10BF700040911E0150911F0180910001282F33270D
:10BF8000649FC001659F900D749F900D1124B901AD
:10BF90000E949A8ACB0101C09927909382018093D5
:10BFA00081018091810190918201873491051CF477
:10BFB00086E490E005C08639910534F086E990E08A
:10BFC000909382018093810189819A8190932F03BC
:10BFD00080932E0380913602806C8093360280918C
:10BFE00035028D7F809335028091360299279C011E
:10BFF0002270307081FF2BC180913003909131030A
:10C00000A0913203B09133030097A105B10521F04F
:10C0100080916A028130B1F4E981FA81CF01AA27C7
:10C0200097FDA095BA2F1EE0880F991FAA1FBB1F6E
:10C030001A95D1F78093300390933103A093320384
:10C04000B093330380916A02813019F482E08093C7
:10C050006A02E980FA80C701AA2797FDA095BA2F46
:10C060009501442737FD4095542FBC01CD010E9416
:10C070005B8ADC01CB018093FF0290930003A093C5
:10C080000103B0930203B7FF04C08150904EAF4F3D
:10C09000BF4F7C018D01FDE015950795F794E7945E
:10C0A000FA95D1F7E092FF02F092000300930103AA
:10C0B0001093020360913702709138022FE0603ACA
:10C0C000720750F58091300390913103A0913203B3
:10C0D000B09133039C01AD01EAE056954795379541
:10C0E0002795EA95D1F7821B930BA40BB50BA801FA
:10C0F0009701F4E0220F331F441F551FFA95D1F723
:10C10000820F931FA41FB51F8093300390933103B8
:10C11000A0933203B093330360547F4118F58091AC
:10C12000300390913103A0913203B09133039C010D
:10C13000AD01ECE05695479537952795EA95D1F7EF
:10C14000821B930BA40BB50BA801970172E0220F81
:10C15000331F441F551F7A95D1F7820F931FA41FD9
:10C16000B51F38C08091ED019091EE018091ED01F5
:10C170009091EE0197FF03C0909581959F4F843673
:10C18000910584F580916602909167022091620288
:10C1900030916302821B930B81509F4F8F5F9140C0
:10C1A00008F58091300390913103A0913203B09152
:10C1B00033039C01AD016EE0569547953795279561
:10C1C0006A95D1F7821B930BA40BB50B8E0D9F1DA7
:10C1D000A01FB11F8093300390933103A0933203CB
:10C1E000B09333038091300390913103A0913203D7
:10C1F000B09133035EE0B695A795979587955A95CC
:10C20000D1F790935302809352024091E205442368
:10C2100099F055279C01BA010E949A8AC901861B90
:10C22000970B90937F0280937E02260F371F3093E7
:10C23000800120937F011FC010927F0210927E0226
:10C240008FEF93E09093800180937F0114C0109250
:10C250006A0210923003109231031092320310924E
:10C260003303309353022093520205C0809136026B
:10C27000806C8093360220918307822F9927880F44
:10C28000991F880F991F889669817A818617970769
:10C2900014F09A8389837091BE077D8B872F99272D
:10C2A000880F991F880F991F80559040A981BA81E6
:10C2B0008A179B0714F49A83898380912502882327
:10C2C00041F4809151088F3F21F4809146038823E7
:10C2D000E9F080913702909138020297C097B0F44C
:10C2E000E981FA811E161F068CF481E090E090939C
:10C2F000380280933702E22EFF24EE0CFF1CEE0C76
:10C30000FF1C8701085D1F4F1A83098329813A8129
:10C3100030933805209337058091F7029091F80209
:10C32000A091F902B091FA0212E0880F991FAA1F9A
:10C33000BB1F1A95D1F70091BF071091C007081BCA
:10C34000190B213A31058CF0C90137FD01969595FD
:10C350008795801791070CF48C01909581959F4FDC
:10C36000081719076CF48C010BC00135110514F086
:10C3700000E510E03FEF003B130714F400EB1FEF64
:10C380004D89242F3327220F331F220F331FC9015A
:10C3900069817A81861B970B801791070CF48C01B9
:10C3A00089819A81821B930B081719070CF48C0161
:10C3B00080917E0790917F0760917C0270917D0251
:10C3C000861B970B90938D0780938C07D0909C07CA
:10C3D00020918E0230918F024091900250919102F3
:10C3E000DD2041F0661A770AC301AA2797FDA095C0
:10C3F000BA2F04C0AA2797FDA095BA2F280F391F7E
:10C400004A1F5B1F20938E0230938F02409390024D
:10C410005093910280918E0290918F02A091900290
:10C42000B091910281509A4FA040B04064F080E0FA
:10C430009AEFA0E0B0E080938E0290938F02A093D9
:10C440009002B093910280918E0290918F02A09100
:10C450009002B091910280509640AF4FBF4F64F46C
:10C4600080E096E0AFEFBFEF80938E0290938F0253
:10C47000A0939002B0939102C090F10520918C0797
:10C4800030918D0778E0E72EEC1498F08C2D9927E9
:10C49000829FA001839F500D929F500D1124CA01CD
:10C4A00057FD07967C0163E0F594E7946A95E1F700
:10C4B00012C08C2D86959927829FB001839F700DA5
:10C4C000929F700D1124CB0177FD03967C01F594AA
:10C4D000E794F594E794A0907C01B0907D019501DC
:10C4E000442737FD4095542F80918E0290918F0202
:10C4F000A0919002B0919102BC01CD010E94CF8A1F
:10C50000E20EF31E90906801692D772788279927FE
:10C51000980117FF04C022273327201B310B37FF58
:10C5200002C02F5F3F4F35952795A981BA812A0F09
:10C530003B1F442737FD4095542F0E945B8A97FF8D
:10C5400004C0615C7F4F8F4F9F4F26E09595879584
:10C55000779567952A95D1F79B016E157F050CF4A9
:10C560007B01309521953F4FE216F3060CF47901DB
:10C5700080916E0790916F0760917A0270917B02B3
:10C58000861B970B90936D0780936C0720918A020E
:10C5900030918B0240918C0250918D02DD2041F050
:10C5A000461A570AC201AA2797FDA095BA2F04C0C0
:10C5B000AA2797FDA095BA2F280F391F4A1F5B1F86
:10C5C00020938A0230938B0240938C0250938D0209
:10C5D00080918A0290918B02A0918C02B0918D0281
:10C5E00081509A4FA040B04064F080E09AEFA0E004
:10C5F000B0E080938A0290938B02A0938C02B09358
:10C600008D0280918A0290918B02A0918C02B09150
:10C610008D0280509640AF4FBF4F64F480E096E0AB
:10C62000AFEFBFEF80938A0290938B02A0938C02AE
:10C63000B0938D0220916C0730916D0748E04C1546
:10C6400098F08C2D9927829FB001839F700D929F47
:10C65000700D1124CB0177FD07966C01B3E0D594E2
:10C66000C794BA95E1F712C0C6948C2D9927829F82
:10C67000D001839FB00D929FB00D1124CD01B7FD65
:10C6800003966C01D594C794D594C794950144271B
:10C6900037FD4095542F80918A0290918B02A09192
:10C6A0008C02B0918D02BC01CD010E94CF8AC20ED6
:10C6B000D31E692D772788279927980117FF04C073
:10C6C00022273327201B310B37FF02C02F5F3F4F3C
:10C6D00035952795E981FA812E0F3F1F442737FDB5
:10C6E0004095542F0E945B8A97FF04C0615C7F4F86
:10C6F0008F4F9F4FE6E09595879577956795EA95DB
:10C70000D1F79B016C157D050CF46B0130952195DB
:10C710003F4FC216D3060CF4690180918307282E7F
:10C720003324509032066CE9862E66E0962E53E54F
:10C73000A52E56E0B52E4BE0442E3DE9632E37E0A2
:10C74000732ED5012C9112160CF029C1203429F436
:10C75000E981FA81FF8BEE8B1FC049815A81CA01A2
:10C76000AA2797FDA095BA2F332727FD3095432F91
:10C77000532FBC01CD010E945B8A97FF04C0615C0E
:10C780007F4F8F4F9F4F26E09595879577956795BB
:10C790002A95D1F77F8B6E8BF5012181203439F4F6
:10C7A0002E893F892E0D3F1D3F8B2E8B2AC0203CAA
:10C7B00039F44E895F894E195F095F8B4E8B21C01A
:10C7C000C701AA2797FDA095BA2F332727FD3095DB
:10C7D000432F532FBC01CD010E945B8A97FF04C0F9
:10C7E000615C7F4F8F4F9F4FB6E09595879577950A
:10C7F0006795BA95D1F7AE89BF89A60FB71FBF8BD2
:10C80000AE8BF5012281203439F42E893F892C0D1D
:10C810003D1D3F8B2E8B2AC0203C39F44E895F8909
:10C820004C195D095F8B4E8B21C0C601AA2797FD6D
:10C83000A095BA2F332727FD3095432F532FBC01E6
:10C84000CD010E945B8A97FF04C0615C7F4F8F4FD0
:10C850009F4FA6E09595879577956795AA95D1F70F
:10C86000AE89BF89A60FB71FBF8BAE8BF5012381A1
:10C87000203439F42E893F89200F311F3F8B2E8BB6
:10C880002AC0203C39F44E895F89401B510B5F8BD5
:10C890004E8B21C0C801AA2797FDA095BA2F332738
:10C8A00027FD3095432F532FBC01CD010E945B8A99
:10C8B00097FF04C0615C7F4F8F4F9F4FF6E09595C7
:10C8C000879577956795FA95D1F7AE89BF89A60FB9
:10C8D000B71FBF8BAE8BF301808191812E893F8979
:10C8E0008217930764F4B901680F791F77FF02C0BC
:10C8F0006F5F7F4F759567957F8B6E8B1DC0552041
:10C9000049F44E895F89440F551F481B590B5F8BB3
:10C910004E8B12C051E0551578F4252D33276E89C2
:10C920007F89861B970BB9010E949A8AAE89BF89BD
:10C93000A60FB71FBF8BAE8BC101880F991F880F41
:10C94000991FEE89FF898E179F0764F4FD898F2F49
:10C950009927880F991F880F991F2E893F892817BB
:10C96000390714F09F8B8E8B8E899F8997FD0396D4
:10C970009595879595958795F4018183880F991FE3
:10C98000880F991F2E893F89281B390BC901880FF1
:10C990008283EE89FF89D301ED93FC9303C0F401F8
:10C9A000118212824A9422E030E0620E731E44E04B
:10C9B00050E0A40EB51E68E070E0860E971E47FE9C
:10C9C000C0CEE2E1C95E0C94068B84B1806A84B962
:10C9D0003D9A82E58CBD1DBC459A81E08093D007CD
:10C9E0008AEA8093E10783E88093E2078AE08093F4
:10C9F000E3071092E5071092E4071092E707109200
:10CA0000E607109249081092050808953091D00762
:10CA1000332309F085C00DB407FE82C084E0809303
:10CA2000DB01459A2EB58091490399278130910504
:10CA300089F0823091051CF4892B21F03EC00297C9
:10CA4000B9F03BC03093040820934A032138A9F57C
:10CA500081E008C0253549F480914A03820F809314
:10CA60004A0382E08093490328C03093490325C0DC
:10CA700080910408E82FFF27EA5DF74F20838F5F3E
:10CA80008093040890914A038032A0F0291769F43A
:10CA900080E2A6E2B8E0E6E0F8E00D9001928A9527
:10CAA000E1F781E08093050802C0309305081092F9
:10CAB000490303C0920F90934A032091E00722326A
:10CAC00008F028C0459800000000000000000000A9
:10CAD0000000000000000000000000000000000056
:10CAE0000000000000000000000000000000000046
:10CAF000000000000000E091D907F091DA07E20F92
:10CB0000F11D80818EBD809102089081890F8093F4
:10CB1000020803C081E08093D0072F5F2093E007D5
:10CB20000895EF92FF920F931F938091EA05992742
:10CB3000880F991F880F991F7C010027F7FC00952B
:10CB4000102F8091C6029091C702A091C802B091A7
:10CB5000C902BC01CD01A80197010E94CF8A309380
:10CB6000E5072093E4078091BE029091BF02A09157
:10CB7000C002B091C102BC01CD01A80197010E9481
:10CB8000CF8A3093E7072093E6072091C6073091BC
:10CB9000C7074091C8075091C907DA01C90163E08E
:10CBA000880F991FAA1FBB1F6A95D1F7820F931F89
:10CBB000A41FB51F820F931FA41FB51F209143010F
:10CBC000309144014091450150914601BC01CD0195
:10CBD0000E94CF8A3093ED072093EC078091D70213
:10CBE0009091D8022091FB013091FC01821B930BA4
:10CBF0009093F3078093F207E091CD02F091CE027B
:10CC00008091930790919407BF010E949A8A9B019B
:10CC1000220F331F220F331F260F371F260F371FF8
:10CC200037FF02C02D5F3F4F3595279535952795E6
:10CC30003093E9072093E8078091C2079091C307DA
:10CC4000BF010E949A8A9B01220F331F220F331FBC
:10CC5000260F371F260F371F37FF02C02D5F3F4FAC
:10CC600035952795359527953093EB072093EA075F
:10CC70001092CE021092CD02109294071092930758
:10CC80001092C3071092C2078091E30799278D3055
:10CC9000910509F48EC08E3091055CF48B309105BE
:10CCA00009F4B6C08C3091050CF037C10A9761F0D9
:10CCB000E7C18F30910509F4B3C18F3091050CF4B1
:10CCC00082C14097A9F1DCC180914B028093F607A5
:10CCD00080914A028093F707809149028093F80778
:10CCE000809148028093F907809147028093FA0768
:10CCF000809146028093FB07809145028093FC0758
:10CD0000809144028093FD07809136028093FE0754
:10CD100080913602837F809336020E94C52F8093D4
:10CD2000FF07809133068093000880913502A6C1E9
:10CD300080914B0890914C089093F7078093F607E9
:10CD400080914F08909150089093F9078093F807CD
:10CD500080911E0190911F018093FA07809100013C
:10CD60008093FB07809142018093FC078091B60776
:10CD70008093FD0780919A078093FE0790914B0363
:10CD80009093FF07E92FFF27A3E0EE0FFF1FAA955F
:10CD9000E1F7E456F94F87818093000885818093FD
:10CDA0000108892F8F5F6CE00E947A8A90934B0371
:10CDB00067C180911E068093F60780911F068093BD
:10CDC000F707809120068093F807809121068093D1
:10CDD000F907809122068093FA07809126068093B6
:10CDE000FB07809127068093FC078091280680939B
:10CDF000FD0780912B068093FE0780912906809382
:10CE0000FF0780912A068093000880912C0636C186
:10CE1000F8948091D105E82FFF27EE0FFF1FE35014
:10CE2000F94F0190F081E02DE038F1051CF0EFE7BB
:10CE3000F0E006C02FEFE138F20714F4E1E8FFEF6D
:10CE4000E093F6078091D205E82FFF27EE0FFF1F32
:10CE5000E350F94F0190F081E02DE038F1051CF02E
:10CE6000EFE7F0E006C06FEFE138F60714F4E1E811
:10CE7000FFEFE093F7078091D005E82FFF27EE0F33
:10CE8000FF1FE350F94F0190F081E02DE038F105EC
:10CE90001CF0EFE7F0E006C08FEFE138F80714F47C
:10CEA000E1E8FFEFE093F8078091CF05E82FFF2737
:10CEB000EE0FFF1FE350F94F0190F081E02DE038B5
:10CEC000F1051CF0EFE7F0E006C02FEFE138F207C4
:10CED00014F4E1E8FFEF7894E093F90780916D0294
:10CEE0008093FA0780916E028093FB0780916F0216
:10CEF0008093FC07809170028093FD0780917102FE
:10CF00008093FE07809172028093FF0780917302E5
:10CF10008093000880917402B1C08091C203863072
:10CF200018F01092C20385E08093F60780912D06D9
:10CF30008093F7078091660290916702A091680242
:10CF4000B0916902BC01CD0125E030E040E050E045
:10CF50000E94CF8A3093F9072093F80780916202EC
:10CF600090916302A0916402B0916502BC01CD0171
:10CF700025E030E040E050E00E94CF8A3093FB078C
:10CF80002093FA07809123068093FC078091240662
:10CF90008093FD07809125068093FE0780916C02A7
:10CFA0008093FF078091FD069091FE068093000814
:10CFB000809137059091380597FD03969595879553
:10CFC000959587955BC01092F60786E58093F707E5
:10CFD00083E08093F8078BE18093F9078091020149
:10CFE0008093FA078091A7038093FB078091A803A1
:10CFF0008093FC071092A70380718093A80380910F
:10D00000A9038093FD078091AA038093FE07809176
:10D01000AB038093FF0780912F068093000830C0F8
:10D02000809103068093F607809137068093F70777
:10D0300080916E018093F8078091FC058093F90739
:10D040008091FD058093FA078091FE058093FB0790
:10D0500080916D018093FC07809100068093FD070D
:10D06000809101068093FE07809102068093FF075E
:10D070008091510880930008809161058093010898
:10D0800080910508882309F449C18AEF80939C01A7
:10D0900081E080938E014091070850910808CA01F1
:10D0A00081509E4F8F5F9340B0F4209109083091DA
:10D0B0000A08C90181509E4F8F5F934060F48091B0
:10D0C000DB0585FF08C050933A0340933903309342
:10D0D00038032093370380910D0890910E0821E0CA
:10D0E0008936920724F49093900180938F012091C8
:10D0F0001708309118088091DC019091DD018217AA
:10D10000930720F43093DD012093DC018091060821
:10D1100099278936910509F49DC08A36910544F412
:10D120008736910571F08836910509F462C0FEC01A
:10D130008A36910509F4EBC08B36910509F4DAC003
:10D14000F5C0809119088093460880911A08809351
:10D15000480880911B088093470880911C088093A1
:10D160008D0180911D0880934A0880911E0880934C
:10D170009D0180911F08809348038091200880932F
:10D180003603809143028823F9F0209121083091E1
:10D19000220837FD19C030938502209384029091B4
:10D1A0000506992389F08FE0989FC0011124281B60
:10D1B000390BC90188599E4F68E671E00E949A8A2E
:10D1C0009093850280938402209141033091420321
:10D1D0008091230890912408280F391F37FF02C03F
:10D1E0002F5F3F4F3595279530934203209341039E
:10D1F0009DC0809119088093DB0780911A08809365
:10D20000DC0780911B088093DD0780911C088093C8
:10D21000DE0780911D088093DF078091270590919C
:10D220001E08892B80932705909128059370809183
:10D230001F088C70982B909328058091200880936C
:10D240004603809121088093920180912208809367
:10D2500049086CC0809119088093D10780911A0801
:10D260008093D20780911B088093D30780911C087C
:10D270008093D40780911D0890911E089093D60743
:10D280008093D50780911F08909120089093D8072C
:10D290008093D70780912108992787FD90959093D7
:10D2A000300780932F078091220880935B02809142
:10D2B0002308909124089C01442737FD4095542F62
:10D2C000DA01C90163E0880F991FAA1FBB1F6A9585
:10D2D000D1F7820F931FA41FB51F820F931FA41FA6
:10D2E000B51F80935C0290935D02A0935E02B093A1
:10D2F0005F021CC0809119088093450380911A0831
:10D300008093440380911B08809343030FC0809156
:10D31000F505863059F40E94817108C010923A03D5
:10D320001092390310923803109237031F910F9116
:10D33000FF90EF9008958091D007882309F43BC0B7
:10D34000459881EE97E09093DA078093D907909102
:10D350004703E92FFF27ED56FE4F9F5F909347034A
:10D3600080818093E307993010F010924703109268
:10D37000D0070E94916581E08093E00700000000E3
:10D38000000000000000000000000000000000009D
:10D39000000000000000000000000000000000008D
:10D3A0000000000000000000000000008091E10784
:10D3B000809302088EBD089587B18C6087B942982A
:10D3C000439810924D0380E880939F0110924C0384
:10D3D00080939E010895809152038150809352035F
:10D3E0008F3F09F0FAC089E08093520380913602A2
:10D3F000992780739070892B21F48091A80380FF76
:10D400001DC080911C06882351F08091550388230C
:10D4100019F484E080934D0381E08093550380915B
:10D420001D068823B9F080915603882319F484E0FF
:10D4300080934C0381E0809356030CC010925503F7
:10D4400010925603809118068093530380911A0618
:10D450008093540380915503882309F040C0809144
:10D460003606282F332724FF07C080916B028823BC
:10D4700019F425FD4DC04EC090911906983F50F00B
:10D48000809195078D3D30F08091530388230CF4F3
:10D490003FC040C0983F48F080919507853029F4FF
:10D4A000809153038823B4F133C080914D038150A0
:10D4B00080934D038F3F79F58091950786958093F2
:10D4C0004D0380919F01813011F480E801C0869561
:10D4D00080939F0180919F019091530317C0809189
:10D4E0004D03815080934D038F3FA9F489E08093D1
:10D4F0004D0380919F01813011F480E801C0869531
:10D5000080939F0180919F0190911C06892311F0C7
:10D51000429A01C0429880915603882309F041C085
:10D520009091360697FF07C080916B02882319F40B
:10D5300096FD50C034C090911B06983F50F08091EA
:10D54000BD078D3D30F08091540388230CF442C018
:10D5500026C0983F48F08091BD07853029F480911E
:10D5600054038823E4F036C080914C0381508093AB
:10D570004C038F3F91F58091BD07869580934C03B6
:10D5800080919E01813011F480E801C086958093DE
:10D590009E0180919E01909154038923D9F4439870
:10D5A000089580914C03815080934C038F3FA9F4E0
:10D5B00089E080934C0380919E01813011F480E8D2
:10D5C00001C0869580939E0180919E0190911D06D9
:10D5D000892311F0439A0895439808954FB724E1A1
:10D5E00030E0F8948091C9008F778093C9008091D2
:10D5F000C9008F7B8093C9008091C9008F7D809383
:10D60000C9005A9A52985B9A539A832F992780930C
:10D61000CD002093CC008091C80082608093C80028
:10D6200080E18093C9008091CA008F778093CA00FF
:10D630008091CA008F7B8093CA008091CA008F7D41
:10D640008093CA008091CA008F7E8093CA00809127
:10D65000CA00877F8093CA008091C9008B7F809326
:10D66000C9008091CA0084608093CA008091CA007A
:10D6700082608093CA008091C80087FF03C08091B8
:10D68000CE00F9CF8091C90080688093C9004FBF58
:10D690000895EF92FF920F931F93CF93DF93482F3C
:10D6A00000E010E08091A001813061F41092A001AF
:10D6B00084E48093570310925903109258031092F8
:10D6C0005A032BC180915703882319F421E030E0DD
:10D6D00001C0980190915803992371F4232B11F004
:10D6E00081E010C084E48093570390935903909392
:10D6F000580390935A03FAC0913069F4232B09F030
:10D70000EBC082E080935803809159038F5F809330
:10D71000590383E0E9C09230D1F4232B09F0DCC037
:10D7200083E08093570340935A03909159039230BA
:10D7300039F410925B0347FF03C081E080935B03E1
:10D7400083E0809358039F5F90935903CFC0933039
:10D7500009F0C2C0232B09F0BFC09093570382E0A9
:10D7600080935803809159038F5F809359032091D0
:10D770005A03822F9927782F6627842F9927682BA1
:10D78000792B8091F505813049F47370CB0180507D
:10D79000924063E070E00E949A8A17C0823061F480
:10D7A0007770CB018050944066E070E00E949A8AC6
:10D7B0002695269526950BC0737068567140CB014F
:10D7C00077FD0196BC017595679526952695022FE4
:10D7D00011270F7010700F5F1F4F0D30110508F0EB
:10D7E00074C07801E00EF11EF701E350F94F80811B
:10D7F00091819B01281B390BC90137FF03C090950C
:10D8000081959F4F069794F480916C02883C30F488
:10D8100080916C02865F80936C0208C088EC8093D4
:10D820006C0280916F008F7D80936F00F701E35051
:10D83000F94F808191819C01220F331F280F391FDE
:10D84000260F371F37FF02C02D5F3F4FE901D595E7
:10D85000C795D595C795CB0101968C179D0714F4F4
:10D86000219706C061507040C617D7070CF4219667
:10D8700080916C02843BD0F0F701E350F94F808136
:10D880009181FE01E81BF90BCF0163E070E00E947B
:10D890009A8ACB01880F991F860F971F21E337E0E3
:10D8A000E20EF31EF7019183808307C021E337E086
:10D8B000E20EF31EF70111821082000F111F0350B8
:10D8C000194FF801D183C08311C00231110570F0E6
:10D8D00081E08093A0010AC081E08093A0011092B2
:10D8E000590310925B0384E480935703809159039A
:10D8F000803198F080915B03882331F48091A001FE
:10D90000882311F4809341011092590310925B0314
:10D910001092580384E480935703E6E0CDB7DEB756
:10D920000C94128BCF93FC0197FF05C0CFEFF095BD
:10D93000E195FF4F01C0C1E028E631E0CF01B90118
:10D940000E949A8AFC018B35910554F08B559040CA
:10D950008A35910538F484EB90E08E1B9F0BFC0117
:10D9600041E00DC0CF01855B90408A35910518F4E8
:10D97000E45BF04003C02E1B3F0BF9014FEFEE0FAD
:10D98000FF1FE356F64F259134918C2F992787FD81
:10D990009095289FB001299F700D389F700D11241C
:10D9A000842F992787FD9095689FA001699F500D4E
:10D9B000789F500D1124CA01CF9108952AE530E0D7
:10D9C000281B390BC9010E94926C0895CF93DF93F5
:10D9D00080E00E94DA7F80911E0190911F016AE031
:10D9E00070E00E949A8A9F938F9380911E0190917C
:10D9F0001F016AE070E00E949A8A7F936F9381E72B
:10DA00009AE09F938F93CDECDFE7DF93CF93E09184
:10DA10008E03F0918F0309952DB73EB7285F3F4FD6
:10DA20002DBF80919C01882361F186E00E94DA7FFE
:10DA30008091920199279F938F938091D507909120
:10DA4000D6076AE070E00E94868A7F936F938FED1D
:10DA500090E09F938F9380917307909174079F93A9
:10DA60008F938AE79AE09F938F93DF93CF93E09110
:10DA70008E03F0918F0309958DB79EB70C968DBFDD
:10DA800012C086E00E94DA7F88E89AE09F938F9325
:10DA9000DF93CF93E0918E03F0918F0309950F9060
:10DAA0000F900F900F9080914603882309F458C07F
:10DAB00080915C0390915D030E94AA19882391F0E4
:10DAC0008091A101882319F01092A10103C081E087
:10DAD0008093A1018CED95E00E94A11990935D03C4
:10DAE00080935C038091A1018823E1F080E00E9493
:10DAF000DA7F1F921F929091460381E1989FC001A7
:10DB000011248559944F9F938F93DF93CF93E09186
:10DB10008E03F0918F0309952DB73EB72A5F3F4FD3
:10DB20002DBF1EC086E00E94DA7F809146039927B0
:10DB30009F938F938FE89AE09F938F93DF93CF9378
:10DB4000E0918E03F0918F0309958DB79EB70696ED
:10DB50008DBF80916B02882319F08FE48093A80118
:10DB600080E10E94DA7F8091AA019091AB016CE381
:10DB700070E00E94868A9F938F938091AA01909172
:10DB8000AB016CE370E00E94868A7F936F93809173
:10DB90004F08909150089F938F938BE99AE09F9341
:10DBA0008F93CDECDFE7DF93CF93E0918E03F0917D
:10DBB0008F0309958091B6072DB73EB7265F3F4F7B
:10DBC0002DBF80FF29C08AE10E94DA7F8091420147
:10DBD00099279F938F938091660290916702A091FD
:10DBE0006802B0916902BC01CD0124E630E040E05A
:10DBF00050E00E94CF8A3F932F9388EA9AE09F9348
:10DC00008F93DF93CF93E0918E03F0918F0309956B
:10DC10008DB79EB708968DBFDF91CF910895CF93B2
:10DC2000DF9380E00E94DA7F8091BB06992787FD11
:10DC300090959F938F938091B306992787FD909538
:10DC40009F938F938091AB06992787FD90959F9323
:10DC50008F938091A306992787FD90959F938F932B
:10DC60008FEA9AE09F938F93CDECDFE7DF93CF931A
:10DC7000E0918E03F0918F03099580E10E94DA7F95
:10DC80002DB73EB7245F3F4F2DBF8091DB0699270C
:10DC900087FD90959F938F938091D306992787FD59
:10DCA00090959F938F938091CB06992787FD9095B0
:10DCB0009F938F938091C306992787FD90959F939B
:10DCC0008F938FEB9AE09F938F93DF93CF93E091A5
:10DCD0008E03F0918F0309958091CD052DB73EB746
:10DCE000245F3F4F2DBF853098F480E10E94DA7F9A
:10DCF0008FEC9AE09F938F93DF93CF93E0918E0305
:10DD0000F0918F0309950F900F900F900F9018C00E
:10DD10008730B0F488E10E94DA7F8FED90E09F9326
:10DD20008F9380EE9AE09F938F93DF93CF93E09150
:10DD30008E03F0918F0309958DB79EB706968DBF20
:10DD4000DF91CF9108950F931F9380E00E94DA7FB7
:10DD50002AE030E080914B0890914C08B9010E9474
:10DD6000868A9F938F9380914B0890914C08B901BC
:10DD70000E94868A7F936F9380911E0190911F016C
:10DD8000B9010E949A8A9F938F9380911E0190916E
:10DD90001F01B9010E949A8A7F936F9389EE9AE0DE
:10DDA0009F938F930DEC1FE71F930F93E0918E03CA
:10DDB000F0918F03099580E10E94DA7F8DB79EB7BD
:10DDC0000C968DBF80914F08909150089F938F9330
:10DDD00080914D0890914E089F938F938BEF9AE01E
:10DDE0009F938F931F930F93E0918E03F0918F0376
:10DDF00009958DB79EB708968DBF1F910F91089515
:10DE0000EF92FF920F931F9380E00E94DA7F8FEDD5
:10DE1000E82EF12CFF92EF9280918F01909190016A
:10DE20009F938F938091450399279F938F9387E0CA
:10DE30009BE09F938F930DEC1FE71F930F93E0914F
:10DE40008E03F0918F03099580E10E94DA7F8DB7F0
:10DE50009EB70A968DBF8091430399279F938F9316
:10DE6000FF92EF928091440399279F938F938AE1C9
:10DE70009BE09F938F931F930F93E0918E03F091FC
:10DE80008F0309958DB79EB70A968DBF1F910F918D
:10DE9000FF90EF9008950F931F93CF93DF9380919E
:10DEA0009C01CDECDFE7882309F47DC080E00E946F
:10DEB000DA7F8091D20799279F938F938091D4071F
:10DEC00099279F938F938DE29BE09F938F938E0171
:10DED000DF93CF93E0918E03F0918F0309958DB777
:10DEE0009EB708968DBF8091D307833031F48CE0C4
:10DEF0000E94DA7F8CE39BE005C08CE00E94DA7F11
:10DF000081E49BE09F938F93DF93CF93E0918E0307
:10DF1000F0918F0309950F900F900F900F908091C3
:10DF2000D10781FF12C08CE00E94DA7F86E49BE07B
:10DF30009F938F931F930F93E0918E03F0918F0324
:10DF400009950F900F900F900F9080E10E94DA7F5B
:10DF50008091920199279F938F938FED90E09F93EB
:10DF60008F938091D7079091D8079F938F9380913B
:10DF7000D5079091D6076AE070E00E94868A7F9369
:10DF80006F938BE49BE09F938F938DEC9FE79F9320
:10DF90008F93E0918E03F0918F0309958DB79EB713
:10DFA0000C968DBF12C082E00E94DA7F8EE59BE066
:10DFB0009F938F93DF93CF93E0918E03F0918F0324
:10DFC00009950F900F900F900F90DF91CF911F91B7
:10DFD0000F910895CF93C82F20915E0320935F0384
:10DFE00099278F329105E1F0803391051CF44F970A
:10DFF00079F027C08F349105D9F08F38910509F554
:10E0000086E0289FF0011124ED5AF54F849117C046
:10E0100086E0289FF0011124EC5AF54F84910FC03F
:10E0200086E0289FF0011124EB5AF54F849107C038
:10E0300086E0289FF0011124EA5AF54F84918093DD
:10E040005E0390915E0380915F039813C0E00E948D
:10E05000E07F90915E0386E0989FF0011124E95AD9
:10E06000F54F259134918C2FF901099580E090E0CE
:10E07000CF91089510924C0810924B0810925008BE
:10E0800010924F0810924E0810924D0810925108AD
:10E090008AE090E00E94A11990936103809360034D
:10E0A0000895CF93DF9380916003909161030E9464
:10E0B000AA19882309F4AFC080916003909161038D
:10E0C0000A969093610380936003E0E0F0E09F0183
:10E0D00090E05FEFACE9B6E04BE0ED018B8187FFAC
:10E0E0000BC09F5F8D81E80FF11D8981280F311DC5
:10E0F0008E81851708F4582F4150189647FFEDCFB1
:10E1000050935108232B41F520916603309167030A
:10E110004091680350916903BB27A52F942F832F4B
:10E120009093650380936403AA27BB27281B390BB0
:10E130004A0B5B0BCF01AA27BB27280F391F4A1FA9
:10E140005B1F2093660330936703409368035093EB
:10E150006903E5E0F0E013C02091640330916503AA
:10E160002E173F0718F4E21BF30B02C0E0E0F0E0CB
:10E17000892F9927880F991FE80FF91F3596F0937B
:10E180004C08E0934B08EF3FF10578F480911E01B5
:10E1900090911F018E9F90018F9F300D9E9F300D9B
:10E1A0001124C90164E670E013C0CF0196958795EC
:10E1B0009695879520911E0130911F01289FA001FF
:10E1C000299F500D389F500D1124CA0169E170E05C
:10E1D0000E94868A70934E0860934D0820916203D6
:10E1E000309163032E0F3F1F30936303209362032C
:10E1F0005EE02131350778F080914F08909150080A
:10E2000001969093500880934F0820513E403093E0
:10E21000630320936203DF91CF91089530916F03E0
:10E22000E32FFF2783E0EE0FFF1F8A95E1F7E45607
:10E23000F94F2781422F552747FD50958091700354
:10E240009927841795072CF4209370033093720359
:10E250000AC0222341F0809171039927481759077A
:10E2600014F420937103832F8F5F80936F038D309D
:10E27000D0F010926F03809171038F3F19F080935B
:10E280006B0302C010926B038091700380936C0348
:10E290008091720380936A038FEF809371031092D1
:10E2A000700310927203089595E1899F802D1124C7
:10E2B0000E94298484E19DE09F938F938BEF93E8E4
:10E2C0009F938F93E0918E03F0918F0309950F90A8
:10E2D0000F900F900F9008958091360285FF03C034
:10E2E00080E190E0089580916B02882339F080915D
:10E2F0004603882319F085E090E0089580E090E0DF
:10E30000089530E08091240899278A38910591F08A
:10E310008B38910524F48938910541F016C08D3869
:10E32000910581F08E38910549F00FC04AE958E017
:10E3300031E10BC047E559E03DE107C042E558E057
:10E3400036E203C048E758E032E29091190820E035
:10E3500080911A08281770F4931760F4DA01A90F56
:10E36000B11DE22FFF27EA5FF74F85898C939F5FEE
:10E370002F5FEECF089520E335E7809142018B3285
:10E3800011F08D32F9F48091E005282F3327809128
:10E39000600290916102829FA001839F500D929F25
:10E3A000500D1124CA0163E070E00E949A8ACB01EB
:10E3B0009B01205D3A48C196C19708F03FC02EEFFF
:10E3C00034E73CC0803229F58091360281FF36C0A7
:10E3D00020916D0330916E03205D3A4855E721335B
:10E3E000350748F085E72439380718F420E335E786
:10E3F00002C02456304045E720333407F8F454E790
:10E400002D3C350718F020E335E718C02C593F4F55
:10E4100015C08E3549F490915B028AE0989F900177
:10E420001124205D3A480AC0863741F490915B027E
:10E430008AE0989FC0011124281B390BC901089557
:10E44000EF92FF920F931F9399278A38910509F451
:10E450005DC08B38910524F48938910551F0D2C103
:10E460008D38910509F416C18E38910509F483C0E1
:10E47000C9C18091660290916702A0916802B09133
:10E480006902BC01CD0124E630E040E050E00E948A
:10E49000CF8ADA01C9018C509E4F90939E088093D9
:10E4A0009D080E94BB719093A4088093A308909349
:10E4B000A6088093A5089093A8088093A7082091A8
:10E4C0009D0830919E088091A1089091A20828177C
:10E4D000390724F43093A2082093A10880919F0863
:10E4E0009091A0088217930724F43093A0082093FA
:10E4F0009F080E946C7180939C088AE998E0909331
:10E500007E0380937D0381E190E07EC1809166026D
:10E5100090916702A0916802B0916902BC01CD019F
:10E5200024E630E040E050E00E94CF8ADA01C901E1
:10E530008C509E4F90936A09809369090E94BB7129
:10E5400090936C0980936B0988E790E090936E0933
:10E5500080936D091092700910926F090E946C717E
:10E560008093590987E599E090937E0380937D031A
:10E570008DE190E049C10E940E71809166029091F8
:10E580006702A0916802B0916902BC01CD0124E646
:10E5900030E040E050E00E94CF8ADA01C9018C509F
:10E5A0009E4F90936A088093690880911E01909114
:10E5B0001F01909364088093630880911E019091DD
:10E5C0001F0190936608809365088091730790916E
:10E5D000740797FD019695958795809355088093CC
:10E5E0005C082091D7073091D80737FF02C02F5F12
:10E5F0003F4F3595279520935A088091D5079091E4
:10E60000D60764E170E00E94868A60935B082093DD
:10E610006108609362080E94BB71909372088093B6
:10E62000710888E790E09093740880937308809154
:10E630001E0190911F0190936E0880936D08809148
:10E640006B038C5E8093670880916C038C5E809373
:10E65000680880914F08909150086AE070E00E942D
:10E66000868A7093700860936F080E946C71809323
:10E67000540880914B0890914C0890936C088093BB
:10E680006B0882E598E090937E0380937D0386E299
:10E6900090E0BAC00E940E718091D5079091D60784
:10E6A00064E670E00E94868A70938B0860938A0803
:10E6B000809173079091740797FD019695958795C2
:10E6C00080937B088091D7079091D80797FD01969A
:10E6D000959587958093800880910001482F552754
:10E6E0009A012B5F3F4F80911E0190911F012817C7
:10E6F000390784F480911E0190911F01841B950BB2
:10E700009C01220F331F280F391F822F82518093C3
:10E71000870802C010928708E0906602F0906702B6
:10E720000091680210916902C801B70124E630E047
:10E7300040E050E00E94CF8A3093890820938808F7
:10E7400037FF04C01092890810928808C801B701E9
:10E7500024E630E040E050E00E94CF8ADA01C901AF
:10E760008C509E4F90938D0880938C0880911E0151
:10E7700090911F01909382088093810880911E01DF
:10E7800090911F0190938408809383080E94BB712D
:10E7900090938F0880938E0888E7809390088091EB
:10E7A0001E0190911F01909394088093930880918B
:10E7B0006B038C5E8093850880916C038C5E8093E4
:10E7C000860880914F08909150086AE070E00E949E
:10E7D000868A70939608609395080E946C71809366
:10E7E0007A0880914B0890914C08909392088093FE
:10E7F000910888E798E090937E0380937D0382E2FE
:10E8000090E002C080E090E01F910F91FF90EF90A8
:10E810000895EF92FF920F931F93CF93DF93809110
:10E820006D0390916E039C0103E0220F331F0A9544
:10E83000E1F7281B390B8091ED019091EE01280F33
:10E84000391F37FF02C0295F3F4F13E035952795E9
:10E850001A95E1F730936E0320936D039091740342
:10E86000992309F050C380917303282F332744273D
:10E8700055278F5F80937303F9012131310508F02B
:10E880003FC3E058FF4F0C94218B8091360285FFE7
:10E890002AC080E00E94298480911E0190911F016E
:10E8A0006AE070E00E949A8A9F938F9380911E0184
:10E8B00090911F016AE070E00E949A8A7F936F93A3
:10E8C0008AE29DE09F938F938CE194E89F938F93CE
:10E8D000E0918E03F0918F0309952DB73EB7285F25
:10E8E0003F4F2DBF28C080E00E94298480911E01E7
:10E8F00090911F016AE070E00E949A8A9F938F9323
:10E9000080911E0190911F016AE070E00E949A8A36
:10E910007F936F9387E39DE09F938F938BEF93E8B3
:10E920009F938F93E0918E03F0918F0309958DB79C
:10E930009EB708968DBF8091B60780FF39C0809141
:10E9400083028823E9F08AE00E94298480914201B1
:10E9500099279F938F938091660290916702A0916F
:10E960006802B0916902BC01CD0124E630E040E0CC
:10E9700050E00E94CF8A3F932F9384E49DE0BAC673
:10E980008AE00E9429848091660290916702A0919A
:10E990006802B0916902BC01CD0124E630E040E09C
:10E9A00050E00E94CF8A3F932F9380E59DE0DAC725
:10E9B0008AE00E9429848BE59DE04DC68091360255
:10E9C00085FF2AC085E10E9429848091AA01909147
:10E9D000AB016CE370E00E94868A9F938F938091D5
:10E9E000AA019091AB016CE370E00E94868A7F934C
:10E9F0006F9385E69DE09F938F938CE194E89F93BE
:10EA00008F93E0918E03F0918F0309952DB73EB758
:10EA1000285F3F4F2DBF28C085E10E942984809147
:10EA2000AA019091AB016CE370E00E94868A9F93EB
:10EA30008F938091AA019091AB016CE370E00E94EA
:10EA4000868A7F936F9382E79DE09F938F938BEFEE
:10EA500093E89F938F93E0918E03F0918F03099534
:10EA60008DB79EB708968DBF8FE10E94298480E6FE
:10EA700090E09F938F9380917307909174079F9379
:10EA80008F938FE79DE09F938F93CBEFD3E8DF9336
:10EA9000CF93E0918E03F0918F0309958091350219
:10EAA0002DB73EB7285F3F4F2DBF80FF06C089E2DC
:10EAB0000E9429848AE89DE0ACC389E20E942984EF
:10EAC0008CE89DE0EBC68091360285FF1BC08AE290
:10EAD0000E94298480914F08909150089F938F93B2
:10EAE0008EE89DE09F938F938CE194E89F938F93A2
:10EAF000E0918E03F0918F0309958DB79EB706962E
:10EB00008DBF1BC08AE20E94298480914F0890919A
:10EB100050089F938F9386E99DE09F938F938BEF8F
:10EB200093E89F938F93E0918E03F0918F03099563
:10EB30002DB73EB72A5F3F4F2DBF86E30E94298441
:10EB400080914B0890914C086AE070E00E94868AA0
:10EB50009F938F9380914B0890914C086AE070E0EE
:10EB60000E94868A7F936F938EE99DE09F938F9397
:10EB70008BEF93E89F938F93E0918E03F0918F0337
:10EB800009958DB79EB70896FBC689E00E94298437
:10EB90008AEA9DE09F938F930BEF13E81F930F93E7
:10EBA000E0918E03F0918F0309958EE10E942984F4
:10EBB0000F900F900F900F908CEA9DE09F938F9392
:10EBC0001F930F93E0918E03F0918F03099583E3D8
:10EBD0000E9429840F900F900F900F908EEA9DE075
:10EBE0009F938F931F930F93E0918E03F0918F0368
:10EBF00009958FE30E9429840F900F900F900F903A
:10EC000080EB9DE09F938F931F930F93E0918E0372
:10EC1000F0918F0309958EE70E9429840F900F9041
:10EC20000F900F9086EC9DE09F938F931F930F930F
:10EC3000CCC780919C01882309F462C08DE50E94B5
:10EC400029848CED9DE09F938F93CBEFD3E8DF93E6
:10EC5000CF93E0918E03F0918F03099584E50E9494
:10EC600029840F900F900F900F908091D2079927D1
:10EC70009F938F938EED9DE09F938F93DF93CF9320
:10EC8000E0918E03F0918F0309958EE50E9429840F
:10EC90002DB73EB72A5F3F4F2DBF8091D50790918A
:10ECA000D6076AE070E00E94868A7F936F9387EEB2
:10ECB0009DE09F938F93DF93CF93E0918E03F0912C
:10ECC0008F0309958DB79EB706968DBF8091D307A8
:10ECD000833081F48091D10781FF06C08BE50E94CB
:10ECE000298481EF9DE0DAC58BE50E94298484EFB9
:10ECF0009DE0D4C58BE50E94298487EF9DE05FC726
:10ED000084E010C480919C01882309F497C080910D
:10ED10007603CBEFEC2EC3E8FC2E882309F44BC01E
:10ED200089E60E9429848091450399279F938F93B8
:10ED30008AEF9DE09F938F93FF92EF92E0918E0375
:10ED4000F0918F03099585E70E9429842DB73EB77E
:10ED50002A5F3F4F2DBF8091920199279F938F93F8
:10ED600000E610E01F930F938091D7079091D8078A
:10ED70009F938F9385E09EE09F938F93FF92EF92F6
:10ED8000E0918E03F0918F03099582E70E94298418
:10ED90008DB79EB70A968DBF8091430399279F93A5
:10EDA0008F931F930F938091440399279F938F9381
:10EDB00081E19EE0A5C682E70E94298481E29EE06F
:10EDC0009F938F93FF92EF92E0918E03F0918F03C8
:10EDD000099589E60E9429840F900F900F900F905B
:10EDE0008091D20799279F938F938091D407992779
:10EDF0009F938F9383E29EE09F938F93FF92EF9276
:10EE0000E0918E03F0918F03099584E70E94298495
:10EE10008DB79EB708968DBF8091920199279F93D9
:10EE20008F9380E690E09F938F938091D707909186
:10EE3000D8079F938F938EE29EE062C685E072C3EF
:10EE4000909146039923E1F180917A038823A1F000
:10EE5000993190F487E00E94547183E90E942984DB
:10EE60008091460399279F938F938BE39EE09F9316
:10EE70008F938BE094E87AC583E90E94298486E425
:10EE80009EE09F938F930BEF13E81F930F93E091F6
:10EE90008E03F0918F0309951F921F929091460364
:10EEA00081E1989FC00111248559944F9F938F93BE
:10EEB0001F930F93E0918E03F0918F03099529C65C
:10EEC00083E90E9429848CE49EE0C5C30E946C7192
:10EED0008093AD0880917409863059F4809176034F
:10EEE000882319F0109276039CC681E08093760304
:10EEF00098C6883009F095C60E942E8481E0CCC364
:10EF00009093730396C6913009F0D1C38091730337
:10EF1000282F3327442755278F5F80937303F901E8
:10EF20002131310508F080C6EF56FF4F0C94218B3C
:10EF30008091360285FF38C080E00E94298480914C
:10EF40004F08909150089F938F9380911E0190914C
:10EF50001F016AE070E00E949A8A9F938F938091CC
:10EF60001E0190911F016AE070E00E949A8A7F93CF
:10EF70006F938091AA019091AB016CE370E00E94C5
:10EF8000868A9F938F938091AA019091AB016CE345
:10EF900070E00E94868A7F936F9382E69EE09F9343
:10EFA0008F938CE194E80DC380E00E9429848091C6
:10EFB0004F08909150089F938F9380911E019091DC
:10EFC0001F016AE070E00E949A8A9F938F9380915C
:10EFD0001E0190911F016AE070E00E949A8A7F935F
:10EFE0006F938091AA019091AB016CE370E00E9455
:10EFF000868A9F938F938091AA019091AB016CE3D5
:10F0000070E00E94868A7F936F938DE79EE09F93C6
:10F010008F938BEF93E89F938F93E0918E03F09102
:10F020008F0309952DB73EB7225F3F4F76C585E127
:10F030000E94298480E690E09F938F9380918F01B6
:10F04000909190019F938F9388E99EE09F938F9377
:10F05000CBEFD3E8DF93CF93E0918E03F0918F0352
:10F0600009958091B6072DB73EB7285F3F4F2DBF5A
:10F0700080FF51C080918302882339F18FE10E9483
:10F0800029848091660290916702A0916802B091F4
:10F090006902BC01CD0124E630E040E050E00E946E
:10F0A000CF8A3F932F9382EA9EE09F938F938BE0CA
:10F0B00094E89F938F93E0918E03F0918F030995CD
:10F0C0008DB79EB706968DBF38C08FE10E94298408
:10F0D0008091660290916702A0916802B0916902E6
:10F0E000BC01CD0124E630E040E050E00E94CF8A30
:10F0F0003F932F938BEA9EE09F938F93DF93CF9361
:10F10000E0918E03F0918F0309952DB73EB72A5FEA
:10F110003F4F2DBF12C08FE10E94298484EB9EE0F7
:10F120009F938F93DF93CF93E0918E03F0918F03A2
:10F1300009950F900F900F900F9089E20E942984FB
:10F140008091420199279F938F938EEB9EE09F932E
:10F150008F93DF93CF930CC480919C018823F9F0A7
:10F160008BE20E9429848091920199279F938F932B
:10F170008091D5079091D6076AE070E00E94868A58
:10F180007F936F9380E690E09F938F938091D70752
:10F190009091D8079F938F9381EC9EE05CC182E0B1
:10F1A000C1C18FE30E94298480914D0890914E083F
:10F1B0009F938F9380914B0890914C086AE070E088
:10F1C0000E94868A9F938F9380914B0890914C0860
:10F1D0006AE070E00E94868A7F936F9388ED9EE0DC
:10F1E0009F938F93CBEFD3E8DF93CF93E0918E0380
:10F1F000F0918F030995809135022DB73EB7265FB8
:10F200003F4F2DBF80FF0AC082E50E9429848CEE0B
:10F210009EE09F938F938BE094E8D5C482E50E9493
:10F2200029848FEE9EE03AC380919C01BBEFEB2EC8
:10F23000B3E8FB2E882309F449C084E50E942984A1
:10F240008091D20799279F938F938091D407992714
:10F250009F938F9382EF9EE09F938F93E701FF929E
:10F26000EF92E0918E03F0918F0309958DB79EB7D1
:10F2700008968DBF8091D307833051F484E60E94B5
:10F28000298485E09FE09F938F93FF92EF920BC0BC
:10F2900084E60E9429848BE09FE09F938F938CE10A
:10F2A00094E89F938F93E0918E03F0918F030995DB
:10F2B0000F900F900F900F908091D10781FFB9C4EC
:10F2C00084E60E94298481E19FE0E8C284E50E94EF
:10F2D000298487E19FE09F938F93FF92EF9275C4FB
:10F2E00080917503ABEFEA2EA3E8FA2E882309F488
:10F2F00050C089E60E9429848091B9066AE00E9484
:10F300007A8A892F99279F938F938091B9060E94BB
:10F310007A8A99279F938F938091B1060E947A8A67
:10F32000892F99279F938F938091B1060E947A8AA3
:10F3300099279F938F938091A9060E947A8A892F9B
:10F3400099279F938F938091A9060E947A8A992783
:10F350009F938F938091A1060E947A8A892F992783
:10F360009F938F938091A1060E947A8A99279F93F9
:10F370008F938DE29FE09F938F93FF92EF92E091A6
:10F380008E03F0918F0309952DB73EB72C5E3F4F4A
:10F39000C4C389E60E94298480E690E09F938F93FE
:10F3A0008091BB06992787FD90959F938F938091BD
:10F3B000B306992787FD90959F938F938091AB0615
:10F3C000992787FD90959F938F938091A306992706
:10F3D00087FD90959F938F938AE49FE09F938F93EF
:10F3E000FF92EF92E0918E03F0918F0309958DB714
:10F3F0009EB70E96C5C2809175039091CD05882366
:10F4000009F48DC0943009F48CC09630A1F58EE7D4
:10F410000E9429848091C9066AE00E947A8A892F15
:10F4200099279F938F938091C9060E947A8A992782
:10F430009F938F938091C1060E947A8A892F992782
:10F440009F938F938091C1060E947A8A99279F93F8
:10F450008F938DE59FE09F938F938BEF93E89F931E
:10F460008F93E0918E03F0918F0309952DB73EB7EE
:10F47000245F3F4F52C3973008F4DBC38EE70E94EE
:10F4800029848091D9066AE00E947A8A892F992777
:10F490009F938F938091D9060E947A8A99279F9390
:10F4A0008F938091D1060E947A8A892F99279F9302
:10F4B0008F938091D1060E947A8A99279F938F9388
:10F4C0008091C9060E947A8A892F99279F938F93EA
:10F4D0008091C9060E947A8A99279F938F93809181
:10F4E000C1060E947A8A892F99279F938F938091D2
:10F4F000C1060E947A8A99279F938F938CE69FE09A
:10F500009F938F938BEF93E89F938F93E0918E035C
:10F51000F0918F0309958DB79EB7449631C2943010
:10F5200021F486E00E94547184C39630F1F48EE792
:10F530000E94298480E690E09F938F938091CB0670
:10F54000992787FD90959F938F938091C306992764
:10F5500087FD90959F938F9389E89FE09F938F936A
:10F560008BEF93E89F938F93CFC2973008F461C3DA
:10F570008EE70E94298480E690E09F938F9380918C
:10F58000DB06992787FD90959F938F938091D306F3
:10F59000992787FD90959F938F938091CB0699270C
:10F5A00087FD90959F938F938091C306992787FD40
:10F5B00090959F938F938CE99FE09F938F938BEF10
:10F5C00093E89F938F930ECF909146039923F1F187
:10F5D00080917A038823B1F09931A0F487E00E94EA
:10F5E000547183E90E9429848091460399279F934F
:10F5F0008F938FEA9FE09F938F938BE094E89F9384
:10F600008F93D8C083E90E9429848AEB9FE09F935F
:10F610008F930BEF13E81F930F93E0918E03F091FC
:10F620008F0309951F921F929091460381E1989F45
:10F63000C00111248559944F9F938F931F930F936B
:10F64000E0918E03F0918F03099588C083E90E94B1
:10F65000298480EC9FE09F938F938BEF93E8B3C254
:10F660000E946C718093AD0880917409863079F4A2
:10F6700080917503882319F01092750303C081E00F
:10F680008093750385E00E94547186E0BFC2883084
:10F6900031F40E942E8482E080937403C0C28130D2
:10F6A00009F0BFC20E942E8410927403B8C2923037
:10F6B00009F0BDC280917303282F332744275527B3
:10F6C0008F5F80937303F9012131310508F0ACC2DB
:10F6D000EE55FF4F0C94218B80E00E94298489E332
:10F6E00096E09F938F930E94C52F99279F938F93A6
:10F6F00086ED9FE09F938F938BE094E89F938F9389
:10F70000E0918E03F0918F0309952DB73EB7285FE6
:10F710003F4F03C285E10E94298487E496E09F93CE
:10F720008F93809100016AE00E947A8A892F99273D
:10F730009F938F93809100010E947A8A99279F93CB
:10F740008F9385EE9FE09F938F938BEF93E89F932A
:10F750008F93E0918E03F0918F0309958DB79EB73B
:10F760000A960EC18AE20E94298486EF9FE09F9349
:10F770008F93CBEFD3E8DF93CF93E0918E03F0919B
:10F780008F0309958091B6070F900F900F900F90FF
:10F7900080FF4AC08091DB0590917A0181FD14C001
:10F7A000892F99279F938F938BEF9FE09F938F9340
:10F7B000DF93CF93E0918E03F0918F0309952DB7DE
:10F7C0003EB72A5F3F4FA9C1E0918E03F0918F03AE
:10F7D000933318F085E090E102C08CE090E19F93B4
:10F7E0008F93DF93CF9309950F900F900F900F9009
:10F7F00080919A07E0918E03F0918F0390917A01A6
:10F8000080FF0BC0892F99279F938F9383E190E10D
:10F810009F938F93DF93CF93AFC0892F99279F93A7
:10F820008F9389E190E1CFC08FE190E137C08FE302
:10F830000E94298488E290E19F938F93CBEFD3E8D5
:10F84000DF93CF93E0918E03F0918F0309950F9092
:10F850000F900F900F9080913006882319F48CE25E
:10F8600090E11CC080914302E0918E03F0918F03E0
:10F87000882319F085E390E102C08CE390E19F9327
:10F880008F93DF93CF9309950F900F900F900F9068
:10F890008091380686FFCDC183E490E19F938F93DA
:10F8A000DF93CF9392C184E50E9429848AE490E19A
:10F8B0009F938F93CBEFD3E8DF93CF93E0918E03A9
:10F8C000F0918F0309958091B6070F900F900F90DC
:10F8D0000F9085FD03C08FE490E111C080911E065A
:10F8E000883F10F4E82F07C0EFEFF0E0E81BF109C4
:10F8F000E359FD4FE081E23358F488E590E19F93AE
:10F900008F93DF93CF93E0918E03F0918F0316C016
:10F91000E43B18F08FE590E1F2CF80913806E0915A
:10F920008E03F0918F0385FF03C086E690E102C04D
:10F930008DE690E19F938F93DF93CF9309950F907E
:10F940000F900F900F9080913406882309F471C1B5
:10F950008EE50E9429848091340699279F938F9386
:10F9600084E790E19F938F938BEF93E89F938F931E
:10F97000E0918E03F0918F0309958DB79EB706969F
:10F980008DBF57C189E60E9429848FE790E19F933C
:10F990008F93CBEFD3E8DF93CF93E0918E03F09179
:10F9A0008F0309950F900F900F900F908091330661
:10F9B000E0918E03F0918F03882351F099279F9354
:10F9C0008F9389E890E19F938F93DF93CF93F6CE47
:10F9D0008DE890E19F938F93DF93CF93FAC080914E
:10F9E0007703FBEFEF2EF3E8FF2E882309F053C0D7
:10F9F0008EE70E94298480916E0199279F938F93AF
:10FA00008091D005E82FFF27EE0FFF1FE350F94F3D
:10FA1000808191819F938F938091CF05E82FFF275D
:10FA2000EE0FFF1FE350F94F808191819F938F93D9
:10FA300083E990E19F938F93FF92EF92E0918E0381
:10FA4000F0918F03099583E90E9429848DB79EB7B1
:10FA50000A968DBF8091D205E82FFF27EE0FFF1F7A
:10FA6000E350F94F808191819F938F938091D105CD
:10FA7000E82FFF27EE0FFF1FE350F94F80819181A0
:10FA800081589F4F9F938F9387EA90E19F938F9325
:10FA9000FF92EF9235CE8EE70E94298480916F020B
:10FAA00099279F938F9380916E0299279F938F93AD
:10FAB00080916D0299279F938F9386EB90E19F939E
:10FAC0008F93FF92EF92E0918E03F0918F0309954F
:10FAD00083E90E9429848DB79EB70A968DBF8091D5
:10FAE000720299279F938F938091710299279F9318
:10FAF0008F938091700299279F938F938AEC90E166
:10FB00009F938F93FF92EF92E0918E03F0918F037A
:10FB100009952DB73EB7265F3F4F2DBF8AC0809114
:10FB20007A03882309F485C08EE70E942984809196
:10FB3000B60786FD11C08EED90E19F938F938CE107
:10FB400094E89F938F93E0918E03F0918F03099532
:10FB50000F900F900F900F908091360699278F701D
:10FB60009070892B89F08DEE90E19F938F938CE1BB
:10FB700094E89F938F93E0918E03F0918F03099502
:10FB80000F900F900F900F908091B60782FF11C0D9
:10FB900087EF90E19F938F938CE194E89F938F93ED
:10FBA000E0918E03F0918F0309950F900F900F90C5
:10FBB0000F908091B60783FD3CC08CEF90E19F933E
:10FBC0008F938CE194E89F938F93E0918E03F09153
:10FBD0008F0309950F900F900F900F902AC00E94ED
:10FBE0006C718093AD0825C000917409063089F4CA
:10FBF00080917703882319F01092770303C081E086
:10FC00008093770386E00E94547187E00E945471CC
:10FC100008C0013031F40E942E84009374031092C6
:10FC200073031092740905C01092730302C01092FE
:10FC30007403E6E0CDB7DEB70C94128B4FB720E427
:10FC400030E0F8948091C9008F778093C90080914B
:10FC5000C9008F7B8093C9008091C9008F7D8093FC
:10FC6000C9005A9A52985B9A539A832F9927809386
:10FC7000CD002093CC008091C80082608093C800A2
:10FC800088E18093C9008091CA008F778093CA0071
:10FC90008091CA008F7B8093CA008091CA008F7DBB
:10FCA0008093CA008091CA008F7E8093CA008091A1
:10FCB000CA00877F8093CA008091C9008B7F8093A0
:10FCC000C9008091CA0084608093CA008091CA00F4
:10FCD00082608093CA008091C80087FF03C0809132
:10FCE000CE00F9CF8091C90080688093C9004FBFD2
:10FCF00008950F931F93CF93DF93482F4F5F893160
:10FD000008F08BC08091FC06841720F44F5F40936D
:10FD1000FC064150CB0183539B4268E170E00E9496
:10FD20009A8AA42FBB27FD01EA0FFB1FE350F94F6E
:10FD3000808191819B01281B390BC90137FF03C0CA
:10FD4000909581959F4F069794F480916C02883C22
:10FD500030F480916C02865F80936C0208C088EC5E
:10FD600080936C0280916F008F7D80936F00FD0106
:10FD7000EA0FFB1FE350F94F808191819C01220F14
:10FD8000331F280F391F260F371F37FF02C02D5F83
:10FD90003F4FE901D595C795D595C795CB010196FC
:10FDA0008C179D0714F4219706C061507040C61748
:10FDB000D7070CF4219680916C02843BD8F08D011A
:10FDC0000A0F1B1FF801E350F94F80819181FE015A
:10FDD000E81BF90BCF0163E070E00E949A8ACB0127
:10FDE000880F991F860F971F0F5C184FF80191839A
:10FDF000808307C0AA0FBB1FAF5CB84F11961C923F
:10FE00001E92E42FFF27EE0FFF1FE350F94FD1831F
:10FE1000C083443011F410924101DF91CF911F91C2
:10FE20000F910895CF93DF9320917509822F992721
:10FE3000807F9070409709F06CC02F3109F046C068
:10FE40008091760980938103209178092093830320
:10FE50008091790980938203822F99279093FE06DF
:10FE60008093FD06222309F054C08091CF05282FEE
:10FE70003327220F331FF901EF5CF84F11821082F4
:10FE80008091D005A82FBB27AA0FBB1FFD01EF5CF7
:10FE9000F84F118210828091D205E82FFF27EE0FD4
:10FEA000FF1FCF018F5C984FEC01198218822350FD
:10FEB000394FE90119821882A350B94F11961C924B
:10FEC0001E92E350F94F1182108223C0C22FCF70CF
:10FED000CA30F8F4809176098093A109809177095E
:10FEE0008093A009809178098093A3098091790972
:10FEF0008093A2096091A0097091A1098C2F0E94A2
:10FF0000797E6091A2097091A3098C2F8F5F0E9466
:10FF1000797EDF91CF910895CF93C82F8F3F49F419
:10FF2000809184038F3F29F41092860310928503F9
:10FF300032C020918603222339F4CF3111F485E0B9
:10FF400001C084E0809387038091870390918503AB
:10FF50008217A0F4892F8095809385038F3F19F431
:10FF60008EEF8093850380918503C81711F40E945A
:10FF7000127F10928603109285030BC0E22FFF2799
:10FF8000EB58F64FC0832F5F209386039C0F90930E
:10FF90008503C0938403CF91089590918003933299
:10FFA00040F4E92FFF27E358F64F80839F5F90933B
:10FFB00080030895833218F48D5F80938003089541
:10FFC00090E2E0E8F9E08FE19193815087FFFCCF68
:10FFD0000895CF93CFB723E031E0F8948091C90022
:10FFE0008F778093C9008091C9008F7B8093C9006F
:10FFF0008091C9008F7D8093C9005A9A52985B9A6C
:020000021000EC
:10000000539A832F99278093CD002093CC00809121
:10001000C80082608093C80088E18093C900809105
:10002000CA008F778093CA008091CA008F7B80932B
:10003000CA008091CA0080628093CA008091CA0081
:1000400080618093CA008091CA0088608093CA0052
:100050008091C90084608093C9008091CA00846047
:100060008093CA008091CA0082608093CA00809108
:10007000C80087FF03C08091CE00F9CF8091C900EE
:1000800080688093C9008091C90080648093C90012
:100090000E94E07FCFBFCF910895282F99278F70BE
:1000A0009070892B31F4209580917F03822B80936F
:1000B0007F0308958091A401882309F44BC08091A7
:1000C000360285FD04C08091A801882381F082E971
:1000D00080937D0983E280937E098091A801882323
:1000E00009F485E580937F091092A80102C08093EE
:1000F0007D098091A5018F3071F480917F030E946A
:10010000EA6F882341F081E980937D0980937E091D
:1001100081E380937F091092A4018091C80085FF3C
:10012000FCCF8091C9008F7E8093C9008091C90067
:100130008E7F8093C90080917D09882311F48EEF12
:1001400001C08EE78093CE0080917F038093A5014C
:1001500010927F0308951F920F920FB60F921124F1
:100160008F939F93EF93FF939091A401992309F0AC
:1001700040C080918803882361F480917D098823A1
:1001800011F483E003C0813999F481E080938803FE
:100190000FC0833099F480917D09882349F09093B2
:1001A0007D098091C9008E7F8093C9008EEF1EC0AB
:1001B0008091C90081608093C9000EC0833261F4D0
:1001C0008091C9008E7F8093C9008FEF8093CE000D
:1001D00081E08093A40114C080918803E82FFF2759
:1001E000E358F64F8F5F8093880380818093CE0021
:1001F00007C0109288038091C90080618093C90074
:10020000FF91EF919F918F910F900FBE0F901F90D4
:100210001895EF92FF920F931F93CF93DF937C017A
:100220008B01EA01452B39F0F80181918F01F7012B
:1002300009952197C9F7E6E0CDB7DEB70C94128B8C
:10024000EF92FF920F931F93CF93DF937C018B016B
:10025000EA01452B41F0F8010F5F1F4F8491F70130
:1002600009952197C1F7E6E0CDB7DEB70C94128B64
:100270000F931F93CF938C01C62F161634F480E290
:10028000F8010995C1501C16D4F3CF911F910F911D
:1002900008950F931F93CF938C01C62F161634F435
:1002A00080E3F8010995C1501C16D4F3CF911F913A
:1002B0000F910895A5E3B0E0E0E6F1E80C94EA8A36
:1002C0002E96EEADFFAD2E9788249924540180918F
:1002D0007903882321F42C961FAE1EAE2C975EE482
:1002E000452E512C4C0E5D1E6F01B60105C0153216
:1002F00039F00894C11CD11CF60114911123B9F7EF
:10030000A601461B570B31F02C968EAD9FAD2C9756
:100310000E942081112309F46AC20894C11CD11CD7
:10032000FF24FDA6FCA64FEFE42EF9A6F6010894E3
:10033000C11CD11C1491153721F0812F80628837A0
:10034000B1F4F0FE0AC0F20124E030E0420E531E88
:1003500080809180A280B3800AC0F20142E050E028
:10036000440E551E808191814C01AA24BB24103279
:1003700021F489A58823D1F61DC0133219F458E061
:10038000F52AD4CF1A3211F01D3291F41A3259F4F1
:10039000F20182E090E0480E591EE081ECA7EE23C6
:1003A0002CF6E195ECA790E1F92AAFEDFA22BECF49
:1003B0001B3211F419A7BACF1E32C1F5F601089409
:1003C000C11CD11C14911A3279F4F20122E030E000
:1003D000420E531E408151813FEF4F3F530714F4AB
:1003E0004FEF5FEFE42EA2CF40E050E0812F80532B
:1003F0008A30A0F4CA0133E0880F991F3A95E1F7DB
:10040000840F951F480F591F410F511D40535040F5
:10041000F6010894C11CD11C1491E8CF8FEF4F3F17
:10042000580714F44FEF5FEFE42E85CF103329F413
:10043000F4FC7CCF90E2F92A79CF812F8153893067
:10044000D8F440E050E0CA0123E0880F991F2A95B4
:10045000E1F7840F951F480F591F410F511D40535D
:100460005040F6010894C11CD11C1491812F805377
:100470008A3048F34CA75FCF183619F4A4E0FA2A63
:1004800055CF1C3619F4B1E0FB2A50CF133661F476
:100490003E010894611C711CF20122E030E0420E22
:1004A000531E808189833CC1143421F0143611F02D
:1004B000193651F5143411F431E0F32AF0FE0AC074
:1004C000F20144E050E0440E551E80809180A280ED
:1004D000B3800CC0F20182E090E0480E591E80818A
:1004E00091814C01AA2497FCA094BA2CB7FE0AC0B3
:1004F000B094A09490948094811C911CA11CB11C78
:100500008DE289A70AE06FC01F3411F01F3631F465
:100510001F3411F491E0F92A08E064C0103779F42F
:10052000F201A2E0B0E04A0E5B1E808191814C0195
:10053000AA24BB2400E1B0E4FB2A18E753C0133718
:10054000C1F5F20122E030E0420E531E608071805E
:100550006114710489F43E010894611C711C88E2E5
:1005600089838EE6F301818385E78B838CE68C8318
:100570008D8389E28E831F82E7FC13C08E2D99271D
:1005800087FD9095AC0160E070E0C3010E94B788E0
:10059000009729F0382E3618E3140CF0C3C03E2C17
:1005A000C1C0F30101900020E9F731973E2E3618C3
:1005B000B9C0153511F0153731F4153511F4F1E0E6
:1005C000FF2A0AE00FC0183519F0183709F0A0C04B
:1005D00000E1F3FE07C081149104A104B10411F0FD
:1005E00020E4F22A19A6EDA6E7FC02C03FEDF322B3
:1005F00089E2682E712C6C0E7D1E81149104A10479
:10060000B10421F44DA5442309F47BC0802F992720
:10061000AA27BB278EA79FA7A8ABB9AB202E332450
:1006200090E0891690E0990691E0A90690E0B9065D
:1006300048F0C501B4012EA53FA548A959A90E94BB
:10064000AD8A17C0AFEF8A169104A104B10449F036
:1006500040F0C401B1010E94868A9B0144275527BE
:1006600008C0882D602F0E947A8A282F33274427BC
:1006700055272AAB3BAB4CAB5DAB0A3059F48AA98A
:10068000880F880F880F9AA9990F890F382D381B6A
:10069000832F10C0003139F48AA98295807F482DBC
:1006A000481B842F07C08AA9880F880F880F582DF0
:1006B000581B852F90E02EA53FA548A959A9821661
:1006C0009306A406B50608F091E08AA89BA8ACA8FA
:1006D000BDA88A3010F4805D04C0895A183509F429
:1006E0008F7DD3018E933D01992309F099CF083076
:1006F00041F4F3FE06C0803321F080E3FD018293D4
:100700003F01CE010196382E3618F8E23F0E0BC09D
:10071000112309F46CC03E010894611C711C1983FB
:10072000B1E03B2E19A6032D2DA4231827FC22246B
:1007300089A5882311F00F5F02C0F6FC0E5F020D41
:10074000EF2CFF24C70180739070892B49F48CA58E
:10075000801B682F2C968EAD9FAD2C970E94388100
:1007600089A5882331F041E050E0BE01675D7F4FED
:100770000AC0E6FE0EC080E38AA71BA742E050E055
:10078000BE01665D7F4F2C968EAD9FAD2C970E946B
:100790000981C70180739070809749F48CA5801BF4
:1007A000682F2C968EAD9FAD2C970E944981622DAB
:1007B0002C968EAD9FAD2C970E944981832D992751
:1007C00087FD9095AC01B3012C968EAD9FAD2C9713
:1007D0000E940981E4FE89CD2CA5201B2CA7622F45
:1007E0002C968EAD9FAD2C970E9438817ECDE2E194
:1007F000CB5C0C94068B982F80917C09883A50F43E
:1008000080917C09E82FFF27E555F74F93838F5F91
:1008100080937C090895982F80917C09883A58F438
:1008200080917C09E82FFF27E555F74F9068938367
:100830008F5F80937C090895982F80917A03882395
:1008400021F0892F0E940B840895892F0E94FB8339
:100850000895883A10F480937C09089580E090E22E
:10086000EEEAF8E091938F5F883AE0F308954FB78E
:1008700021E830E0F8948091C9008F778093C90017
:100880008091C9008F7B8093C9008091C9008F7DC2
:100890008093C9005A9A52985B9A539A832F99274A
:1008A0008093CD002093CC008091C800826080931B
:1008B000C80088E18093C9008091CA008F77809337
:1008C000CA008091CA008F7B8093CA008091CA00C1
:1008D0008F7D8093CA008091CA008F7E8093CA006A
:1008E0008091CA00877F8093CA008091C90084608C
:1008F0008093C9008091CA0084608093CA0080916F
:10090000CA0082608093CA008091C9008160809390
:10091000C9008091C80087FF03C08091CE00F9CF45
:100920008091C90080688093C9004FBF3CE7309335
:1009300052082DE7209377088EE880935308109291
:100940006C0810926B081092550830939A08209307
:10095000AA081092A4081092A3081092A608109258
:10096000A5081092A8081092A70884EF91E0909330
:10097000A2088093A1089093A00880939F08909369
:100980009E0880939D0810929C0889E880939B089C
:100990001092A908309357092093730910925909AE
:1009A0008AE88093580910925C0910925B091092B2
:1009B0005A0910925E0910925F0910926009109214
:1009C00061091092630910926409109265091092EE
:1009D000660910926A0910926909109268091092CA
:1009E0006709309378082093990810927A088DE867
:1009F000809379088BE78093AB0880E88093AC08FC
:100A00001092AD088091550890E2EEEAF8E09193DB
:100A10008F5F883AE0F38DE7809356090895CF936E
:100A2000C82F80918903803879F48C2F0E9420721E
:100A300080937C0380917C03882309F1C0937B0918
:100A400080917C038F5F11C08F37C9F48091740946
:100A5000882321F48C2F8095809374098BEA98E089
:100A600090937E0380937D038DEA80937C03809135
:100A7000C9008F7E8093C90082E080937B03C0937E
:100A80008903CF91089530917B03332331F0809116
:100A90007B03815080937B03089580917C0388239E
:100AA00081F140917C0390918A03413091F4292F88
:100AB00030938A038091C90080618093C90080913E
:100AC0007A03882319F030937A0310C040937A0395
:100AD0000DC0E0917D03F0917E038191F0937E0340
:100AE000E0937D03282F980F90938A038091C8008C
:100AF00085FFFCCF2093CE0080917C0381508093B2
:100B00007C0308952FB740E0F894E0E0F0E081E244
:100B1000809357009491E2E0F0E080935700349185
:100B2000E4E0F0E08093570084912FBF9E3199F468
:100B3000363941F4893011F441E00DC08A3059F45E
:100B400042E009C0373939F4863011F443E003C07C
:100B5000853009F444E0842F992708959FB7F894CD
:100B60008091C900877F8093C9008091C9008F7EE2
:100B70008093C9008091C9008F778093C9008091CC
:100B8000C9008F7B8093C9008091C9008F7D8093BD
:100B9000C90052985A9A53985B9A9FBF08951F9321
:100BA000CF93DF93182F80917903882309F4AEC087
:100BB0008091A301181709F4A9C0809178038823B4
:100BC00021F40E9482858093780382ED91E09093D6
:100BD000400180933F0184E092E19F938F93C2E9AB
:100BE000D5E1DF93CF93E0918E03F0918F030995C8
:100BF0000F900F900F900F90812F992783309105C0
:100C000039F1843091054CF48130910591F08230B6
:100C10009105DCF4892B51F036C085309105F1F057
:100C200085309105C4F00697E1F02DC084EF91E185
:100C300002C082EE91E19F938F93DF93CF93E09177
:100C40008E03F0918F0309952AC089EC91E1F3CFCF
:100C500086EA91E1F0CF88E991E1EDCF80E991E179
:100C6000EACF82E891E19F938F93DF93CF93E09156
:100C70008E03F0918F03099588ED91E090934001E8
:100C800080933F010CC081E192E19F938F93DF93AA
:100C9000CF93E0918E03F0918F03099510E00F90B0
:100CA0000F900F900F9080917803843011F0823074
:100CB000C1F40E94AE85812F8150833018F40E94C8
:100CC000EE6A22C0143019F40E94E97F1DC015306D
:100CD00019F40E941E7E18C01630B1F40E943784A9
:100CE00013C0112389F087E292E19F938F9382E9E9
:100CF00095E19F938F93E0918E03F0918F03099577
:100D00000F900F900F900F901093A301DF91CF9150
:100D10001F9108950F931F9381E080937903409171
:100D2000A201E2E3F1E120E030E05FE48491992761
:100D30002F5F3F4F829FB001839F700D929F700D78
:100D4000112446275150319657FFF0CF4093A2010E
:100D5000EAE0F1E120E030E057E2849199272F5F4B
:100D60003F4F829FB001839F700D929F700D1124A1
:100D700046275150319657FFF0CF4093A201809102
:100D80007803882321F40E948285809378038091E0
:100D9000A201833459F088E190E029E20FB6F8947B
:100DA000A895809360000FBE209360008AE591E8CB
:100DB00090938F0380938E0382E492E19F938F93AD
:100DC00002E915E11F930F93E0918E03F0918F03D9
:100DD00009950F900F900F900F9084E690E09F93ED
:100DE0008F9386E590E09F938F931F921F9280913F
:100DF00002016AE00E947A8A892F99279F938F9334
:100E0000809102010E947A8A99279F938F9388E6A6
:100E100092E19F938F931F930F93E0918E03F09134
:100E20008F03099582E391E19F938F931F930F9313
:100E3000E0918E03F0918F0309958AE091E19F93F1
:100E40008F931F930F93E0918E03F0918F03099579
:100E50008DB79EB746968DBF8CE992E19F938F9395
:100E60001F930F93E0918E03F0918F03099582EC0D
:100E70008093810080916F00806280936F000F905B
:100E80000F900F900F901F910F910895809134064D
:100E90008F3138F08091D10787FD03C08EE18093B8
:100EA00034068091E405882331F08055853618F0AA
:100EB0008FE78093E405089580917903882309F4EE
:100EC00073C080918B03815080938B03882309F03A
:100ED0004FC089E180938B0380913406803238F0D3
:100EE0008091D10787FD03C08FE180933406809104
:100EF0006C02823800F58091370290913802885E4A
:100F0000934020F410928D0310928C0380918C03F7
:100F100090918D03009739F1019790938D03809301
:100F20008C03419728F18091D10784FF21C08091E3
:100F3000350284601BC080916C02853BC8F09091A3
:100F4000340684E1989FC0011124409620918C03BF
:100F500030918D032817390730F42F5F3F4F3093BE
:100F60008D0320938C03809135028B7F8093350213
:100F70009091A301963019F40E9443850FC080918F
:100F8000A601882321F081508093A601089586E967
:100F90008093A601943011F40E945A808091A2019E
:100FA000833411F01092790308951F920F920FB6B7
:100FB0000F9211242F933F934F935F936F937F93DF
:100FC0008F939F93AF93BF93EF93FF932091CE00A6
:100FD0008091B2018823B1F02093C6008091B201C4
:100FE000823059F52F3F49F58FEF94E3ACE0B0E044
:100FF000C297A109B109B7FFFBCF8091D1038093BC
:10100000CE001BC09091A301892F8150833020F422
:10101000822F0E94496B11C0943021F4822F0E94CC
:101020004D800BC0953021F4822F0E948C7F05C02B
:10103000963019F4822F0E940F85FF91EF91BF9196
:10104000AF919F918F917F916F915F914F913F9160
:101050002F910F900FBE0F901F90189500242227FC
:101060003327442751E0BB27EE27FF27A0E1660F77
:10107000771F881F991F001C221F331F441F660FF4
:10108000771F881F991F001C221F331F441F2AF43B
:10109000050E2B1F3E1F4F1F04C0051A2B0B3E0BC6
:1010A0004F0B550FBB1FEE1F587F556047FD525029
:1010B000AA95E9F6E695B7955795E695B7955795AC
:1010C000852F9B2F08952227332741E0552768E07D
:1010D000880F991F221F331F880F991F221F331F4C
:1010E0001AF4240F351F02C0241B350B440F551F63
:1010F000487F456037FD42506A9551F756954795B0
:1011000056954795842F0895AA2797FF04C0809588
:1011100090958A1F9A1F77FF04C0609570956A1F8B
:101120007A1F669F9001779FA001679F300D411D38
:101130005A1F300D411D5A1F889FF001999F2E0F95
:101140003F1F401D511D899F300D411D5A1F300DFD
:10115000411D5A1FCA01B901112480CFFB01DC01D6
:1011600002C005900D9241505040D8F70895FC01FF
:101170004150504030F001900616D1F73197CF0121
:101180000895882799270895A0E0B0E0EAECF8E8F0
:101190000C94F28A6C017B01EA01590121978FEFCF
:1011A000CF3FD80789F086010894C11CD11CC70124
:1011B0000894E11CF11CF5010995F8018083219741
:1011C000FFEFCF3FDF0779F7EAE0CDB7DEB70C944A
:1011D0000E8BCF92DF92EF92FF920F931F937C01C1
:1011E0006B01FB010995082FC7010196F6010995CE
:1011F000182FC8011F910F91FF90EF90DF90CF90B3
:101200000895A0E0B0E0E7E0F9E80C94F48A8C01DE
:101210007B01EA01690121978FEFCF3FD80771F079
:10122000F70121917F01C8010F5F1F4F622FF60167
:1012300009952197FFEFCF3FDF0791F7E8E0CDB7A2
:10124000DEB70C94108BCF92DF92EF92FF920F9348
:101250001F936C018B017A01FA010995812F99275F
:10126000682FC6010196F70109951F910F91FF9014
:10127000EF90DF90CF9008955058BB27AA270ED04B
:10128000E0C0D1D030F0D6D020F031F49F3F11F43F
:101290001EF4C6C00EF4E095E7FBBCC0E92FE2D017
:1012A00080F3BA17620773078407950718F071F483
:1012B0009EF5FAC00EF4E0950B2EBA2FA02D0B016F
:1012C000B90190010C01CA01A0011124FF27591B8B
:1012D00099F0593F50F4503E68F11A16F040A22F91
:1012E000232F342F4427585FF3CF46953795279502
:1012F000A795F0405395C9F77EF41F16BA0B620B01
:10130000730B840BBAF09150A1F0FF0FBB1F661F47
:10131000771F881FC2F70EC0BA0F621F731F841F8A
:1013200048F4879577956795B795F7959E3F08F0B0
:10133000B3CF9395880F08F09927EE0F979587956F
:10134000089598D088F09F5790F0B92F9927B751FA
:10135000A0F0D1F0660F771F881F991F1AF0BA9579
:10136000C9F712C0B13081F09FD0B1E008959CC0A0
:10137000672F782F8827B85F39F0B93FCCF386956F
:1013800077956795B395D9F73EF4909580957095CC
:1013900061957F4F8F4F9F4F0895E89409C097FB49
:1013A0003EF490958095709561957F4F8F4F9F4F3C
:1013B0009923A9F0F92F96E9BB279395F695879580
:1013C00077956795B795F111F8CFFAF4BB0F11F443
:1013D00060FF1BC06F5F7F4F8F4F9F4F16C08823EA
:1013E00011F096E911C0772321F09EE8872F762F20
:1013F00005C0662371F096E8862F70E060E02AF061
:101400009A95660F771F881FDAF7880F969587954C
:1014100097F9089597F99F6780E870E060E0089574
:101420009FEF80EC089500240A94161617061806FC
:101430000906089500240A941216130614060506D8
:101440000895092E0394000C11F4882352F0BB0F69
:1014500040F4BF2B11F460FF04C06F5F7F4F8F4FCC
:101460009F4F089557FD9058440F551F59F05F3F07
:1014700071F04795880F97FB991F61F09F3F79F0B6
:1014800087950895121613061406551FF2CF469538
:10149000F1DF08C0161617061806991FF1CF8695BA
:1014A0007105610508940895E894BB27662777279E
:1014B000CB0197F90895629FD001739FF001829F3D
:1014C000E00DF11D649FE00DF11D929FF00D839FD3
:1014D000F00D749FF00D659FF00D9927729FB00D70
:1014E000E11DF91F639FB00DE11DF91FBD01CF0183
:1014F00011240895991B79E004C0991F961708F0EC
:10150000961B881F7A95C9F780950895AA1BBB1B67
:1015100051E107C0AA1FBB1FA617B70710F0A61BF3
:10152000B70B881F991F5A95A9F780959095BC0114
:10153000CD01089597FB092E07260AD077FD04D028
:10154000E5DF06D000201AF4709561957F4F08956D
:10155000F6F7909581959F4F0895A1E21A2EAA1B48
:10156000BB1BFD010DC0AA1FBB1FEE1FFF1FA21753
:10157000B307E407F50720F0A21BB30BE40BF50B50
:10158000661F771F881F991F1A9469F760957095D9
:10159000809590959B01AC01BD01CF01089597FB0B
:1015A000092E05260ED057FD04D0D7DF0AD0001C27
:1015B00038F450954095309521953F4F4F4F5F4FF0
:1015C0000895F6F790958095709561957F4F8F4FB0
:1015D0009F4F08952F923F924F925F926F927F920A
:1015E0008F929F92AF92BF92CF92DF92EF92FF9233
:1015F0000F931F93CF93DF93CDB7DEB7CA1BDB0BDF
:101600000FB6F894DEBF0FBECDBF09942A88398883
:1016100048885F846E847D848C849B84AA84B9848A
:10162000C884DF80EE80FD800C811B81AA81B98196
:10163000CE0FD11D0FB6F894DEBF0FBECDBFED01AA
:101640000895EE0FFF1F0590F491E02D0994FFCF50
:101650005E010A010164FF01FFFFC01FC01F0101FD
:1016600001737373FF03007D0000C409C4096400A3
:10167000104661737400004E6F726D616C0000451E
:10168000617379000051756164726F00006400D26B
:101690000101200B050000ECFF000204060708080A
:1016A000080706040200FEFCFAF9F8F8F8F9FAFC5B
:1016B000FE000204060708086440415A4664640AB2
:1016C00002969696960840403A10FB30380132FF59
:1016D00003780090D0030090D0030032002064FF14
:1016E000FF64200B0A0D0B0C0E0B0F10FA200101EA
:0816F000010170FF010F64000D
:00000001FF
